:0200000280007C
:100000003DB8F3960000000000020000F806020070
:1000100000000000000000000000000000000000E0
:10002000FFFFFFFFFFFFFFFFFFFFFFFFFFFFFFFFE0
:10003000FFFFFFFFFFFFFFFFFFFFFFFFFFFFFFFFD0
:10004000FFFFFFFFFFFFFFFFFFFFFFFFFFFFFFFFC0
:10005000FFFFFFFFFFFFFFFFFFFFFFFFFFFFFFFFB0
:10006000FFFFFFFFFFFFFFFFFFFFFFFFFFFFFFFFA0
:10007000FFFFFFFFFFFFFFFFFFFFFFFFFFFFFFFF90
:10008000FFFFFFFFFFFFFFFFFFFFFFFFFFFFFFFF80
:10009000FFFFFFFFFFFFFFFFFFFFFFFFFFFFFFFF70
:1000A000FFFFFFFFFFFFFFFFFFFFFFFFFFFFFFFF60
:1000B000FFFFFFFFFFFFFFFFFFFFFFFFFFFFFFFF50
:1000C000FFFFFFFFFFFFFFFFFFFFFFFFFFFFFFFF40
:1000D000FFFFFFFFFFFFFFFFFFFFFFFFFFFFFFFF30
:1000E000FFFFFFFFFFFFFFFFFFFFFFFFFFFFFFFF20
:1000F000FFFFFFFFFFFFFFFFFFFFFFFFFFFFFFFF10
:10010000FFFFFFFFFFFFFFFFFFFFFFFFFFFFFFFFFF
:10011000FFFFFFFFFFFFFFFFFFFFFFFFFFFFFFFFEF
:10012000FFFFFFFFFFFFFFFFFFFFFFFFFFFFFFFFDF
:10013000FFFFFFFFFFFFFFFFFFFFFFFFFFFFFFFFCF
:10014000FFFFFFFFFFFFFFFFFFFFFFFFFFFFFFFFBF
:10015000FFFFFFFFFFFFFFFFFFFFFFFFFFFFFFFFAF
:10016000FFFFFFFFFFFFFFFFFFFFFFFFFFFFFFFF9F
:10017000FFFFFFFFFFFFFFFFFFFFFFFFFFFFFFFF8F
:10018000FFFFFFFFFFFFFFFFFFFFFFFFFFFFFFFF7F
:10019000FFFFFFFFFFFFFFFFFFFFFFFFFFFFFFFF6F
:1001A000FFFFFFFFFFFFFFFFFFFFFFFFFFFFFFFF5F
:1001B000FFFFFFFFFFFFFFFFFFFFFFFFFFFFFFFF4F
:1001C000FFFFFFFFFFFFFFFFFFFFFFFFFFFFFFFF3F
:1001D000FFFFFFFFFFFFFFFFFFFFFFFFFFFFFFFF2F
:1001E000FFFFFFFFFFFFFFFFFFFFFFFFFFFFFFFF1F
:1001F000FFFFFFFFFFFFFFFFFFFFFFFFFFFFFFFF0F
:1002000090800020DD02010003350200B1020100F0
:10021000B1020100B1020100B1020100B10201000E
:100220000000000000000000000000009DFD000034
:10023000B10201000000000045FD0000B102010014
:100240001DFE00001DFE00001DFE00001DFE000042
:100250001DFE00001DFE00001DFE00001DFE000032
:100260001DFE00001DFE00001DFE00001DFE000022
:100270001DFE00001DFE00001DFE00001DFE000012
:100280001DFE00001DFE00001DFE00001DFE000002
:100290001DFE00001DFE00001DFE00001DFE0000F2
:1002A0001DFE00001DFE00001DFE00001DFE0000E2
:1002B0001DFE00001DFE00001DFE00001DFE0000D2
:1002C0001DFE00001DFE00001DFE00001DFE0000C2
:1002D0001DFE00001DFE00001DFE00001DFE0000B2
:1002E0001DFE00001DFE00001DFE00001DFE0000A2
:1002F0001DFE00001DFE00001DFE00001DFE000092
:100300001DFE00001DFE00001DFE00001DFE000081
:100310001DFE00001DFE00001DFE00001DFE000071
:100320001DFE00001DFE00001DFE00001DFE000061
:100330001DFE00001DFE00001DFE00001DFE000051
:100340001DFE00001DFE00001DFE00001DFE000041
:100350001DFE0000FFFFFFFF53B94AB9002908BF87
:1003600000281CBF4FF0FF314FF0FF3000F00CB8F9
:10037000ADF1080C6DE904CE00F008F8DDF804E0FA
:10038000DDE9022304B07047704700BF2DE9F04754
:1003900086468C460846089E154674461946002B2C
:1003A00040F0C1808542B2FA82F245D94AB1C2F129
:1003B000200300FA02FC954094402EFA03F343EA2E
:1003C0000C0C4FEA154EA8B2230CBCFBFEF80EFB3A
:1003D00018CC08FB00F943EA0C43994528D9EB18DF
:1003E00008F1FF3704D2994502D9A8F102072B443E
:1003F000A3EB0903A4B2B3FBFEFC0EFB1C330CFB06
:1004000000F044EA0344A04214D92C190CF1FF3344
:1004100004D2A04202D9ACF102032C44241A43EACC
:1004200007401EB1D440002334607360BDE8F087FC
:100430004746DDE76346F1E792BB431B01214FEAE4
:10044000154EAFB2200CB3FBFEFC0EFB1C330CFBB5
:1004500007F840EA0343984561D9EB180CF1FF30E7
:1004600004D2984502D9ACF102002B44A3EB080357
:10047000A4B2B3FBFEFC0EFB1C330CFB07F744EAF3
:100480000344A7424DD92C190CF1FF3304D2A742E3
:1004900002D9ACF102032C44E41B43EA0040C0E75C
:1004A000C2F120039540944020FA03F12EFA03F3A1
:1004B0004FEA154E9040AFB20343B1FBFEFC0EFB7A
:1004C0001C10190C0CFB07F841EA0041884522D9A1
:1004D00069180CF1FF3004D2884502D9ACF1020052
:1004E0002944A1EB08019BB2B1FBFEFC0EFB1C11E1
:1004F0000CFB07F743EA01439F420ED9EB180CF1BE
:10050000FF3104D29F4202D9ACF102012B44DB1B24
:1005100041EA004193E76046E3E76146F7E760465A
:10052000A4E76346B8E7834206D916B90021084616
:100530007CE7C6E900E0F9E7B3FA83F78FB98342B5
:1005400001D3724508D8BEEB020460EB030301201F
:100550009C461EB9002169E73846FAE7C6E9004C17
:10056000F8E7C7F1200CBB400EFA07F522FA0CF4AD
:100570002EFA0CF1BA401C4320FA0CF3B8404FEAB3
:10058000144901431FFA84FEB3FBF9F809FB183044
:100590000B0C08FB0EFA43EA00439A4540D9E318D6
:1005A00008F1FF3004D29A4502D9A8F10200234491
:1005B000A3EB0A0389B2B3FBF9F809FB183308FB74
:1005C0000EFE41EA03418E452CD9611808F1FF3334
:1005D00004D28E4502D9A8F10203214443EA004027
:1005E000A1EB0E01A0FB02984145CE46434602D343
:1005F00006D14D4504D20138B9EB020E68EB040375
:10060000002EA7D0B5EB0E0261EB030101FA0CFC42
:1006100022FA07F3F9404CEA0303C6E9003199E7EF
:100620004046C5E74346D9E72DE9F3415B4DD5F890
:100630006031996811F001011AD140F6034001AA16
:1006400004F02EFE0446002840F0A3800198C36801
:100650001B785BB905F1CC03D3E8AF2F02F0090298
:10066000D3E8EF1FC3E8E42F002CF9D10DF03AF8DE
:10067000002141F2030001AA04F012FE0446002802
:1006800040F08780019E0822F1684548013117F04B
:1006900037F830460DF026F8214641F2010001AA54
:1006A00004F0FEFD0446002873D10198C3685A780F
:1006B00085F868205A88A5F86A201A7985F8692093
:1006C000B3F80720A5F86C20B3F80530A5F86E3014
:1006D0000DF008F8214641F2020001AA04F0E0FD05
:1006E0000446002855D1019C4022E1682D48013183
:1006F00017F006F820460CF0F5FF06F007FA04465E
:10070000002846D195F882309A0638D5072140F660
:10071000334004F07BFD0746002800F04D8107219F
:100720000C300DF0E5F821460722064616F0F3FFDF
:100730006FF009034FF0010833700623224634712D
:10074000394640F6334086F80180F37004F0A8FD86
:100750000446F0B9414640F6314004F057FD0646E4
:10076000002800F0298141460C3019F08FFB224609
:10077000314640F6314004F093FD044648B995F8FF
:1007800074305B0612D44521074815F072FC6FF0F7
:100790001204204602B0BDE8F08100BF0020002016
:1007A0007020002078200020109E0200002142F2DC
:1007B000030001AA04F074FD04460028E9D1019E5B
:1007C0000822F168B848013116F09AFF30460CF063
:1007D00089FF214642F2020001AA04F061FD0446AD
:1007E0000028D6D1019CE368B3F8012091B2A5F8A6
:1007F000FC2021B1DA78AD4811461AF061FF20469D
:100800000CF070FF95F8746016F0200618D10221E4
:1008100040F66D4004F0FAFC0446002800F0CC805D
:1008200002210C300DF064F801232146037046705C
:10083000324640F66D4004F033FD04460028A8D14E
:1008400095F894301F0712D5002142F21C0001AA2E
:1008500004F026FD044600289BD10198C368D3F814
:100860000120D3F80530C5E936230CF03BFF95F89D
:10087000D0309E0624D568460DF1020104F068FDD3
:100880000446002885D1042142F2240004F0BEFC75
:100890000646002800F0908004210C300DF028F866
:1008A000BDF8003022460380BDF802303146438057
:1008B00042F2240004F0F4FC044600287FF469AFFF
:1008C00095F8D0305C0610D5002142F22A0001AA2A
:1008D00004F0E6FC044600287FF45BAF0198C3688F
:1008E0005B7885F818310CF0FDFE082142F201001A
:1008F00004F08CFC044600285ED008210C300CF07B
:10090000F7FF95F8D01040F2022311F0400F08BF16
:100910000323024688074CBF43F02C0043F00C0031
:1009200095F8D1308F0648BF40F0400013F0090F12
:1009300095F89A3018BF40F4006003F00603CE0724
:1009400048BF40F01000062B08BF40F4C0700021E3
:1009500016F0DDFF2146002242F2010004F0A0FC67
:10096000044600287FF415AF95F87430B5F8FC10F4
:10097000980624D4C9B941F2050001AA04F090FCFC
:10098000044600287FF405AFB5F8FC30019C4BB954
:10099000E368B3F80120A5F8FC209A884348114683
:1009A0001AF08EFE20460CF09DFE082140F6014014
:1009B00004F02CFC044658B96FF06804E9E60029FD
:1009C000F3D145213A4815F054FB6FF00404E0E6FA
:1009D00008210C300CF08CFF95F8D0300246D90776
:1009E00057D44FF00051334816F091FF21460022B2
:1009F00040F6014004F054FC044600287FF4C9AEE0
:100A0000014601AA4FF6014004F04AFC044648BBE7
:100A100001980CF067FE21464FF6024001AA04F04F
:100A20003FFC0446F0B9019E0222F16822480131E0
:100A300016F066FE30460CF055FE95F8B9305B07AF
:100A400010D521464FF6034001AA04F029FC48B90D
:100A50000122019C1948E168114416F051FE20461C
:100A60000CF040FE17F0BDF8044600287FF491AE6C
:100A700007F09EF8044600287FF48BAEEB79002B3C
:100A80003FF487AE08210E4816F02DFF05F002F95D
:100A90007FE603A1D1E90001A6E700BFAFF3008024
:100AA0009088000200800020D0200020002100203B
:100AB000399E020010880002B9200020B8200020D2
:100AC000CC200020014B1878704700BF384600202A
:100AD00008B5044814F0F7FFBDE80840012019F0FC
:100AE0006ABC00BF568A020008B521B1BDE80840C3
:100AF000054814F0E8BF054814F0E5FFBDE80840DC
:100B0000012019F055BC00BF708A02008C8A0200D7
:100B1000CB0710B506D500F00104204602F092FD87
:100B2000014B1C7010BD00BF3846002070B5037823
:100B30008AB004460E4607AD032B20D8DFE803F049
:100B400002191B1D1149284616F066FD05956378AC
:100B50001E210493A37830460393E3780C4A029352
:100B60002379019363790093A37914F0B9FF0AB054
:100B700070BD0849E7E70849E5E70849E3E70A21C6
:100B80002846074A14F0ACFFE0E700BF978A02004E
:100B9000C08A02009E8A0200A58A0200AF8A020073
:100BA000B98A020030B5154689B00C4617F000FA34
:100BB0006946FFF7BBFF35B922466946054814F080
:100BC00082FF09B030BD2B4622466946024814F028
:100BD0007AFFF6E7E38A0200028B020010B50C46AA
:100BE00088B017F0E5F96946FFF7A0FF224669468D
:100BF000024814F068FF08B010BD00BF278B020048
:100C000010B50C4688B017F0D3F96946FFF78EFF90
:100C100022466946024814F056FF08B010BD00BFD6
:100C20004B8B020000B589B017F0C2F96946FFF797
:100C30007DFF6946024814F046FF09B05DF804FBE9
:100C40006E8B020010B50C4688B017F0B1F96946FA
:100C5000FFF76CFF22466946024814F034FF08B0E3
:100C600010BD00BF858B020030B5304889B014F04C
:100C70002AFF0EF085FE014628B12D4809B0BDE8D7
:100C8000304014F020BF2B480EF0AAFE044648B9AD
:100C9000294806F057FF60B1284809B0BDE8304048
:100CA00014F011BF0146264814F00DFF21462548D7
:100CB000E4E7254806F060FF08B12448EDE704F0BA
:100CC000FBFF014608B12248D8E7224814F0FBFE9A
:100CD00015F0C6FE204802F0ABFC014608B11F48E3
:100CE000CCE71F4D03AC0FCD0FC42B68022223604D
:100CF00001231C49009303A81B4B05F003FE044687
:100D000028B10146194814F0DEFE09B030BD18487C
:100D100014F0D9FE013404F0010100200EF0F0FEC1
:100D200000214FF4803013F015FDF3E79B8B020098
:100D3000C78B020011CB0000802100201E8C020016
:100D4000E28B0200018C0200702100204B8C02001B
:100D50007D8C02009D8C020068210020B48C020072
:100D6000D07F02009080020088800200D18C0200B7
:100D7000F78C0200014B1B68184700BF9821002028
:100D8000014B1860704700BF9821002007B50B4643
:100D9000002102460091034800F0E2FB03B05DF839
:100DA00004FB00BF75CD000030B5002587B0CDE94C
:100DB00003010446009503A90548059500F0D0FB02
:100DC000DDE904309842B8BF255407B030BD00BFFC
:100DD000A11A020070B589B306680122304614F0EA
:100DE000CEFE01460446304614F091FEC30708D4F7
:100DF0001349AF22134815F028F9AF21104815F018
:100E00001DF92146304614F098FE25182946002287
:100E1000304614F07CFE2D1AAC4206D00849B722A9
:100E2000084815F012F9B721E8E72146304614F0DA
:100E30008AFE2146BDE8704014F0C6BF70BD00BFF9
:100E4000358D0200568D02002DE9F8430F460668E5
:100E50001446B2684B1EB2F5004F34BF042108217E
:100E60003B4010D0C7F1000909EA0709494503F1E1
:100E7000FF3028BF494618420CD11F46BCB9002597
:100E80002846BDE8F8838F420FD82146BDE8F843D5
:100E900014F0DCBF2C492D484FF4A27215F0D5F8A0
:100EA0004FF4A271284815F0C9F89946E6E7B2EB6D
:100EB000D40FE4D9E319591A104614F06AFE01461A
:100EC000304614F0C0FE80460028D8D0B36809EB45
:100ED000C005B3F5004F34BF042308231D44354437
:100EE0007B1E1D447F423D40A5EB09052946304647
:100EF00014F045FE2C44073424F00704A41B80455D
:100F000007464FEAE40408D202464146304614F050
:100F1000D4FE4146304614F015FF3946304614F0F1
:100F20000CFE3844844208D239463046224614F03A
:100F3000C4FE2146304614F005FF012239463046F2
:100F400014F001FE9CE700BF358D0200568D0200B3
:100F5000B2F5802FF8B50CD2042A20D83B494FF4C3
:100F6000F9723B4815F071F84FF4F971374815F0F4
:100F700065F80823D21ACC1D114424F0070421F08F
:100F80000701091B17294FEAD1060AD82F4940F259
:100F9000FB122F4815F059F840F2FB11E6E7042345
:100FA000E8E70027046031463046A660E76014F0A9
:100FB000F9FD012185000246304614F0EAFD1B359B
:100FC000ED082844B04234D83B46384604F10C01C1
:100FD0009A4237DA2A462046002114F0CCFD00233D
:100FE00020461A46194614F09DFD771B19462046E7
:100FF000012214F0A8FD3A46294614F0BCFD2B4608
:1010000000222946204614F08DFD3146204614F07A
:10101000B2FD3B4631462046002214F083FD3146A6
:101020002046012214F08FFD2946BDE8F84014F057
:1010300089BE06494FF40372054815F006F84FF4CF
:10104000037193E741F8040F0133C1E7358D0200C6
:10105000568D02002DE9F84F0446A38B0846190768
:10106000164612D4022803F0070162D1204614F07C
:101070001FFF88B10138042800F22181DFE810F059
:1010800059001F017E00C400F10001280CBF43F08D
:10109000100143F02001A18304F1140011F056FC6B
:1010A000002800F0A98086F31188BFF36F8FBDE898
:1010B000F88F03F00702501F01281ED80020062ACF
:1010C0002768C4E9000014D13A4603E0E08B013000
:1010D000E0831268002AF9D123F0070343F00202EB
:1010E0002046A28314F0E4FE90B342F02002A283D3
:1010F0002EE023F007039AB2F2E7042A33D123F05B
:1011000007039AB22046A28314F0D2FE10B142F037
:101110002002A283A38B03F00709894540F0D88001
:10112000A18BCA0640F11E8121F01003A38301F0B8
:101130000701D4F81880A38BB8F1000FB9DA0022A8
:10114000276823F00703C4E9002243F00103A383C7
:10115000A38B03F00709894540F0BB80002FDFD047
:101160000025AA463EE0844940F21B12834814F051
:101170006CFF40F21B11804814F060FF41B17E49C2
:101180004FF4AB727D4814F060FF4FF4AB71F2E79F
:10119000236843B9784940F25712784814F055FF54
:1011A00040F25711E7E723691D6845B972494FF4CA
:1011B000AD72724814F049FF4FF4AD71DBE70F4692
:1011C00088464FF00609A38B23F0070343F006037C
:1011D0009BB2A383A268002A7DD1002F7ED1002D6F
:1011E0009ED0BA4643F0080304F1140B5846A3837B
:1011F00011F0ACFB002873D16149C2225F4814F0A2
:1012000024FFC2215E48B7E7022908D05A4940F2BC
:101210005D125A4814F019FF40F25D11ABE7E78BFD
:1012200047B155494FF4AF72544814F00EFF4FF4D4
:10123000AF71A0E723695D6845B94F4940F261127B
:101240004E4814F002FF40F2611194E7A38BB846B8
:1012500023F0070343F004039BB24FF00409A38378
:10126000B8E7012908D044494FF4B272434814F05A
:10127000ECFE4FF4B2717EE7236843B93E4940F279
:1012800065123E4814F0E1FE40F2651173E72369F0
:101290009D6845B938494FF4B472384814F0D5FE0A
:1012A0004FF4B47167E70027A38BB84623F0070318
:1012B00043F005039BB24FF00509A3838AE72E494B
:1012C00040F26B122D4814F0C0FE40F26B1152E751
:1012D000002700257EE74FF0010A83E7924681E769
:1012E00086F31188BFF36F8FBAF1000F17D14FBB90
:1012F00015B120462349A8474FF02003EFF311868C
:1013000083F31288BFF36F8F584611F011FB08BBAF
:101310001B499422194814F098FE942172E7A168A1
:101320000029E4D00E680029E1D043464A46204611
:10133000D1F804A0D0471EB1336831461E46F2E70B
:101340003346FAE7394643464A4620463F6814F09A
:10135000DBFDCCE7584611F007FBA38B23F0080315
:10136000A383DDE68B067FF597AE21F02003A383F0
:1013700001F007017AE600BF6E8D0200568D020073
:10138000908D020089D30000F8B504460D4600F1A7
:1013900014064FF02003EFF3118783F31288BFF395
:1013A0006F8F304611F0C4FA40B90A490A489422B6
:1013B00014F04BFE9421074814F040FE304611F023
:1013C000D3FAA5613A462046BDE8F8400121FFF76F
:1013D00041BE00BF908D0200568D02002DE9F047FE
:1013E00004460F4614F080FD051E5CDB04F1140971
:1013F0004FF02003EFF3118A83F31288BFF36F8F4E
:10140000484611F095FA804638B93249942232485C
:1014100014F01BFE94212F483AE0484611F0A4FA3C
:101420004FF6FF72E38BA68B934206F007063DD082
:10143000022E0ED135460133E383484611F086FA79
:10144000002839D12349C222234814F0FEFDC221CD
:10145000E1E7062E13D8DFE806F0092C1212090482
:1014600009006FF085054FF00008E6E700233B60B8
:1014700063687BB9C4E900777EB13546F3E7174965
:1014800015484FF4E47214F0E0FD4FF4E471134892
:1014900014F0D4FD1F606760EEE75246022120463B
:1014A000FFF7D8FD35462846BDE8F0876FF00A05FE
:1014B000D9E76FF00405D6E78AF31188BFF36F8F81
:1014C000B8F1000FEFD0002332463946204614F021
:1014D0001BFDE8E7908D0200568D02006E8D020024
:1014E00008B54268034602F00302022A81600AD06E
:1014F000032A4FF0000103D0012A0AD1596006E007
:101500001868596008BD186800225A6050B9002058
:10151000F8E706490648452214F097FD452103489F
:1015200014F08CFD13F0F4FFF1E700BFBD8D020055
:10153000568D020010B5094C0A44914200D110BDED
:1015400011F8013B58400309E35C0001C0B243407D
:101550001809205C1B01DBB25840EEE7E08D020069
:101560002DE9F04F81468B4617461C46002595B065
:10157000387808B9284657E37B1C2528039306D002
:101580005946C8470028C0F24F830135FBE11822B5
:1015900000210EA816F0BFF87B78252B7DD0002304
:1015A00098469E469C461E46781C014610F8012B24
:1015B0002B2A00F0A18000F29880202A00F09F8062
:1015C000232A00F09F802BB19DF8403043F0400368
:1015D0008DF84030B8F1000F05D09DF8403043F051
:1015E00020038DF84030BEF1000F05D09DF840304B
:1015F00043F010038DF84030BCF1000F05D09DF88A
:10160000403043F008038DF840302EB19DF8403053
:1016100043F004038DF840309DF8403003F044005F
:10162000442803D16FF386138DF840309DF8403085
:101630002A2A43F080038DF840307FD19DF8412065
:101640004B1C42F001028DF841201A782E2A0CBF63
:10165000012100219DF8412061F341028DF84120D4
:1016600078D15A782A2A6ED000224FF00A0C013322
:10167000194611F8010BA0F13006092E40F29580B1
:101680009DF840101292C1F3400040EAD2700A4621
:1016900060F341028DF840205CE0BA1C03928DF8A3
:1016A00043309DF84130DA0740F12E8154F8048B25
:1016B000B8F1000F07DA9DF84020C8F1000842F0A9
:1016C00004028DF840205E0740F1278154F804ABF6
:1016D000BAF1000F80F226819DF841306FF341038B
:1016E0008DF841304FF0FF3A1CE12D2A0DD0302A01
:1016F0007FF469AF012358E74FF0010C55E74FF035
:10170000010E52E74FF001084FE701264DE703466F
:101710000EFB0262303A184610F8016BA6F1300C4D
:10172000BCF1090FF3D999428FD09DF84010119266
:10173000D20F62F341018DF8401086E70B4600227C
:101740004FF00A0EE7E79DF84120023342F0040211
:101750008DF841201A786C2A47D02BD8682A31D0CE
:101760006A2A4BD04C2A51D01A4612F8013B782BEA
:1017700003928DF843309DF8412000F2BE806D2B1E
:1017800051D8692B00F2B980572B67D8412B03D071
:10179000453B022B00F2B18004229DF8423062F3F7
:1017A00002038DF84230012373E00CFB02020B466A
:1017B000303A5DE7742A25D07A2AD5D106219DF8E2
:1017C00041200CE05A78682A9DF8412006D1012179
:1017D00061F3C6028DF841200233C5E7022161F3AF
:1017E000C6028DF841200133BEE75A786C2A9DF875
:1017F000412001D10421EBE70321F0E705219DF809
:101800004120ECE707219DF84120E8E7BDF84020A2
:1018100022F4F04222F0020242F4804242F002023C
:10182000ADF84020DFE76E3BD9B201238B4040F298
:1018300082410B4237D113F0240F51D1D8075CD528
:1018400003219DF8423061F302038DF8423002F02B
:101850007803A3F140014B424B411AE00120A3F170
:101860005801C9B200FA01F111F4624F94D140F667
:10187000010631421DD111F4043F3ED09DF84230A3
:1018800060F3020302F07802402A8DF8423034D02F
:1018900000239DF84020C2F340010B4363F3410253
:1018A0008DF84020FDE602219DF8423061F30203ED
:1018B000E8E702209DF8421002F0780260F302018E
:1018C000402A8DF8421002BF9DF8401041F00101FE
:1018D0008DF84010632BDBD1131E18BF0123D8E70E
:1018E00003219DF8423012F0780F61F302038DF866
:1018F000423014BF01230023CBE79DF8403043F072
:1019000001038DF84030C3E79DF94020002AACBFA9
:101910004FF0FF38DDF84480D5E698077FF5E2AE5A
:10192000DDF848A00023CDE911339DF842309DF841
:10193000411003F00703012BC1F3C30133D1CB1EC8
:10194000042B04D8DFE803F0214646212100236858
:1019500001294FEAE372CDE90E321CD19DF93830EE
:10196000DA17CDE90E3204349DF8403013F0030647
:1019700050D03A4659464846039B14F048FB00288D
:10198000C0F252810544039FF2E554F8043BDA1794
:10199000CDE90E32E8E70229E5D11AB243F3C033AC
:1019A000CDE90E23DFE7022B24D1CB1E042B04D874
:1019B000DFE803F018101018180001294FF000029A
:1019C00054F8043B14D00229CDE90E32CCD19BB29D
:1019D0000E93C9E7073424F00704F4E80223CDE9A5
:1019E0000E23C1E754F8043B0E9300230F93BBE78B
:1019F000DBB2CDE7042B08D1073424F00704D4E987
:101A000000230834CDE90E23AEE7032BACD154F804
:101A1000043BDDE79DF843007828B4D862281CD841
:101A200025283FF4ADAD5828ADD1DDE90E010DF10B
:101A30003603009310AA08AB14F0A3FABAF1000F12
:101A4000074680F29980002F9DD00DF13603D81BF8
:101A5000002E00F0C0800130BDE06338152892D818
:101A600001A252F820F000BF3DDB00004FDB000078
:101A700087D9000087D9000087D9000087D90000E6
:101A80004FDB000087D9000087D9000087D900000C
:101A900087D90000DBDB000073DB000099DB00006E
:101AA00087D9000087D90000C1DA000087D900007B
:101AB00073DB000087D9000087D9000073DB0000CA
:101AC000BAF1000F0E9F35DB5146384615F0C9FDBF
:101AD00007EB000A002F3FF456AF00269DF8423076
:101AE00013F01002059200F0928002305B06119A0A
:101AF00048BF129B104448BFC018B8F1000F0492B1
:101B000040F39F809DF84020A8EB0008C2F38003BB
:101B10005007069300F19580510640F188803EB150
:101B200059463046C84700287EDB069B01351E46D5
:101B300030227DE0384615F08DFDC9E70E9B00266A
:101B400001208DF8203008AF0DF1210AC6E71907F2
:101B50005ABFC3F300135E012B26DDE90E23002BD1
:101B6000BFF663AF524263EB43032D26CDE90E234C
:101B70005BE7002659E700269DF840200DF136036B
:101B8000DB1B6FF386129A458DF840207FF65BAF22
:101B9000AAEB0303119356E70E9890B30DF13603A9
:101BA0000093002108AB10AA14F0EBF9BDF8423005
:101BB000BAF1000F03F0EF0343F4F04343F01003D6
:101BC0000746ADF84230D6DA00283FF4DCAE0026F6
:101BD0000DF13603181A9A4680E70E9B07293FF647
:101BE000D2AEDFE801F00C04060C08080C0C1D70E6
:101BF000C9E61D80C7E6EA17C3E90052C3E61D60C7
:101C0000C1E62F4F064607F1050A052066E71A07C9
:101C100048BF01306AE71046079306925946C84705
:101C2000DDE90623002804DA15B0BDE8F08F202294
:101C300043461946002903F1FF33ECDC454498463E
:101C40006D1A2EB159463046C8470028ECDB0135E5
:101C50009DF84230DA0601D41B0705D559463020DD
:101C6000C8470028E0DB0135059B33B159469DF894
:101C70004300C8470028D7DB0135049E2E4405E009
:101C800059463020C8470028CEDB0135731B002B96
:101C9000F6DC53463A465946484614F0B8F900284F
:101CA000C2DB0544A844A8EB0503002B7FF76BAE0D
:101CB00059462020C8470028B6DB0135F3E700BFAE
:101CC000F08D020008B54FF02002EFF3118382F38C
:101CD0001288BFF36F8F02F031FB034813F0F3FE5D
:101CE00001F04CFFFCE700BFF68D020008B5430988
:101CF0000CD0012B1BD01249124840F2472214F09D
:101D0000A4F940F247210E4814F098F94FF0FF3340
:101D1000C340DA07EFD50C4B03EB8003D3F8002266
:101D200022F0E04242EA0171C3F8001208BD4FF60A
:101D3000FF7300F01F00C340DB07DCD5034BEBE76C
:101D40001F8E0200568D020000258450002884500A
:101D5000F8B54FF02003EFF3118783F31288BFF338
:101D60006F8F0124234B244EC3F800450223032127
:101D7000C6F8D0360020FFF7B9FF20460321FFF751
:101D8000B5FF7E237F220025C6F80C37C6F83C3904
:101D90001A4B2146C3F81821194A2120C2F8045EC3
:101DA000C2F8085E02F54822C2F81051C3F8245167
:101DB000C3F82C5103F5FF1303F58053C3F8A05269
:101DC000C6F80447C6F80449C6F8004BFFF78EFF73
:101DD00021462020FFF78AFF21460B20FFF786FFD0
:101DE00021460A20FFF782FF87F31188BFF36F8F28
:101DF0002846F8BD00100050004000500020005060
:101E000000900350F8B50523194D1A4F2C781A4E3F
:101E10000134B4FBF3F303EB8303E41A18F0EDF998
:101E2000164A137873B157F82430C01A072809D816
:101E300033782BB95721124814F01BF90123337062
:101E40000020F8BD00214FF050233170D3F8140169
:101E500038B1C3F81411D3F814312C700CB9012324
:101E600013702C7818F0C9F947F824000120E8E72E
:101E70003B460020C8360020394600203A46002064
:101E8000528E020048B1054B054A1B68B3FBF2F3C2
:101E90005843044B43F00103184770476424002063
:101EA00040420F0080800200062807D10122044B27
:101EB000C3F80025BFF34F8F20BFFDE7704700BF79
:101EC000004000500DF0CABF2DE9F7430F4606460B
:101ED0000821C06A14F067F980463C68DFF8489032
:101EE000241A3C6004EA0905AC4203D8002003B080
:101EF000BDE8F08308236A462146304614F0C6F850
:101F00000028F4D16946304614F057F940B1BDF8C5
:101F10000230BDF8042005EA090513441D443C6065
:101F2000A4EB0804E0E700BF0000FFFF2DE9F04745
:101F3000044688B000F11407384619F08CFBA06AFB
:101F40008368DB689847E06248B94521AB4814F0E4
:101F500090F86FF01505284608B0BDE8F087A06A34
:101F60008368DB6898470368013B1F2B02D9452132
:101F7000A348ECE7A06A216805AA18F0A1F810B1FF
:101F80004521A048E3E7A5892DB1069BB5FBF3F2F7
:101F900003FB125515B145219B48D8E7E389012B76
:101FA00002D845219948D2E7E36A009593F8049056
:101FB0004FF0FF334FF0FF32384610F00BFD082191
:101FC000E06A14F0F0F8A8460646E3891FFA85FA9D
:101FD000534508D8E389434523D1384610F0B0FD76
:101FE0006FF02C05B7E7A1892B04891B13FA81F147
:101FF0004A4608232046009114F08DF878B16946CE
:10200000204614F051F808F1010808234A462046FA
:1020100000991FFA88F814F07EF80028DAD001350C
:10202000D3E753450BD1009908234A462046891B24
:1020300014F071F818B96946204614F035F869466D
:102040002046FFF741FF054618B1384610F078FDED
:1020500081E7009B4FEA13484FEA08486360C4F8E1
:102060000880D4E9011399420FD30823204601AA1E
:1020700014F00CF805460028E7D101AB13F8012B4A
:1020800091453CD10135082DF8D1636869461B0C98
:102090001B042046009314F007F84A462046A38903
:1020A000009914F038F8051ECFDB636869D04FF64D
:1020B000FF7906EB0308A3891FFA88F29B1B9A425B
:1020C000CDF8008037D34921514813F0D2FF204684
:1020D000616814F045F805460028B6D163684D4A9A
:1020E000A18913400B44A3EB4603636013402046D1
:1020F000A36014F044F90546002D5ED0A5E7204604
:1021000001A914F05AF8626810B9921B6260A8E73E
:10211000BDF80850BDF80610E06AC4F808802944EC
:1021200014F041F840449042A060EED1002DECD074
:102130006FF01C057AE008234146204603AA13F0FD
:10214000A5FF0546002880D1204603A914F035F8E4
:1021500038B1BDF80C304B4503D1BDF81030002B21
:102160006AD0B044A7E74A4620465B1A13F0D3FF73
:10217000051EFFF66AAF08D0E26AA368126813442E
:10218000A360D4E901318B42EDD86168A38901EBEA
:1021900046029A42B0D1DFF87C80A26801EA0803C7
:1021A0009A42A9D0204613F0DBFF054600287FF4B1
:1021B0004CAF636803EA0803A360A389A288A3EB7A
:1021C00046039A422ED0384610F0BAFC012349212A
:1021D000E28911482374A38913F04BFF62684921F7
:1021E00093B20E48120C13F044FFA268492193B237
:1021F0000B48120C13F03DFF0025ACE69D8E02004B
:10220000C48E0200E68E0200038F02001C8F0200C3
:102210008D8F02000000FFFF448F0200608F0200DC
:10222000778F0200204614F095F80546384610F0E6
:1022300087FC002DCAD08EE64921084813F019FF0B
:10224000636869461B0C20461B04009313F02CFFA7
:102250002046009913F084FF4DE700BFB98F0200BC
:102260002DE9F04F1D46037C04468946904689B00F
:102270004BB94521624813F0FCFE6FF00C06304666
:1022800009B0BDE8F08FC26A0821104613F08BFF39
:1022900082462946104613F086FFA3890746A3EB22
:1022A0008A039D4200F2A9801DB1B8F1000F00F031
:1022B000A48063680393204604AA03A9DDF80CB048
:1022C00013F0B3FF06460028D9D1BDF810304B45B6
:1022D00005D06268039B9A42EDD1E5B9CFE720466D
:1022E00004A913F06AFF0028F3D0BDF81200BDF86E
:1022F000143075B19D420ED14FEA1B4109040144CF
:102300002B464246204613F0DCFE002803DC06463E
:10231000B5E7002BB3D0002F3ED104F11403019395
:102320004FF0FF324FF0FF3304F1140010F052FB76
:10233000DFF8D0B0E3899E425CD0D4E90123F918DC
:102340008A422CD3ADF81A30FF2306A88DF81E3030
:10235000ADF81890ADF81C5013F01CFF2B46424608
:10236000A168204613F0ABFF29468246E06A13F0CD
:102370001AFFA2680244A260BAF1000F07D12046FA
:1023800006A913F0D6FF002814BF8246AA4601987A
:1023900010F0D6FB564672E75744BFB2BDE708219E
:1023A000E06A13F000FF4FF6FF73ADF8183000231A
:1023B000ADF81C301318ADF81A30A38902EA0B02ED
:1023C0001A44101A606006A813F0E4FE06A920461D
:1023D00013F0AFFF2046211D13F066FE6368204610
:1023E00003EA0B03A36013F0CAFF82460028CED194
:1023F00001369FE76FF01B0AC9E76FF015063EE74D
:10240000848E02000000FFFF2DE9FF471E46037C7B
:1024100004460F469046BDF8309043B92C484521FC
:1024200013F027FE6FF00C0004B0BDE8F087082120
:10243000C06A13F0B8FEA389A3EB40039E4243D8C1
:102440000025D4F804A0CDF804A0A9455146DDF834
:1024500004A009D2636853451ED1BDF80830BB42C1
:102460001AD06FF00100DFE7204602AA01A913F09D
:10247000DCFE0028D8D1BDF80830BB4206D120468A
:1024800002A913F09AFE08B10135ADB26268019B52
:102490009A42DAD15146E0E7BDF80C30002BE0D08B
:1024A000A945DED8BDF80A00090CB3424FEA014144
:1024B00028BF334601444246204613F0E7FD00287A
:1024C000B2D1BDF80C00AFE76FF01500ACE700BF6C
:1024D000848E020010B530B90B48452113F0C9FDB8
:1024E0006FF0150010BD836833B90848452113F01B
:1024F000C0FD6FF00400F5E71B6813B1BDE81040A4
:1025000018471846EEE700BFDA8F0200F08F02008E
:1025100070B508B101B132B90B48452113F0A9FDDE
:102520006FF0150070BD84680CB1E56835B90748D7
:10253000452113F09EFD6FF00400F3E741F8040B12
:10254000E368BDE87040184713900200F08F020066
:1025500070B51346044630B91048452113F089FD83
:102560006FF0150070BD006830B90D48452113F0BB
:1025700080FD6FF00100F5E782680AB1956835B912
:102580000848452113F075FD6FF00400EAE70A469C
:10259000AC466168BDE87040604700BF44900200EF
:1025A0005A900200F08F020008B504220021024870
:1025B00015F0B1F8002008BD0000072030B50C462A
:1025C0000E4985B00291D0F8AC110546CDE9003135
:1025D00000F1E0014FF0FF3320460FF0C9F950B988
:1025E000012384F86430D5F8A83123B1204605B022
:1025F000BDE83040184705B030BD00BF1F260200BF
:1026000038B50C461146054614F00BF8034638B9A8
:102610002846044914F005F803460020236038BD1D
:102620000120FBE7C1B302002DE9F04F01238146F1
:102630000569466885B005F55977D7E8EF2F002A78
:1026400003D1C7E8E13F0029F7D140F0B880B36873
:10265000B26A043B2632B3EB420F4FEA420126BF77
:10266000B3FBF1F3B3FA83F300234FF0010428BF67
:10267000C3F12003013B9C4005F5E47800F099800C
:102680001022082170689A4002EB440204309940FD
:102690000932C5F86002063122F003020A44B16A29
:1026A00001FA03FC510001EB4C01C5F86412B16A58
:1026B000994000EB4103C5F858320333134423F02B
:1026C0000303C5F854327368C5F85C42C5F850324C
:1026D0003C4B4046C5E9A963316800F01DFA044649
:1026E00030BBD9F804A0D9F81090DAE9073409F51D
:1026F000307B012B584608BF103C10F0EFFE002342
:10270000DAF8240030494FF4806201EB8021009315
:102710005846234610F0F8FE09F52C702B4910F0AE
:10272000EFFDDAF8140083685C681CB96FF0570499
:10273000002137E04B46264ADAF81810A047044635
:102740000028F5D1DAF8140083681B69002BEDD05E
:102750000122DAF81810984704460028E8D11D4BEA
:102760002846C5F8A8311C4BC5F8AC311B4B039368
:10277000D5F810320293D5F80832CDE90083D5F8A8
:102780006832B26AD5F8601300F08EF9044600286A
:10279000CED105F1E0000FF085FA0028C5F86803F6
:1027A0000ADB0221384613F071FF204605B0BDE870
:1027B000F08F6FF00B04BBE76FF01504B8E76FF014
:1027C0007704F2E775260200A84600205B26020087
:1027D0004F260200A5E800002D270200BD260200BA
:1027E0002DE9F84306464FF001090569D0F8048049
:1027F00005F55977D7E8EF3F022B03D1C7E8E29FF1
:10280000002AF7D149D1264805F1400114F032FFE2
:1028100020B16FF00F042046BDE8F883204805F191
:10282000B00114F027FF0028F3D12846D5F8601333
:1028300013F0AFFF044670BB71683669486983685E
:102840001B6933B3224689699847044618BB06F5CD
:1028500030764946304610F0B7FE304605F5E4764E
:1028600001F0B6FD3046D8F8001013F0CFFF044653
:1028700088B90146E822304614F04DFF21464FF456
:10288000E272284614F047FF2146384613F0FEFE58
:10289000C1E76FF057040221F7E76FF07704BAE75A
:1028A000C1B3020013B5044640B100230122CDE9B3
:1028B0000032074BD0E909120FF00EF8A36E1B6827
:1028C00023B1E06E02B0BDE81040184702B010BD61
:1028D000C1B3020013B504460846216901F55971D8
:1028E000D1E8AF1F022910D193B1A0B10121CDE9E8
:1028F00000311346D0E909120EF0EEFF074B984263
:1029000008BF6FF00B0002B010BD6FF00F00FAE7C8
:102910006FF04C00F7E76FF00100F4E72EF8FFFFCF
:102920002DE9F74388461546066906F55973D3E83D
:10293000AF3F022B5FD1136823B96FF0150003B0CE
:10294000BDE8F0831B78002BF7D0D6F86093B9F17F
:10295000000F33D106F5D8774FF0FF324FF0FF3339
:10296000384610F037F830462A6801A9FFF748FECC
:10297000019C1CB9384613F087FEDEE705F1080319
:10298000A3666B6984F86490E366E46360B13846DB
:1029900013F07AFE21463046236E2A68FFF70EFEBA
:1029A0000020C8F80040CAE72022296804F140004E
:1029B00014F03CFE384613F067FEF1E730460F494D
:1029C00013F02FFE04460028B7D005F108038366F4
:1029D0006B69C063C366002380F8643020222968D5
:1029E000403014F023FE22460121304600F03EF82C
:1029F0000028D5D0A1E76FF00F00A0E7C1B3020017
:102A00002DE9F04F05460E4690460027D0F8B0A0BD
:102A100085B0AAF5AE742146304614F02BFEE0B91D
:102A2000114BA4F1400B0293DAF810303246CDE995
:102A3000008329464FF0FF335846AAF5CE790EF0B1
:102A400097FF60B97023012203FB079383F864208A
:102A5000DAF80C300BB158469847703417B105B00E
:102A6000BDE8F08F0127D6E78F2702001FB5144677
:102A700090B18AB1012912D10A4B00F1E001029311
:102A8000D0F8AC31403201934FF0FF332046009331
:102A90000EF06EFF04B010BD6FF01500FAE70020D5
:102AA000F8E700BF8F2702002DE9F04387B00E46FC
:102AB000DDE90E811446DDE910251F4630B329B348
:102AC000DFF850C000F1E009002D08BF65469EB94F
:102AD000CDE9034400F5CE742046059618F08CFA33
:102AE00003ABCDE900432A463B46414648460FF03A
:102AF000FFF807B0BDE8F083002241460E92484639
:102B00002A4607B0BDE8F0430FF01CBA6FF015007D
:102B1000EFE700BF01EA0000F0B50E46044689B0B9
:102B200000286FD001230246C3630023D0F8981019
:102B3000364F403040F80C7C42F8301FCDE901336D
:102B40004FF0FF330093C36D17F0BFFD304A06AB63
:102B500092E8030083E8030018460EF0DDFD054609
:102B6000D8B904F134000EF0B7FD0546A8B93946CE
:102B7000284805AA17F081FD054670B9059B9A689B
:102B800072B10C33D4F89400C4F8A03013F030FEC6
:102B9000C4F8D40030B96FF00B05284609B0F0BD79
:102BA0000346EFE7D4F8940013F022FEC4F8D800EF
:102BB0000028F0D0D4F88C30D4F8A010C4F8A83095
:102BC0000423C4F8AC30C4F8C4300223A362124B0F
:102BD000B4F89420D4F8D470C4F8B810C4F8D01065
:102BE000D4F89010236204F1A403A4F8B020C4F830
:102BF000A470C4F8C010A4F8C820C4F8BC00A66132
:102C0000E362CAE76FF01505C7E700BF89900200CD
:102C1000E47F020093900200CC80020070B5114B5B
:102C20000D461C68DCB1104B196800238B4202DB97
:102C30006FF0010070BD224612F8106B864202D080
:102C400014460133F2E7E06810B96FF01200F1E7C3
:102C500018F0A9FC0028F8D000202C60EAE76FF0FB
:102C60000C00E7E7082200206881020070B588B0F8
:102C700005460C46C0B269461646FFF7CFFF00284E
:102C80001BDB0098C8B143682268029383680195F2
:102C9000CDE903360023CDE906230593C56813F07B
:102CA00024FE6DB12846084901AA17F00DFA0798CD
:102CB00008B9059B236008B070BD6FF01500FAE7F6
:102CC0006FF01200F7E700BF89290200F8B58368AA
:102CD0000446002B31D0D0E90476C06813F076FEAC
:102CE000A568B5FBF0F300FB13555DB1451BE0682B
:102CF0008368DB689847A368017920682A461844EE
:102D000014F009FDA368E06822683E442B44816802
:102D10004D683146A847054638B10246334645213D
:102D2000174813F0A6F92846F8BDE3695BB9236993
:102D3000A268134423610023A3600025F3E7535DD9
:102D4000DB4353550135A3682268AB42F7D8E068EE
:102D500081680D683146A847054628B145210246DD
:102D6000084813F086F9DEE73246E369A168206877
:102D7000984705460028DAD0024645210248F0E788
:102D80009B900200C4900200DF90020010B54368DF
:102D90000A680C469A4207D90548452113F069F99B
:102DA00000231846636010BD4A6801201344F9E708
:102DB000F89002002DE9F7430D46DDE90A869146B9
:102DC0001F46044680B179B172B1009300230846D2
:102DD000019313F0FBFDB7FBF0F303FB107040B160
:102DE0004521184813F045F96FF00D0003B0BDE818
:102DF000F0836A462846144917F066F9019B002BB8
:102E0000F2D008EB0602934202D245210F48E9E7CF
:102E1000284613F0DBFDB8FBF0F303FB108000281D
:102E2000F3D1C4E90097E5602061A060C4F8148084
:102E300016B9019EA6EB08060C9B0020A661E36173
:102E4000D4E700BF1D9102008DED000059910200F2
:102E50002DE9F0410F4B05461C680E461746ACB1F4
:102E60004FF0FF324FF0FF330B480FF0B3FD6368B4
:102E70003246D3F8088029463B462046C0470446E0
:102E800005480FF05DFE2046BDE8F0816FF00104BB
:102E9000F9E700BFDC360020842700200023036010
:102EA000044B5A6812B9C3E90000704710605860BB
:102EB000704700BFE0360020014B1860704700BF2C
:102EC000DC360020002330B585B00546CDE902335D
:102ED00001904FF0FF334FF0FF320B480FF07AFDB7
:102EE0000A4B1C684CB9284600F0DCF8044606483A
:102EF0000FF026FE204605B030BD636820461B68F3
:102F000001A998472468EDE784270020E0360020D7
:102F10001FB5CDE9010103924FF0FF334FF0FF32AF
:102F200009480FF057FD094B1C682CB906480FF0F3
:102F300007FE204604B010BD636820461B6801A947
:102F400098472468F1E700BF84270020E03600207E
:102F50000022024BC3E90022704700BFE036002088
:102F60000022024BC3E90022FFF7F2BFE83600203F
:102F70002DE9F74307460C4609B100230B600026F4
:102F8000234DDFF890904D4520D9234923489422C2
:102F900013F05BF89421204813F050F8D5F8008026
:102FA0003846414601AA13F062FD50B116B954B932
:102FB0002E4606E000224046316813F058FD0028F6
:102FC000F5D11435DFE7019B2360F1E7E6D3144B1D
:102FD0001D68C5B155F8148C3846414601AA143D08
:102FE00013F045FD50B116B954B92E4606E0002243
:102FF0004046316813F03BFD0028F5D16D69E8E7E4
:10300000019B2360F1E7304603B0BDE8F08300BFC9
:10301000447F0200BC7F02007F910200568D0200B7
:10302000E83600202DE9F341DDF8208004460D4606
:1030300016461F460190B8F1000F07D0D8F80010CF
:10304000C1B9D8F804E0BEF1000F1CD1204601A997
:10305000FFF78EFF98B13B46D0F8088032462946EC
:103060000198C047034650B1224645210C4813F051
:1030700000F804E001AA13F0FAFC0028E1D10020D6
:1030800002B0BDE8F081D8F80830324608932946EE
:103090003B46F446019802B0BDE8F041604700BFEE
:1030A000B1910200F8B5064600251C4C1C4FBC42ED
:1030B0001BD91C491C48F42212F0C7FFF4211948FF
:1030C00012F0BCFF2EB9E3685BB9284605461434FC
:1030D000EDE700223146206813F0C9FC0028F2D148
:1030E000F3E79847002DF0D1F0E7EBD30F4B1C68C6
:1030F00094B1143C1EB9E3684BB96469F8E7002247
:103100003146206813F0B3FC0028F4D1F5E7984766
:10311000002D08BF0546F0E72846F8BD447F0200B1
:10312000BC7F02007F910200568D0200E83600202D
:1031300038B50C4D4FF0FF334FF0FF320A480FF017
:1031400049FC2B783BB9FFF70BFF00F06DF8044604
:1031500010B901232B70002403480FF0F1FC204626
:1031600038BD00BF3C460020842700202DE9F047F1
:1031700080468946048FDFF8ACA0013498B0A4B231
:1031800000F10806651EADB2B5F5004F47D04A23E1
:10319000294605AA304613F0C3F904F57F543F349D
:1031A000A4B207462146012330460DF10B0213F06D
:1031B000B7F9002F014603DC002803DC2C46E1E7C9
:1031C000002816DCB8F83830AB4209D142466B1EF5
:1031D00022F8383F4FF4004102233046FFF740F811
:1031E0002946304613F098F92146304613F094F9F9
:1031F000E4E707F160030DEB03070023524607F8ED
:103200004C3C05A8CDF8009003AB0396ADF81040F8
:10321000FFF708FF0028D1D018B0BDE8F0870020E4
:10322000FAE700BFDF2A02007FB5012369460620C6
:103230000193FFF7F3FC0446002834D1062002AACC
:1032400001A9FFF713FD10F1130F04462BD038B17D
:103250000C3405D0404080F311884FF0040002DFA9
:103260000399B1F5803F23D200231846009A946851
:10327000084484421AD30133082BF9D10E4DA98298
:10328000EB8253682846AB60D368EB6313F0C1FC54
:10329000044640B9094E28466E60FFF7FFFD2846F8
:1032A0006E60FFF709FE204604B070BD9BB2E5E7F3
:1032B0006FF02004F7E700BFF0360020C82100209F
:1032C0002DE9F84305464FF02003EFF3118683F311
:1032D0001288BFF36F8F1B480FF02AFB40B91A49C1
:1032E00094221A4812F0B1FE9421174812F0A6FE5B
:1032F0004FF00C0913480FF037FB154B154F1C68A6
:10330000DFF8548054B90F480FF020FBA0B90E49E4
:10331000C2220E4812F099FEC221E6E7D4E9012349
:10332000002D18BF13462BB198F8142009FB02F2A8
:10333000B85C98472468E5E786F31188BFF36F8F80
:10334000BDE8F88330370020908D0200568D0200D2
:103350005037002044370020E8430020012270B598
:10336000164B1C7D04F01F039A40D043144B610997
:1033700003EB8103D3E8EF1F01EA0005C3E8E65F32
:10338000002EF7D10A4213D00E4B0F4D8BB10C23F8
:103390006343EA185178E85C12F065FE0020FFF7FD
:1033A0008FFF0C235C4300232A192B51C2E9013300
:1033B00070BD83F31188BFF36F8FEFE7E843002000
:1033C0005837002067200200443700202DE9F041E3
:1033D000404B07461D7D4FF02003EFF3118883F328
:1033E0001288BFF36F8F3C480FF0A2FA40B93B49F7
:1033F00094223B4812F029FE9421384812F01EFE18
:103400000C246C4334480FF0AFFA364B364E195D3E
:103410001A1991B107CA06EB040C8CE807000022C8
:103420001A552D480FF092FA044688B92B49C2224A
:103430002B4812F00AFEC221DFE73946284600F089
:103440005DF80028EDD007C8344484E80700E8E7B9
:1034500088F31188BFF36F8F0C236B43F218F35C72
:10346000ABB37B1C0FD04FF4004C0021D2F808E026
:103470001E480023EEFB0C011D4AFCF76DFF0121E5
:10348000381A11F01BFC10F075FC0120FFF718FF33
:10349000184B6A0903EB8203012205F01F018A40E1
:1034A000D3E8EF0F1043C3E8E10F0029F8D1124B26
:1034B00033B10C236B43F2185178F05CFEF7F4FC47
:1034C000FFF74CFF10F0A2FC2046BDE8F0811C463F
:1034D000FAE700BFE843002034370020908D020057
:1034E000568D020038370020443700203F420F003D
:1034F00040420F0058370020A9DE00002DE9F04FB0
:1035000085B00E4603A900F043F84FF40047044687
:103510004FF0000B1B4B039DD3F800A0431E1BB2C2
:1035200003EB4303DFF8608005EB830524B9A14674
:10353000484605B0BDE8F08FC44659466868002388
:10354000E0FB07C1114A6046FCF706FFC446594636
:103550000190A8680023E0FB07C10C4A6046FCF715
:10356000FBFEBAF1FF3FA94601D0824505D9731C85
:10357000DED0019B1844B042DAD9013CA4B20C3D24
:10358000D4E700BFDC2100203F420F0040420F0083
:1035900008B9024B0B600020704700BFF0800200AA
:1035A0004B1E59425941014B197070473E4600204D
:1035B00008B5012BBDF808100CD171B90A4B1B6876
:1035C0000BB9012008BD1078012809D800F00100CE
:1035D0009847F6E76FF00C00F4E76FF00600F1E7AC
:1035E0006FF01200EEE700BF5C3700202DE9FF41CD
:1035F0001F460D4B054658680C46164680B1D1F85B
:103600000C808047094B324618700123CDE90183B5
:10361000BDF828302146009328463B4615F0ADFC06
:1036200004B0BDE8F08100BF5C3700203D460020BB
:1036300020B1034B02681A6042685A60002070474C
:103640005C37002000B50E4B89B01B788DF8070061
:103650009BB10021182202A814F05DF8094B00204C
:1036600003930DF107030493012302A9ADF814306D
:1036700006F06AFD09B05DF804FB6FF00C00F9E795
:103680003E460020188102000449431E0F3013F803
:10369000012F8A5C83421A70F9D17047E5910200CC
:1036A000F0B50746264E8DB001AD0C460FCE0FC5C6
:1036B0000FCE0FC596E8070085E807003846002FB3
:1036C00039D0002C39D0381F0246214610344B78AF
:1036D0000D781B0443EA0563CD7804312B4311F8C0
:1036E000025C8C4243EA052342F8043FEFD10421F7
:1036F000144C8A07036916D1C3F30742A55C1A0E5E
:10370000A25C42EA0562C3F30725655DDBB2E35CB8
:1037100042EA054242EA032221F0030330336B44BC
:1037200053F82C3C534050F8042F013153402C29BE
:103730000361DED101200DB0F0BD2046FBE700BFE4
:10374000EC7F0200E59102002DE9F04F00270368AD
:103750009DB002934368DFF8BCA103938368DDE961
:1037600002460493C36805930369DDE904BE06932A
:10377000436907938369DDE9062C0893C36998467A
:103780000993089B0093CD590CAB2DBA5AF8049BB2
:10379000DD514FEAF223A94483EAB213009D83EA84
:1037A00072634B4425EA020502EA0C0985EA090521
:1037B0002B44434486EA0B054FEA743888EAB40880
:1037C000254006EA0B0985EA090588EAB45804375A
:1037D000A844402F03EB0E054344DE46DDF800808D
:1037E00040F088804FF0100A4B490A9151460AF187
:1037F000010A0DF1700E0AF00F070EEB870757F85C
:10380000407C01F00F094FEAB748019788EAF718A2
:1038100001F10E0707F00F070EEB870757F8407C02
:1038200009314FEAF74E8EEA774ECDF82CE001F0E1
:103830000F010DF1700E0EEB81010EEB890959F8A5
:1038400040EC51F8401CBAF1400F7144DDF804E03F
:1038500088EADE08DDF82CE041448EEA972E7144B8
:1038600005EA02084FEAF52E2CEA050787EA080761
:103870008EEAB51EDDF828808EEA756E774458F81A
:1038800004EF49F8401C77440F4400994FEA733E17
:10389000394484EA0607CDF828808EEAB30E07EA99
:1038A000030704EA06088EEAB35E87EA080777444E
:1038B0000F4401EB0B0ECDF800C0B34622D10299A4
:1038C0003944016003991944049B41602344836097
:1038D000059B3344C360069B73440361079B2B44E1
:1038E0004361089B13448361099B6344C3611DB01A
:1038F000BDE8F08FB346CDF800C0264694461C467E
:103900002A4640E7944626462A461C4675463B46CC
:103910006CE700BFEC8102002882020010B504466B
:10392000C8B17022002113F0A2F90B4B0B4A0C49CD
:10393000C4E900230B4B0C48C4E902130B4BC4E948
:10394000040301200A4BA36103F17453A3F523037D
:10395000A3F69243E36110BD85AE67BB67E6096AD3
:1039600072F36E3C3AF54FA57F520E518C68059B61
:10397000ABD9831F014811F0D1BE00BFEC82020019
:1039800038B5044618B90F4B0F485B689847616813
:10399000B1F5683F0FD0B1F5680F0CD00B4DA942BF
:1039A00009D011F4686107D0214609480EF072FE73
:1039B00000232360656038BD1422206813F0ABFE3D
:1039C000F8E700BF24250020E59202002C5F5CA9E7
:1039D000643C002008B560B34368B3F5683F0ED07F
:1039E000B3F5680F18D0144A934220D000684FF006
:1039F000FF324FF0FF330EF0EDFF58B115E001221A
:103A00000368D3E8EF1F002903D1C3E8E02F0028A3
:103A1000F7D10AD1002008BD0368084A1B7803F5D6
:103A2000807352F82330002BF4D00548F3E70548A3
:103A3000F1E76FF4E040EEE72C5F5CA90000035073
:103A4000E98FFFFFEA8FFFFF08B520B34368B3F5A6
:103A5000683F09D0B3F5680F13D0114A93421DD0C7
:103A600000680FF06DF814E000220368D3E8EF1F40
:103A7000012903D1C3E8E02F0028F7D109D0094874
:103A800008BD00210368084A1B7803F5807342F8DB
:103A900023100020F4E76FF4E040F1E70348EFE77C
:103AA0002C5F5CA9E98FFFFF00000350EA8FFFFF46
:103AB00010B5044618B91D4B1D485B6898476368EC
:103AC000B3F5683F2FD0B3F5680F2CD0194A934255
:103AD00019D1236803BB4FF0FF324FF0FF3321466B
:103AE00015480EF07FFD08B923681BB90F4B13482A
:103AF0005B68984714220021206813F00CFE4FF4F5
:103B00006863636008E0B3F5683F0DD83A2B03D0D3
:103B100040F6BA629342DED1206817F09CFD6368DC
:103B200043F03A03636010BD054AF3E72425002003
:103B3000E59202002C5F5CA9643C00200B9302001C
:103B40003A00003A08B5064940231422054817F008
:103B500057FDBDE808400449044811F051BE00BFBC
:103B600064370020643C0020F482020008830200D5
:103B7000014910220A60704710ED00E072B6404023
:103B800080F31188BFF36F8F01B5FEF73BF9002872
:103B900002D0BFF34F8F30BFBDE8014062B6BFF324
:103BA0006F8F704772B6494081F3118801B5FEF7F7
:103BB00029F9002802D0BFF34F8F20BFBDE8014094
:103BC00080F3118862B6704737B505460C46C9B117
:103BD0008B6810480093D1E90023452112F049FA7F
:103BE000636945210093D4E903230B4812F041FA9D
:103BF0004521E269094812F03CFA4521A2690848CA
:103C000012F037FA2146284603B0BDE830400EF0E6
:103C10009BBA00BF389302006C930200A09302008D
:103C2000B493020040B2002807DB01234109034A94
:103C300000F01F00834042F82130704700E100E0AF
:103C400040B200280CDB01220649430900F01F00A6
:103C50008240203341F82320BFF34F8FBFF36F8F93
:103C6000704700BF00E100E0054B420953F82220F5
:103C7000012300F01F0003FA00F01040704700BF5E
:103C800000E100E00131072908B508D90D490E48C7
:103C90005B2212F0DAF95B210A4812F0CFF940B248
:103CA0000028ACBF00F16040084B4FEA4111C9B297
:103CB000ABBF00F5614000F00F0080F8001319540D
:103CC00008BD00BFE7930200568D020014ED00E02E
:103CD00030BFFFF7FDBF00BF0B4A08B50B4B22F00A
:103CE0007F029A60BFF34F8FBFF36F8FD3F88820A6
:103CF00022F47002C3F888200EF0BEFA10F05CFEC9
:103D000000F0E0FA0EF0F8FA00C2000000ED00E06A
:103D1000094A0A49936809689867D96708494B684E
:103D200043F080534B60002383F31188BFF36F8F00
:103D30009368D86F704700BFE84300207489020081
:103D400000ED00E013498A684FF030001044EFF3B3
:103D5000098C80E8F01F202080F31288BFF36F8F5A
:103D60000D4F4FF00066CA698A603E60906F002375
:103D7000936780F3118802F1300090E8F01F8CF314
:103D8000098802F1000004B513F0C2FBBDE804404D
:103D900070470000E843002004ED00E01EF0040F2F
:103DA0000CBFEFF30880EFF30980816911F8021C62
:103DB0000229FFD001B513F09CFB01BD42F8203C65
:103DC000009B0B4942F81C3C019B21F0010142F889
:103DD000183C029B42F8081C42F8143C4FF08073D8
:103DE00042F8043C0023203A02658367704700BF15
:103DF000FB1A0200084B9860836E83F30B88104611
:103E000081F30988002163B681F31188BFF36F8FB6
:103E10000022002311F071FEE843002001B572B6C4
:103E20000B4A906900281EBF0021916117F004FC25
:103E300062B6EFF30580A0F110004FEAC00005491B
:103E4000014409C99847BDE80140034908470000FB
:103E5000E84300202C7B02005DFE0000044B9968C3
:103E6000D869884203D003494FF080520A607047F6
:103E7000E843002004ED00E038B5214C45212148FD
:103E800012F0F7F8A36A9D0103D545211E4812F0F0
:103E9000F0F8A36ADC0103D545211C4812F0E9F8CB
:103EA000174DAC6A14F4801404D04521184812F060
:103EB000E0F80224AB6A180303D54521154812F037
:103EC000D8F80F4DAB6A590303D54521124812F0BB
:103ED000D0F8AB6A9A0303D54521104812F0C9F80F
:103EE000074DAB6ADB0303D545210D4812F0C1F83D
:103EF000AB6A20466FEA03436FEA1343AB6238BDF7
:103F000000ED00E01D9402003A9402005294020079
:103F100071940200A0940200C3940200ED94020088
:103F20000C95020070B5234C06460D4622484521EB
:103F300012F09FF8A36AD90403D545211F4812F057
:103F400098F8A36A1A0503D545211D4812F091F887
:103F5000184CA36A9B0510D51A48452112F089F820
:103F6000A26BA36A180408D54521174812F081F8FE
:103F70001EB1A36A23F40043A3620E4CA36A590541
:103F800003D54521114812F074F8A36ADA050BD560
:103F900045210F4812F06DF80020064A936A43F459
:103FA0007F439362287070BDA36A9B04F4D54521BA
:103FB0000848EFE700ED00E03C950200579502004D
:103FC0006D95020085950200A3950200BD95020043
:103FD000DD950200FA95020070B52E4C06460D469E
:103FE0002D48452112F045F8A36ADB0603D545218B
:103FF0002A4812F03EF8A36A1C0703D54521284839
:1040000012F037F8234CA36A980710D545212548AC
:1040100012F02FF8626BA36A190608D545212248D1
:1040200012F027F81EB1A36A23F08003A362194C93
:10403000A36ADB0703D545211C4812F01AF8A36ACE
:104040009E0603D545211A4812F013F8114B9A6ABF
:10405000D40602D49A6A90070DD59B6AD9060AD570
:10406000144915484FF4AE7211F0EFFF4FF4AE71E2
:10407000104811F0E3FF0020064B9A6A920642BFF7
:104080005A6A22F400525A629A6A42F0FF029A6215
:10409000287070BD00ED00E02E96020049960200E7
:1040A0006D950200819602009E960200B99602006C
:1040B000FA950200DD960200568D020070B5694B3C
:1040C0000546586800268AB0C0F3080386F31188B5
:1040D000BFF36F8F02F07F44B4F17F4F07D102F03E
:1040E0000C04082C0ED145215F4811F0C2FF5F4936
:1040F0004FF484625E4811F0A8FF4FF484615B487E
:1041000011F09CFF14074CBF0D460126002DEED088
:104110000024DA1E8DF80740092A00F29280DFE8B9
:1041200002F00585897090909090908D45215148BE
:1041300011F09FFF8DF807404A4CE36A9A0705D5B6
:1041400045214D4811F095FF002429E0E36A002B3A
:1041500002DA45214948F5E7E36A5B005DD5452170
:10416000474811F086FF6369AA6943F4807363616D
:10417000BFF34F8FBFF36F8F636932F8022C23F4C4
:1041800080736361BFF34F8FBFF36F8F4DF6027380
:104190009A421ED145212A683A4811F06AFF2C68DC
:1041A0009DF807309BB92022294602A813F0A8FAEF
:1041B000099B002E51D0C3F3080222B96FEA5323A2
:1041C0006FEA43230993204602A9FFF7FDFC0AB0DA
:1041D00070BDA36ADBB233B101200DF10701FFF717
:1041E000FBFE0446DCE7A36A13F47F4F05D00120F1
:1041F0000DF10701FFF796FEF3E7A36AB3F5803FE1
:1042000002D3FFF739FEECE7184940F2F2221848D2
:1042100011F01BFF40F2F22171E7144940F2F6223F
:10422000134811F012FF40F2F62168E700200DF16B
:104230000701D4E700200DF10701DBE74521124813
:1042400080E7124910F4F87F114A124808BF0A4665
:10425000103B452111F00DFF76E723F4FF7323F0A7
:104260000103AFE700ED00E045970200DD96020094
:10427000568D02007597020091970200B7970200D1
:10428000CA970200EE9702000F98020017970200EB
:104290002C97020038980200044B5A6942F0100231
:1042A0005A615A6942F480625A61704700ED00E039
:1042B000EFF30880EFF3098101B57246FFF7FEFEC8
:1042C00001BD00BF002320210348C2180133452B44
:1042D00082F80013F9D1704700E100E0002080F37C
:1042E0001488BFF36F8F002080F30A8880F30B8857
:1042F000FDF7E8FD00200E490860BFF34F8F0D4821
:1043000080F3088800F03EF8202080F311880A48E6
:104310004FF40061401880F30988EFF31480022104
:10432000084380F31488BFF36F8FFFF7D5FC0000BC
:1043300094ED00E090800020506F0020BFF34F8F7D
:104340000549064BCA6802F4E0621343CB60BFF331
:104350004F8F00BFFDE700BF00ED00E00400FA054D
:10436000002318460649D1F89020C2F30722934251
:1043700000DB7047C1F89830C1F8A0000133F6E7C0
:1043800000ED00E010B572B6002484F31388FFF747
:10439000E7FF23464FF0FF300C4A03F120010133C1
:1043A000102B42F82100F8D100234FF0FF30074ACC
:1043B00003F160010133102B42F82100F8D162B6FD
:1043C000BFF34F8FBFF36F8F10BD00BF00E100E060
:1043D000084B9B6883420BD1EFF3058343B1064B37
:1043E0005A6842F080525A605A6A22F400425A6275
:1043F00010F0E2B9E843002000ED00E01FB5094CE1
:10440000094A23460121094800F024F900230393B7
:10441000074B0121E41A01A80193029400F034F93A
:1044200004B010BD00000720002000201883020007
:10443000B829002010B50C7A0B6804F01F0223F095
:104440001F031A43CB68640923F01F03054943EA9D
:10445000440343F00103C1F89800C1F89C20C1F85F
:10446000A03010BD00ED00E030B50C684B6885B0A1
:104470000A894D890094013B24F01F04234402F073
:104480001F0242EA451223F01F03072804468DF855
:104490000820039309D902464521064811F0E9FD99
:1044A0006FF01504204605B030BD6946FFF7C2FF26
:1044B000F8E700BF549802002DE9F04F89461446F2
:1044C00006464FF00008544D85B0C84527DAD6F8A7
:1044D00004A0BAF1000F44D0BAF11F0F18D91AF096
:1044E0001F0F15D1D6F800B01BF01F0F10D1584682
:1044F00013F012F807460AEB0B00013813F00CF822
:10450000874210D06FF015073A464521434802E034
:1045100042464521424811F0ACFD6FF0150420469B
:1045200005B0BDE8F08F17F1160FEDD0BC42EBDD02
:10453000C5F89870D5F89C10C5F89870D5F8A030DB
:1045400021F01F0143F01F0BD6E900321A449942B3
:1045500002F1FF3A1DD1D34507D13146F8B2FFF73A
:1045600083FF08F101080C36AFE73146C5F89870B3
:10457000D5F89C3022F01F0203F01F031343C5F847
:104580009C30E0B2FFF770FF10F1160FC5D0441C4D
:10459000E7E7C5F89870D5F8A020013B23F01F038A
:1045A00002F01F021343D3453146E0B2C5F8A030F4
:1045B000E8D0FFF759FF10F1160FAED0C5F898708C
:1045C000D5F89C209DF808300BF1FF3B62F3040303
:1045D0008DF80830D5F8A0309DF808205B0863F30B
:1045E0004712D6E900310B44009323F01F0301303A
:1045F0005B44A3EB0A03C0B223F01F0307288DF826
:104600000820039303D902464521064883E76946FB
:10461000FFF710FFBBE700BF00ED00E0A798020026
:104620007F980200549802000522044BC3F894209E
:10463000BFF34F8FBFF36F8F704700BF00ED00E0F7
:10464000BFF35F8F0022024BC3F89420704700BF76
:1046500000ED00E010B5094C2278FFF72DFF207027
:1046600016300AD1064907484FF48D7211F0EDFC5F
:104670004FF48D71024811F0E1FC10BD3F4600205F
:10468000CF980200568D02002DE9F74F2E4D8A4635
:1046900006464FF00008AB462C4FD04502DB03B076
:1046A000BDE8F08FD6F80490B9F1000F47D031681B
:1046B0000846019112F030FF0199044609EB010010
:1046C000013812F029FF84424FF01402204B10D021
:1046D00002FB08F36FF015024BF803201D491E483A
:1046E0004FF4957211F0B1FC4FF49571194811F027
:1046F000A5FC14F1160F2C60F0D01978A142EDDD65
:1047000002FB08B0C7F89840C7F89840D7F89C401B
:1047100000F10801007B64F304000871D7F8A000E1
:104720000C79400860F347140C71D7F89C1021F005
:104730001F016960D7F8A01021F01F01296108F15D
:10474000010814350C36A8E7843C002000ED00E099
:104750003F460020CF980200568D020038B51A4D12
:104760002C68082C0AD9194940F25112184811F046
:104770006CFC40F25111154811F060FC0020FFF76D
:104780005FFF144B144AC3F8C020844213D1134B6B
:104790001C70FFF749FF0F4BD3F89030C3F307238A
:1047A000082B0FD0094940F2BB12094811F04DFC0B
:1047B00040F2BB11DFE7696801EB0011FFF73AFE39
:1047C0000130E2E7002038BD24830200CF980200C8
:1047D000568D020000ED00E0AAFF44003F46002095
:1047E000014B1860704700BF2C2200200CB410B59C
:1047F00086B009B90DF10B000024CDE9040109AB25
:10480000089A009404A905480393FCF7A9FE049BA9
:104810001C7006B0BDE8104002B070472F37020090
:104820001022044B0020C3F840244FF05023C3F85B
:10483000140670470030005030B503788BB0044642
:1048400007AD032B21D8DFE803F0021A1C1E124922
:10485000284612F0E1FE059563781E210493A378A3
:104860000E4A0393E3780E48029323790193637908
:104870000093A37911F034F909480BB030BD094910
:10488000E6E70949E4E70949E2E70A212846084A38
:1048900011F026F9DFE700BF978A0200C08A020004
:1048A000404600209E8A0200A58A0200AF8A0200CC
:1048B000B98A020008B508490848CA79C2EBC202A1
:1048C000FEF7C6FA024628B1BDE808404521044873
:1048D00011F0CFBB08BD00BF002000204F9902009F
:1048E00055990200F7B5054616461F461A4CD4E8FE
:1048F000AF3FDA0729D538B94521184811F0B9FB7F
:104900006FF0010003B0F0BD01A912F0D4F8144912
:104910000246284612F0BAFE0028F1D1D4E8AF3F93
:10492000C3F3C0051B0710D4CC3C072221463846F0
:10493000B04706280BD845210A4811F09AFB0722F8
:104940002946204612F0E7FEE5710020DAE707234A
:10495000B0FBF3F0E071F8E7CC200020759902007D
:10496000AC8A02009B9902002DE9F04188B0DDF885
:1049700038809C795D791E79DF7893F802C093F8CE
:1049800001E01B78B8F1000F0ED0CDE90638CDE973
:1049900004CE1346CDE90267CDE90045084A11F07F
:1049A0009FF808B0BDE8F081CDE905E3CDE9037CCF
:1049B0001346CDE90156034A009411F091F8F0E74F
:1049C000C5990200E999020001480EF033BD00BF0D
:1049D00030220020F8B5184DD5E8AF3F13F0010F95
:1049E0002E4627D015F8C53CA5F1CC0783B901F0B8
:1049F000A3FC044628B14521104811F03AFB20469B
:104A0000F8BDFB7923B901F0D9FC04460028F2D1A6
:104A1000D5E8AF3F5A0701D401F03CF9D6E8EF3FA3
:104A200023F48032C6E8E12F0029F7D1DB0301D55A
:104A3000FFF7CAFF0024E2E7CC2000200A9A020018
:104A400010B5FEF775FB044620B102464521024829
:104A500011F00FFB204610BD339A020030B5002440
:104A6000094D0A4B85B02846029303940EF036FD9B
:104A700002AB284600934FF4A3620A2304490EF0C8
:104A800043FD204605B030BD282D00206C9A020061
:104A9000A84A0020014601480EF032BE282D002011
:104AA000014601480EF092BE282D0020034630B486
:104AB0001A780846012A13D0022A26D072B9154A5C
:104AC00002F1100452F8045BA24241F8045BF9D1F0
:104AD00012780A705B8843731B0A837330BC70477B
:104AE0000C4A02F1100452F8045BA24241F8045B44
:104AF000F9D112780A705B68C3F3072243731B0C69
:104B0000C3731B0A82730374E8E7112230BC194691
:104B100012F0F6BD759A020038B50546012D104613
:104B200019460CD0032D16D0052D14D00C490D4874
:104B30003D2211F08AFA3D21094811F07FFA0A4816
:104B400015F076F9044620B101210C3008F0F2FC92
:104B50002576204638BD02460B460448F0E700BFE4
:104B6000869A0200568D0200B028002014280020EA
:104B700010B50B460A490246D1F8380120B9BDE804
:104B800010400120FFF7C8BF08F0EEFD012100230F
:104B90000446017603820C3008F0CCFC204610BDA0
:104BA0000020002070B504460F2C0D461046194613
:104BB00005D80D2C0DD9BDE87040FFF7D9BF132CD7
:104BC00007D10C4815F034F9044638B900242046C2
:104BD00070BD02460B4645B10748F3E701210C3092
:104BE00008F0A8FC01232376F1E70120BDE870401E
:104BF000FFF792BF4C2900207C28002038B5C368FD
:104C0000B3F801401B7863B9204602F085FB0546E6
:104C100040B9084B1A8822B96FEA04506FEA105065
:104C2000188038BD012102F07FFB2846BDE83840DE
:104C300002F04ABB1C460020F8B5C5682E78BEB904
:104C4000B5F80170384602F067FB044630B93A46C1
:104C5000BDE8F8404521074811F00BBAEB78314622
:104C6000037302F061FB2046BDE8F84002F02CBB64
:104C7000F8BD00BFB59A020010B5C368B3F8014093
:104C8000204602F049FB30B92246BDE810404521DC
:104C9000034811F0EEB9BDE8104002F015BB00BFAB
:104CA000E09A020010B5C3681C88204602F034FB6D
:104CB00030B92246BDE810404521034811F0D9B96A
:104CC000BDE8104002F000BBE09A0200012108B5E7
:104CD0000C3008F0F3FDBDE808400278452101489A
:104CE00011F0C7B9099B0200014608B5074808F052
:104CF00041FC0749074816F046FD021E05DABDE8EB
:104D000008404521044811F0B4B908BD3C210020F9
:104D10007C220020482E0020309B020010B5084C59
:104D20000146052294F8670002F03CFD38B994F87A
:104D300067000422BDE81040024902F033BD10BDF7
:104D4000002000202E99020070B5C568B5F80160FA
:104D5000304602F0E1FA044630B93246BDE8704010
:104D600045210A4811F085B92B7823B90822E91C9E
:104D7000B53012F0C5FC201D4FF4805112F0B3FD88
:104D80002046BDE8704002F09FBA00BFE09A0200E2
:104D900030B405461446084602EBC3039C4201D1D9
:104DA00030BC7047224612F8081BA9420CD1028A77
:104DB0006378934205D92B4630BC4521034811F056
:104DC00058B9636830BC18471446E7E7529B0200A5
:104DD00010B5012104460C3008F070FD2146BDE8F5
:104DE00010400A23014A0078FFF7D2BFE483020093
:104DF00070B5444808F010FC0446002800F081809B
:104E0000027E012A4DD0032A78D1038A032B0BD8C6
:104E100040F2ED123C493D4811F017F9404080F353
:104E200011884FF0030002DF042104F10C0008F0A8
:104E300045FDFF22438806886276228AC6F30B006E
:104E40009342608307D04521314811F012F9204682
:104E500008F048FC14E002F05FFA054628B9452145
:104E6000628B2C4811F005F9F1E702F00FFB2146A7
:104E70006076320B284602F015F9284602F024FA33
:104E8000254BD3F83C31002B3BD02449244816F065
:104E90007AFC021E35DABDE870404521214811F048
:104EA000E8B8038A012B0BD840F66D121649174853
:104EB00011F0CBF8404080F311884FF0030002DF7F
:104EC000022104F10C0008F0F9FC0546007812F00C
:104ED000DCFC83070BD440F671120B490B4811F030
:104EE000B4F8404080F311884FF0030002DF06233E
:104EF00021460D4A2878FFF74BFFA8E745210B48CC
:104F0000B0E770BD3C210020799B0200568D020065
:104F1000AD9B0200D69B0200002000207C220020D6
:104F2000482E0020309B0200B4830200FD9B02004B
:104F3000F8B50746907A0E46144608F0D3F9284B88
:104F400083424BD1204608F0D5F90C23254D03FBB5
:104F500000504388BB4241D1234FD7F8380120B1DC
:104F600008F0C0FB0023C7F83831204608F0C2F92A
:104F70000C2707FB005043689BB196B9204608F008
:104F8000B9F9012107FB00504268D2E90003127A07
:104F900003F01F07B9405B09D2B100EB830012F0A8
:104FA000A2FC204608F0A6F90C2707FB00508368F6
:104FB000A3B1204608F09EF978432E54204608F00D
:104FC00099F907FB0055A868BDE8F8400DF008BF47
:104FD000C94300EB830012F091FCE2E7F8BD00BF8B
:104FE00018290020983C00200020002038B504211A
:104FF00004460C3008F062FC45780178224640886F
:10500000FFF796FF25B1BDE8384002480DF0E8BE35
:1050100038BD00BF2021002038B5032104460C30E4
:1050200008F04CFCE368057822461978B0F80100D6
:10503000FFF77EFF25B1BDE8384002480DF0D0BE35
:1050400038BD00BF202100202DE9F0470025A846EB
:10505000C768DFF8D0903B789D4201DBBDE8F08760
:1050600007EB8503B3F801A0B3F80360504602F0E4
:1050700053F90446D0B100F1280A46B34FF020039B
:10508000EFF3118283F31288BFF36F8FE369A3B14B
:10509000013BE36182F31188BFF36F8F204601F07B
:1050A0008FFF013E0DF09CFEB6B2E6E75246452169
:1050B0001D4810F0DEFF0135CDE763695BB982F36F
:1050C0001188BFF36F8F4521484610F0D2FF20466C
:1050D00002F0FAF8EFE7A16918688B42606108BF37
:1050E000A06182F31188BFF36F8F4FF02002EFF3BE
:1050F000118182F31288BFF36F8FDA68E261C3F81F
:105100000C80C3F80080626A4AB9C4E9083381F3AD
:105110001188BFF36F8F50460EF08CF9BEE7136015
:105120006362F4E7379C0200169C020073B5C56801
:10513000B5F80160304602F0EFF8044638B932465F
:105140004521284802B0BDE8704010F092BF2B788E
:10515000061D1A2B19D1C378012B2AD14FF4806177
:10516000304612F0C0FB42050FD4D4F8A83069468F
:105170000093D4F8B0302046019302F045FE20465B
:1051800002B0BDE8704002F09FB82B788BB9B5F83B
:105190000330A4F8A630B5F80530A4F8AC30B5F863
:1051A0000730A4F8AE306FF48071304612F0A6FBE1
:1051B00014E0D6E8AF3FDB05F5D52B78202BF2D1F4
:1051C00094F8B430002BEED0013B84F8B4304FF4A7
:1051D0002032002304F160000EF0F2FA204602F0C3
:1051E0009DF9CCE7E09A020010B5C1E900239DF8D3
:1051F00008300C460B7208F07DF80C22024B02FBC3
:1052000000335C6010BD00BF983C00202DE9F047E2
:105210004FF0FF3206464FF0FF331D480F4614F0A3
:1052200007FE044650B91B491B4840F2011210F01A
:105230000CFF40F20111174810F000FF4FF000087A
:1052400000F10C0A0121504608F074F9204684F858
:10525000188008F04FF84FF00C09104D09FB005072
:105260004680204608F046F809FB0050C0F8088048
:10527000204608F03FF809FB005503215046C5F8C9
:10528000048008F035FB068087702046BDE8F08773
:1052900018290020799B0200568D0200983C0020BE
:1052A00070B515460C4686B021B9FFF7AFFF04462E
:1052B000002841D001220021684616F001FA20465C
:1052C00008F018F80C231E4E03FB0060C0F808D04D
:1052D000204608F049FA01461A4808F0E3F94FF46D
:1052E000A022002368460DF0B5FD58B140F24912E6
:1052F0001549164810F0A9FE404080F311884FF080
:10530000030002DF204607F0F5FF0C235843365C0C
:1053100056B1204608F0E6F9092E14BF6FF00400DC
:105320006FF06E0006B070BD15B12C600020F9E77B
:10533000204608F0D7F9F9E76FF06800F2E700BF00
:10534000983C002044210020799B0200568D0200E9
:1053500073B506460D4642F22F00002101AAFFF761
:105360009FFF044630B14521084810F082FE2046D8
:1053700002B070BD0198C368B3F801203280B3F861
:1053800003302B8008F0AEF9F1E700BF539C020018
:10539000F7B5144B054693F993300C46002B1DDAF4
:1053A00014B9204603B0F0BD082C4FF0000142F2C2
:1053B000180001AA264628BF0826FFF771FF00281B
:1053C000F0D1019F3246F9682846013112F098F970
:1053D000384608F087F93544A41BE1E76FF08500F3
:1053E000E0E700BF002000202DE9F047B0F8017091
:1053F00000266FEA07536FEA135305468B4A9BB2A8
:10540000118888B0994204BF1680012600F0B4FDCF
:105410002C781FFA87F8F4B13C2C44D101F03AF90A
:105420006FF08001103012F069FA0020FFF776FC6F
:10543000054630B945217E4808B0BDE8F04710F078
:1054400018BE0473002101F06FFF284608B0BDE8C4
:10545000F04701F039BF2B7905F10409023B012B1C
:1054600024D8494606A812F03BFA9DF818300622C7
:10547000023B05F111010DF111008DF8183012F009
:105480003FF901238DF81030EB78012B21D04846ED
:10549000FFF7D2F945210246664810F0EAFD1F21C8
:1054A000404612F044FA08B0BDE8F087EB78494670
:1054B000012B04BF604B93F86740204612F052FB6B
:1054C000014606A812F00CFA494604A812F008FAA0
:1054D000DAE706A8FFF722FCEB780446012B0AD195
:1054E00001F0D8F882466FF08001103012F006FA11
:1054F000504612F051FC002CC9D0204606A920F8D5
:10550000907B12F0EDF90022B5F81730A4F8A63020
:10551000B5F81930A4F8AC30B5F81B30A4F8AE30AB
:10552000EB782273012BE37015D104A904F19700E5
:1055300012F0D6F901F0AEF8217A3F4DC1EBC1016E
:10554000294404F19E0012F0CBF9D5F8DC305D0659
:1055500001D501F04BFA0721204601F0E5FE1EB10E
:105560000121204601F0E0FE204612F09AFC637B08
:10557000072B53D1231DD3E8AF3F13F4805F2E4E8A
:105580001FD1E3781BB196F8D030180719D5022146
:1055900042F21600FFF73AFE0546002842D00221EB
:1055A0000C3008F0A5F9238800220380294642F236
:1055B0001600FFF775FE024618B145211F4810F08E
:1055C00058FD96F8D130D9070CD50021022320468A
:1055D0001A46009112F0E4F9024618B14521184824
:1055E00010F047FD96F8D0309A0617D5D6F86031FE
:1055F0009B689B0712D50DF10E0103A8FFF7A8FECB
:1056000060B9BDF80E202046BDF80C1012F0AAF9C2
:10561000024618B145210B4810F02BFD204601F041
:1056200053FE40E76FF06802C7E700BF1C4600204A
:10563000789C02009E9C020000200020BF9C02007B
:10564000E59C0200019D020010B5C16888B00B788E
:10565000164C8DF80030B1F8013001A8ADF80130DA
:10566000CB7804318DF80330B1F80730ADF817303E
:10567000B1F80930ADF81930B1F80B30ADF81B3086
:105680004B7B8DF81D3012F02BF9214606220DF1CF
:105690000B0012F035F8062221460DF1110012F030
:1056A0002FF86846FFF7A0FE08B010BD429902002F
:1056B00029289ABF014B185C09207047AC9E020054
:1056C00070B5C368B3F801601D78304601F024FE60
:1056D000044630B93246BDE870404521154810F007
:1056E000C8BC65B12846FFF7E3FF294602462046BD
:1056F00001F0ECFF2046BDE8704001F0E5BD837885
:10570000012BEFD106F05EF9204612F0D1F8002807
:10571000E8D10520FFF7CCFF05210246204601F025
:10572000D5FF4521044810F0A4FC0521204612F0C5
:10573000C1FBDFE7B59A0200229D0200F8B5C668FA
:10574000B6F801703578384601F0E6FD044630B908
:105750003A46BDE8F84045211A4810F08ABC65B1C8
:105760002846FFF7A5FF29460246204601F0AEFF76
:105770002046BDE8F84001F0A7BD8278F378012A01
:10578000C37205D00020FFF793FF00210246ECE72B
:105790000BB106F017F9204612F08AF80028F1D173
:1057A0000520FFF785FF05210246204601F08EFF08
:1057B0004521054810F05DFC0521204612F07AFBDA
:1057C000D6E700BFB59A0200229D0200024BD3F833
:1057D00060315B69184700BF0020002038B50546DE
:1057E0000C4619B9FFF712FD0446C0B140F6354327
:1057F0009D420ED12046FFF7E9FF054668B10246FB
:105800004521084810F035FC204607F06BFF28467C
:1058100038BD2146044807F045FF0025F7E76FF043
:105820006805F4E74D9D020044210020F8B50446C8
:10583000458B467E807A07F055FD214615F036FFF0
:105840001B4B93F882309B0631D5304602F0A8F905
:1058500068B3437B073B012B03D9BDE8F84001F057
:1058600033BD01F031FD052140F63540FFF7CEFC98
:10587000044628B9BDE8F84045210E4810F0F9BBB0
:1058800000F10C070121384608F032F80126042106
:105890000670384608F02CF8002305808670C37027
:1058A0002146BDE8F84040F63540FFF797BFF8BD08
:1058B00000200020749D0200F0B5C46887B02688DF
:1058C000B7B2384601F028FD054638B93A464521B9
:1058D000204807B0BDE8F04010F0CBBB02AFD4F8D1
:1058E0000220D4F8063001976189009113F01CFE64
:1058F000F8B1122142F21A00FFF788FC044640B9C1
:105900004521154810F0B5FB284601F0DDFC07B035
:10591000F0BD12210C3007F0EBFF3946102220F8C1
:10592000026B11F0EDFE214642F21A00FFF756FF1E
:10593000EAE7022142F21B00FFF768FC0446002858
:10594000DED002210C3007F0D3FF2146068042F260
:105950001B00EBE7E09A02009C9D020070B5064632
:105960000D4642F221000321FFF750FC044628B9FE
:10597000BDE870404521084810F07BBB03210C3086
:1059800007F0B6FF068085702146BDE8704042F200
:105990002100FFF723BF00BFB89D0200F7B5C36821
:1059A000D9789A781F8842EA0122ADF80020597907
:1059B0001A79BCB242EA0122ADF802209A79D9796B
:1059C000204642EA0122ADF804201A7A5B7A42EAC4
:1059D0000323ADF8063001F09FFC064650B945217F
:1059E0001C48224610F045FB02212046FFF7B6FF77
:1059F00003B0F0BD694601F0E1FD38B91E21204633
:105A0000FFF7ACFF304601F05FFCF1E70E2142F2F8
:105A10002000FFF7FBFB05460028F3D00E210C30D9
:105A200007F066FF04460E22002111F074FE278065
:105A3000BDF8003029466380BDF8023042F22000F4
:105A4000A380BDF80430E380BDF806302381FFF762
:105A5000C5FED7E7E09A02002DE9F047414FDFF895
:105A6000088107F11409FB6848466FF39433FB6023
:105A700001F0CEFB451C4FF0FF324FF0FF332946BB
:105A800038480FF093FC58B140F6E61241463748CB
:105A900010F0DBFA404080F311884FF0030002DF82
:105AA000304E15B90EF058FDDDE7F368C3F38633C9
:105AB000042B4CD1337B002B4CD1002200232C48EB
:105AC00014F0BBF9044658B94FF418624146274810
:105AD00010F0BBFA404080F311884FF0030002DF62
:105AE000DFF890A04FF0FF334FF0FF3222480DF067
:105AF000B1F9DAF8383153B14521204810F0B9FA3C
:105B0000DAF8380107F0EEFD0023CAF838312046F4
:105B100007F02AFECAF838012046FFF757FE024672
:105B2000A8B14521164810F0A4FA13480DF058F911
:105B3000204607F0DFFB0C22124B1F2102FB003036
:105B400022464088FFF7F4F9204607F0CBFD1436D3
:105B5000013DA6E7012BFAD13069383801F08CFFFE
:105B6000F5E700BF40220020799B0200568D02001D
:105B7000442100200020002020210020D79D020089
:105B80004D9D0200983C00202DE9F041044600F1B3
:105B90000C06304614F062F9B4F810800546B8F1EE
:105BA000010F0BD840F67B521A491B4810F04DFAF2
:105BB000404080F311884FF0030002DF304602219D
:105BC00007F07CFE0746007811F05FFEC20706462C
:105BD0000BD440F67F520F490F4810F036FA404080
:105BE00080F311884FF0030002DF052321460B4AA2
:105BF0003878FFF7CDF8B30707D56369A4F81080AC
:105C000013FA85F5E560BDE8F0812046BDE8F04176
:105C100007F068BD799B0200568D02008C8302005C
:105C200038B5027E0446012A05D0032A11D1FFF7B8
:105C30005BF8002038BDC368187811F026FEC20753
:105C4000054602D52046FFF79FFFAB07F1D520465A
:105C5000EDE74521044810F00CFA204607F042FD1C
:105C60006FF01500E6E700BFF79D0200084A034603
:105C7000D2F8600130B9D96839B1596929B1C2F88F
:105C8000603170476FF0770070476FF01500704714
:105C9000002000200421014811F025BECC20002066
:105CA00010B5FAF7C1FC034B1B6813B1BDE81040F7
:105CB000184710BD103D002070B5354D0646D5F88B
:105CC000603188B043B94521324810F0D2F96FF005
:105CD0001204204608B070BD6FF0020105F1CC003F
:105CE00011F00CFE012111F0FEFDC3074DD4FEF7AB
:105CF000A7FE04460028ECD1274B1E60012205F5C3
:105D00009070114615F0DCFC05F5A27015F0B6FC9C
:105D100000220023CDE906236FF008034FF48062D0
:105D2000CDE90243CDE900441C4B1D4904941D48B4
:105D30000CF048FD1C491B4815F077FC1B480DF082
:105D4000CDFB6FF0070340F69802194917480094FD
:105D50000DF0DAFB1749154815F067FCD5F86031EE
:105D6000DB689847044628B102464521124810F0E6
:105D700080F9AEE726B908B0BDE87040FAF754BC28
:105D800005F1BC000DF056FBA3E76FF07704A0E728
:105D900000200020619E0200103D0020591A0100E1
:105DA000C04F0020C82D00207F9E0200482E0020FA
:105DB000C0530020859E02008B9E02000048704761
:105DC000198D0200F8B506460025094FFB79ECB2A3
:105DD000A34202D86FF0010009E0C4EBC4013046D1
:105DE000394411F034FE01350028EFD02046F8BDCB
:105DF0000020002037B504460D46A9B128461649B3
:105E000011F025FE80B929461448C4EBC40420448F
:105E100011F025FE124811F025FE430701D5FEF7CB
:105E2000D3FD002003B030BD684611F020FD0028EE
:105E3000F8D16846FFF7C6FF0028F5DA074BC4EB38
:105E4000C4041C446946204611F009FE002DE1D02F
:105E500021462846DCE700BF3599020000200020DB
:105E6000CC20002038B506221249054611F021FC4D
:105E7000D8B1062142F20500FFF7C8F90446B0B1D7
:105E8000062229460C3013F0F5FF0022214642F28B
:105E90000500FFF705FA48B906222946054811F022
:105EA0002FFC0122044B83F86020002038BD6FF0E6
:105EB0006800FBE761200020002000202DE9F04170
:105EC00005460C4686B051B929494FF45772294806
:105ED00010F0BBF84FF45771254810F0AFF8086880
:105EE00040B9234940F25D32224810F0AEF840F24A
:105EF0005D31F1E745B91E4940F25E321D4810F0B0
:105F0000A4F840F25E31E7E7037A5A0708D518494A
:105F10004FF45872174810F098F84FF45871DBE7B7
:105F20004F68F7B92B7A5B071BD5691C013011F05C
:105F30008EFDD4F80080162239460646684611F0D8
:105F4000EAFB1022694608F12A0011F0B2FB58B1B1
:105F50002068102205F12A012A3011F0AAFB18B995
:105F6000656006B0BDE8F081002EF9D1F9E700BF09
:105F7000E29E0200568D0200084BD3E8EF2F22F478
:105F80000041C3E8E01F0028F7D1130404D5002224
:105F90000220034905F00CBE704700BFCC20002052
:105FA000C33B0200002307B50549CDE900036A465B
:105FB000022005F0FDFD019803B05DF804FB00BF71
:105FC000BD1E0100F7B5054670B1494C94F8182183
:105FD00094F819310AB19A4208D2013384F8193180
:105FE0002B7A43F004032B7203B0F0BD002106228C
:105FF000084601F0D7FB064688B1CC34D4E8EF3F21
:1060000043F40043C4E8E23F002AF7D12B7A43F07F
:1060100001032B7203B0BDE8F04001F055B9014611
:10602000344800F031FB94F819318BB994F81921F8
:1060300094F818319A4224D1002242F229001146E4
:10604000FFF72EF998B145212B4810F012F804E023
:10605000304611F044FD0028E8D0012011F03FFD4A
:106060000021264803B0BDE8F04000F00DBB94F8D5
:106070001931013384F819312B7A43F004032B7260
:10608000EBE72A466F1C394612F82A0B11F0EDFC9B
:10609000064610B145211A48D7E794F81931013363
:1060A00084F819312B7A43F004032B7294F89F3053
:1060B0005B07D2D53946684611F0D1FC012308218F
:1060C00042F24E008DF80730FFF7A0F8044660B1A9
:1060D000082269460C3013F0CDFE3246214642F2CA
:1060E0004E00FFF7DDF80028B7D045210548ACE7A2
:1060F00000200020353B0200109F02000F3B0200F1
:10610000359F02005A9F02002DE9F041054698B3E1
:10611000444C94F8182194F81931D2B101329342C9
:1061200023DC00210622084601F03CFB064628B38A
:10613000CC34D4E8EF3F43F40043C4E8E23F002A04
:10614000F7D12B7A43F002032B72BDE8F04101F046
:10615000BBB853B93449354840F223420FF075FFBC
:1061600040F2234130480FF069FF013B84F81931B8
:106170002B7A23F004032B72BDE8F08101462C48F2
:1061800000F082FA304611F0AAFC064680B10246C1
:10619000452128480FF06DFF94F8193113B1012003
:1061A00011F09DFCBDE8F0410021234800F06CBADD
:1061B00094F8193194F818219A420CD2013B84F8D2
:1061C00019312B7A024623F0040302201B492B725B
:1061D00005F0EEFCE0E7072142F22800FFF716F891
:1061E00005F10108074620B9452115480FF041FF88
:1061F000D2E707210C3007F07BFB414611F02FFC62
:106200003246394642F22800FFF74AF80028EBD11F
:1062100094F81931013B84F819312B7A23F00403E7
:106220002B72B9E700200020E29E0200568D02008A
:10623000353B02007A9F02000F3B0200C93A020080
:10624000AC9F020070B50D46044618B9E5B16FF079
:10625000150070BD1D4911F0FAFB0028F6D1237816
:10626000012B04D1A37903F0C003C02B04D0452136
:1062700017480FF0FEFEEAE72046FFF7A3FD0028CF
:10628000E4DB6FF07700E4E7124DEB79012B1AD0D5
:1062900005F1CC0011F0E6FBC3070BD5EE792146E2
:1062A0003046FFF7A7FD0028D3D1EB793046013304
:1062B000EB71CEE7002CCAD02046044911F0C7FB91
:1062C0000028EBD0C3E76FF00B00C2E7359902005E
:1062D000D69F02000020002073B5044698B100212B
:1062E00041F2090001AAFEF7DBFF064658B9019BFF
:1062F0000622DD680E490135284611F0DAF928B981
:10630000019807F0EFF9002002B070BD0622284680
:10631000084911F0CEF90028F2D006222946601C67
:1063200011F0EEF90198267007F0DCF90120EBE797
:10633000429902003C99020007B56846FFF7CCFF7E
:10634000044BD87118B169460020FFF753FD03B024
:106350005DF804FB002000202DE9F341164B0746B1
:1063600093F8BA308846DB0704D40026304602B0E2
:10637000BDE8F08100214FF6094001AAFEF790FF29
:1063800004460028F1D1019BDD686E780235464550
:1063900028BF46464FF01608A64203DC019807F0D6
:1063A000A1F9E3E7294608FB0470162211F0A8F9C9
:1063B00001341635F0E700BF00200020F0B5154E7F
:1063C00089B0F4792CB9012102A8FFF7C5FFF0715B
:1063D000C8B90021084609B0BDE8F040FFF732BF58
:1063E00002AB07FB053106220DF1010011F088F91F
:1063F0000123694628468DF80030FFF7FBFC013485
:1064000010B109B0F0BD1627F379E5B2AB42E7D879
:106410000020F6E7002000202DE9F04190460E46CE
:106420001D46024600284BD0002B49D0CF070478E8
:1064300031D5254FB8F1000F13D088060AD4C4EB2C
:10644000C403FB5C012B15D02B70B2060FD543F0B3
:1064500002030BE097F8D0305906F0D46FF08500B6
:1064600006E0C4EBC403FB5C012B03D02B700020BF
:10647000BDE8F081072101FB04711046013111F0E4
:106480007DFB0028F4D1C4EBC4043B5D2B70B8F154
:10649000000FECD0D9E74B070ED50B4EC4EBC40769
:1064A000F35D012BE2D1072111FB0431314411F0DE
:1064B00065FBF35D2B70DBE711F068FB0123F9E767
:1064C0006FF01500D4E700BF002000202DE9F74F42
:1064D0000C46202192460090FEF798FE05460028C3
:1064E00054D020210C3007F003FA202281460021ED
:1064F00011F011F9002609F1010B04EBCA0A00237F
:10650000D4F80080626893420CD30834A245F6D1D7
:1065100000222946009889F8006003B0BDE8F04FDA
:10652000FEF7BEBE98F80120B01C11181F2998F87C
:1065300000C014D9BCF1090FC0F11F0201D1002A1B
:106540000BDC452113480FF094FD284607F0CAF8EC
:106550006FF0150003B0BDE8F08F4FF0080CD7B214
:10656000791C0BF80610711CC9B20BF801C0D8F8E1
:1065700004105BFA80F00193023711F0C1F8019B1F
:106580003744FEB2013308F10808BBE76FF068003A
:10659000E0E700BF0FA0020070B50546164B15F8E6
:1065A000092B044683F867200E4607222846134924
:1065B00011F07FF8034620786BB9114901F0BCF85F
:1065C000044610B96FF00B0070BD042100F0ACFE62
:1065D00000203460F8E7294611F0E2FC40B9207849
:1065E000294601F0A9F804460028EBD00521EDE783
:1065F0006FF01500E8E700BF002000203599020089
:106600002E99020038B543680446580501D500208C
:1066100038BD22690AB1D907F9D5194D2078EB792F
:106620008342F4D9C0EBC00007221649284411F078
:1066300040F80028EBD06068C20706D495F86830AF
:10664000082B02D8A3689F2BE1D910F0300F02D09D
:106650002369002BDBD0C30601D4236943B9D4E9F5
:1066600002239A42D3D81F2AD1D9B3F5804FCED86E
:1066700000F46030B0F5603018BF0120C8E700BFFB
:10668000002000203599020003460148184700BF4A
:106690001820002000487047182000202DE9F04FF6
:1066A0009A460023D1F810908DB0B9EB0306054649
:1066B000904818BF01260592079311F0A3FA4207EC
:1066C0000C4640F10B810846FFF79CFF28B96FF09C
:1066D000150B58460DB0BDE8F08F204611F06DFA4D
:1066E00080460028F3D005F11007384611F08AFAE9
:1066F0000306C0F3C01B00F1F4800F22594608A81E
:1067000011F009F8A3686068ADF82030E368ADF8CF
:10671000223011F068FA2A7823788DF82D009A42F9
:106720008DF82EB004D06FF40051724811F06DFA5C
:106730002378714A2B7082F86730284632466168A8
:106740000DF12503FFF768FE83460028C1D107221B
:1067500005F10900B9F1000F13D0216910F0D0FF45
:10676000204611F0E2FA62680646D00716D4920578
:1067700003D4169B0BB9022E52D102238DF824307C
:106780001AE05E4910F0BCFF204611F0CEFA6268B4
:106790000646D107EBD58DF824900DE012F0100FCE
:1067A0000CBF0122042221698DF824200DF126005E
:1067B000072210F0A5FFD8460F2142F20600FEF78F
:1067C00025FD8346002800F08F800F2208A90C3099
:1067D00013F050FB0022594642F20600FEF760FD1E
:1067E000002840F08480B9F1000F1FD06368DB07F8
:1067F0002AD42846012111F0A8FA079D83460028D3
:1068000064D045213E480FF034FC002D3FF461AFC9
:106810002846002100F088FD284600F055FD58E785
:106820000323DDF858808DF82430C5E7179B5246C6
:1068300000932846CDE90186169B059911F003FACD
:1068400083460028D2D044E7284607A9FFF7A4FED4
:1068500083460028CDD010F10C0F7FF43AAFB9F188
:10686000000F7FF436AF626890073FF532AF636880
:1068700083F00203C3F3400B0BF001020E213846F4
:1068800011F0CEF9731E5A425A410821384611F0D0
:10689000C7F9B11E4A424A413846092111F0C0F9F0
:1068A00062680A21384602F0010211F0B9F9424645
:1068B0000B21384611F0B4F962680D213846C2F355
:1068C000800211F0ADF94FF0000B02E715B1284638
:1068D00000F0FAFCB9F1000FCED1C8E76FF00A0B57
:1068E000F7E66FF0770BF4E66FF0680BF1E683469E
:1068F000EFE600BFCC2000200020002035990200E8
:106900002DA0020073B51546069A0C46CDE900325B
:106910002B460A4601461148FFF7C0FE21460646AF
:10692000002340F201109D4202D1304602B070BDFA
:106930000A88824204D14A6812B11278D20702D47E
:1069400001330831EFE7064906480CF0B3FE4FF477
:106950007022002303480CF097FFE6E71820002080
:106960009F3D02003020002010B51A4811F014FAA3
:106970006FF48041184811F048F9174811F042F9B6
:1069800003461A06C0F3C01023D5134811F03AF994
:10699000430514D507221149114810F08AFE114B06
:1069A00098B904221049187E00F0FCFE044630B16C
:1069B0000021017300F0B8FC204600F085FCBDE822
:1069C00010400021034811F0C0B9052203F1210154
:1069D000E9E710BD1820002028200020359902008A
:1069E00021200020002000202E99020073B51E4CAB
:1069F000204611F007F9400434D5204611F002F981
:106A000001062FD4204611F0FDF842052AD501A930
:106A1000A4F11000FFF7C0FD054618BB0121A4F149
:106A2000100011F092F9019E28B9304602B0BDE87D
:106A3000704000F049BC2946304600F075FC6FF408
:106A40008041204611F0E1F80546304600F03CFC5C
:106A50006B0407D5D4E8EF3F43F48043C4E8E23F3A
:106A6000002AF7D102B070BD2820002030B58DB0CB
:106A7000202104A8FEF78CFC0446E0B914F0C9FEFE
:106A80004FF47A75A0FB053205FB0121DB0B43EACD
:106A90004143C90BCDE90231082320220093074866
:106AA0006B4404A910F0C1FC28B9452104480FF03B
:106AB000E0FA6FF0040420460DB030BDE82E00204F
:106AC00054A00200884208B501F110030CD9984285
:106AD0000FD20C490C4840F215220FF0B6FA40F2E2
:106AE000152108480FF0AAFAF3D000F110029142E4
:106AF000EEE7013813F8012D8B4200F8012FF9D190
:106B000008BD00BF70A00200568D020007B5082125
:106B10006846FEF73DFC58B908226946074810F060
:106B200064FC40B9064845210FF0A3FA6FF0040059
:106B300003B05DF804FBFFF799FFF9E7E82E0020AA
:106B4000A2A0020038B50D46044698B191B10B4A97
:106B500010F084FC431C07D1FFF788FF48B9294691
:106B60002046064A10F07AFC01280CBF00206FF086
:106B7000040038BD6FF01500FBE700BFE82E0020D1
:106B8000402208B5034910F094FDB0FA80F04009A6
:106B900008BD00BFFFA0020070B52D4B93F89A30DE
:106BA00003F00603062B4AD100284BD0294E326849
:106BB00032B1131F834248D05B680BB1043BF9E745
:106BC00042607268031D336002B97360224CD4E8DE
:106BD000EF2F42F02003C4E8E13F0029F7D112F083
:106BE000200202D00025284670BDD4E8EF3F23F0F4
:106BF0001003C4E8E13F0029F7D1114642F2250015
:106C0000FEF74EFB05460028ECD0452113480FF057
:106C100030FAD4E8EF3F23F02003C4E8E23F002A33
:106C2000F7D134683CB154F8043C043C0BB100206B
:106C300098476468F6E70023C6E90033D3E76FF0AE
:106C40008505D0E76FF01505CDE76FF07705CAE74A
:106C500000200020183D0020CC200020D0A0020001
:106C6000044BD3E8AF3F13F0100F034808BF0020D8
:106C7000704700BFCC2000205E460020F8B51C4DB8
:106C800006462B688B422CD013B16FF00F00F8BD75
:106C9000184BD3E8AF2FC2F340179206F5D4D3E8D0
:106CA000AF3FDB0620D5296042F226004021FEF7E7
:106CB000ADFA044690B140210C3006F019FE402296
:106CC000314610F01DFD3A46214642F22600FEF7FD
:106CD000E7FA0028DBD000232B60D8E76FF06800CC
:106CE000F9E76FF07700D2E76FF07C00CFE700BFE5
:106CF000143D0020CC200020F8B5174CC668D4E81D
:106D0000EF3F23F02003C4E8E23F002AF7D13378B5
:106D100063B940221148711C10F0F2FCD4E8EF3F37
:106D200043F01003C4E8E23F002AF7D10C4D2C6871
:106D30006CB10A4F043C23682BB13278002A0CBF97
:106D400038460020984764680CB1043CF3E7002300
:106D5000C5E90033F8BD00BFCC2000205E4600200E
:106D6000183D002005490B6833B1C2680020086057
:106D7000117801B9501C1847704700BF143D00201E
:106D800070B50446104B1D6875B9104D104EB542D4
:106D900018D91049104840F25B520FF056F940F2F2
:106DA0005B510C480FF04AF92B6813B12046217B48
:106DB0009847AD69E8E72B6813B12046217B9847D7
:106DC0001C35E4E7F7D370BD503D0020AC7D0200D8
:106DD000E47D020046A10200568D02002DE9F0413B
:106DE00004464FF00008144F4FF02002EFF31183D8
:106DF00082F31288BFF36F8F216A29B983F3118858
:106E0000BFF36F8FBDE8F081606A0A68814208BFF6
:106E10006262226283F31188BFF36F8FD1E901565A
:106E20003846C1E90188C1F80C8014F034FC002216
:106E300031462046A847D7E7F827002070B504461A
:106E400041B90D490D4839220FF0FFF839210A48A0
:106E50000FF0F4F80022D1E90156CA60C1E901221D
:106E6000074814F018FC314620462B46BDE8704018
:106E70006FF06D02184700BF46A10200568D020058
:106E8000F82700202DE9F84304460E461746994698
:106E90008D694FF0FF334FF0FF3245480BF0DAFFBA
:106EA000637B072B78D14FF02003EFF3118283F33C
:106EB0001288BFF36F8F002D43D000232B60A3698E
:106EC000002B3BD1C4E9055582F31188BFF36F8FC6
:106ED000042106F10C0006F0BBFC238807F0FD0737
:106EE00043EA07370780338A043B43800223304656
:106EF0003376FEF76BFC0246002857D045212D481B
:106F00000FF0B7F84FF02003EFF3118783F31288E7
:106F1000BFF36F8F15B3294604F1140010F06DFF15
:106F200087F31188BFF36F8F21480BF059FF0023BF
:106F300029462046B361FFF781FF27E01D60A56168
:106F4000C2E7A36933B103F10C08DB680133C8F869
:106F50000030B9E7E36904F11C08F7E7D8F800202E
:106F600052B91549154840F227220FF06EF840F249
:106F7000272111480FF062F8013AC8F8002087F382
:106F80001188BFF36F8F0A480BF02AFFB9F1000F89
:106F900008D10020BDE8F88305480BF021FF002D43
:106FA000C5D1F3E7304606F09DFBF2E70120F1E79B
:106FB000002100204D9D020046A10200568D0200D6
:106FC000004870470021002038B5002204468A425C
:106FD00002D10024204638BD012004F1C403D3E8C7
:106FE000EF5F002D04D1C3E8EC0FBCF1000FF6D128
:106FF00002D0C8340244EAE7002CEAD0C4220021BF
:10700000204610F088FB04F1600004490CF052FBAC
:10701000034904F128000CF073F9DBE71139010092
:10702000473E02002DE9F0410446002704F13806EE
:1070300000230022304612F000FF034660B9636966
:10704000ABB116494FF42D7215480EF0FEFF4FF408
:107050002D7112480EF0F2FF9D699F6106F042FB10
:10706000002DE5D029462046FFF7E8FEDEE7E3697C
:1070700043B10A4940F2B52209480EF0E6FF40F25A
:10708000B521E6E7204610F0E1FE04F160000022A1
:10709000BDE8F04100230CF0F7BB00BF46A10200A1
:1070A000568D020070B5164604460D46FFF796FE53
:1070B000012E1FD0022E49D1236933B12B4845211F
:1070C0000EF0D7FF204610F0C1FE256121690A8A23
:1070D000012A49D9CB681B8804339BB29A4243D317
:1070E0003AD9234845210EF0C4FF2046BDE8704040
:1070F00010F0ACBE206938B945211E480EF0B9FF2A
:10710000204610F0A3FE01E02E8A26B92846BDE8ED
:10711000704006F0E7BA0C3012F0A4FE86420BD99C
:10712000452115480EF0A5FF00222046216900F0F8
:1071300043FE00232361E9E720692A8AE9680C30CD
:1071400012F098FE284606F0CDFABFE732464521F8
:107150000A480EF08EFFD3E7002323612046BDE8E6
:107160007040012200F028BE70BD00BF76A1020071
:107170000AA2020098A10200BBA10200E7A102003E
:10718000F8B51F46437B0446072B0E46154606D02E
:1071900045211B480EF06DFF6FF07F0016E062B3D3
:1071A0000DF004FB174B8342174807BF0022002352
:1071B0004FF0FF324FF0FF330BF0BAFD014630B90C
:1071C000124845210EF055FF6FF06800F8BD637B53
:1071D0000022072B06D0C0E90122C2600A4814F041
:1071E0005AFAD9E7C0E90157C260B16104F1380029
:1071F000314606F057FA0020E8E71146F5E700BFF0
:107200002AA2020020360020F82700203EA2020019
:1072100070B50446174814F0BDFB0022012120463A
:10722000144B0EF099F804F11406134BD3E8AF2F6A
:107230000AB9012070BDA3F1C40513F8B73C53B9D6
:107240006FF04001281D10F0F3FD430603D52846DA
:10725000FFF7E8FEEDE76B7B072BEAD13046074BE3
:10726000002204210EF078F80123022084F8203057
:10727000E0E700BF8C220020E430002058300020DE
:1072800010B580B100F1C402D2E8AF3FB3B1591CD0
:10729000D2E8EF4F9C4204D1C2E8EC1FBCF1000FD2
:1072A000F6D1F1D110BD0649064840F27C420EF0FD
:1072B000CCFE40F27C4102480EF0C0FE1846F1E7D9
:1072C00046A10200568D020010B500F1C403D3E8B8
:1072D000EF2F511EC3E8E41F002CF8D1002A0ADC6E
:1072E0000B490C484FF493620EF0AFFE4FF49361DC
:1072F00007480EF0A3FE40F201124188914206D1E8
:10730000D3E8AF3F1BB9BDE81040FFF76FBB10BD1E
:1073100046A10200568D020002460121014810F0EC
:107320009EBD00BF2030002070B5457B04468D42D5
:1073300000F08980417325B98378082B01D0FFF7CD
:107340009FFF637B012B16D100264E4D4FF020028C
:10735000EFF3118382F31288BFF36F8FE269002A83
:107360006BD0013AE26183F31188BFF36F8F284637
:107370000BF036FDEAE7072B09D0002B63D1A37889
:10738000042B21D12046BDE87040FFF79DBFA378B4
:10739000042B58D004F1380014F070F900213A4859
:1073A0000EF0B6F80023C4E91533E378012B4AD177
:1073B000032384F8B43004F160004FF42032BDE8B8
:1073C000704000230CF0FCB9013D052D3BD801A312
:1073D00053F825F0ED3301002D3401008533010011
:1073E000853301002D3401002D3401002046FFF7C4
:1073F000F5FCA378012B0AD104F16005284614F0AE
:10740000D3F910F00C0F02D028460CF043FA0434E4
:10741000D4E8EF3F43F04003C4E8E23F002AF7D14D
:10742000BDE87040002118480EF072B8237B002B95
:10743000A8D02046FFF7A4FCA4E7616921B983F333
:107440001188BFF36F8F70BDA0690A68814208BFC1
:10745000A261626183F31188BFF36F8F4FF0200246
:10746000EFF3118382F31288BFF36F8FCA68E26172
:10747000CE6083F31188BFF36F8F2046FFF7DEFCE9
:1074800075E700BF002100208C2200200A4A08B5C1
:107490000A49831ADB10904201FB03F30AD0084922
:1074A000084840F2B6420EF0D0FD40F2B641044822
:1074B0000EF0C4FDD8B208BD20300020295C8FC278
:1074C00046A10200568D0200F8B504460D46174647
:1074D0001E4614F0A4F850B10D490E4840F2D242B5
:1074E0000EF0B3FD40F2D24109480EF0A7FD0A4963
:1074F0003A46002C14BF20460846334612F098FC4A
:10750000044618B1691D0C3006F014F82046F8BD89
:1075100046A10200568D020048280020F8B5044616
:107520000430D0E8AF3F9B0511D5B4F8A630B4F8CD
:10753000A8209A420BD8B4F8AA209A4207D3D4E9DB
:107540002B239A4203D16FF4007110F071FC164B9B
:107550001D6875B9154D164FBD4222D915491648FB
:1075600040F2A5520EF071FD40F2A55111480EF007
:1075700065FDEE683EB12046B4F8AE30B4F8AC20FC
:10758000B4F8A610B047AD69E3E7EE683EB1204617
:10759000B4F8AE30B4F8AC20B4F8A610B0471C353F
:1075A000DAE7F2D3F8BD00BF503D0020AC7D020009
:1075B000E47D020046A10200568D02002DE9F04153
:1075C000074608460C4610F016FA054618B900257D
:1075D0002846BDE8F081194B1E687EB9184EDFF8C9
:1075E0006480464523D91849184840F2ED520EF000
:1075F0002CFD40F2ED5114480EF020FDB3680BB99C
:10760000B669EAE72146384698470028DFD0204689
:1076100010F0F1F90028F3D1D9E721463846984710
:107620000028D4D0204610F0E6F920B9CFE7CFD219
:10763000B368002BF1D11C36D3E700BF503D0020CA
:10764000AC7D0200E47D020046A10200568D0200DE
:107650002DE9F041C3780446BBB900F19E06164BF4
:1076600004F190071D689DB9144D154F04F1900861
:10767000BD421DD91349144840F2BC720EF0E5FC1E
:1076800040F2BC710F480EF0D9FC00F19706E6E716
:107690002B691BB13A46314620469847AD69E2E76F
:1076A0002B691BB142463146204698471C35DFE71F
:1076B000F6D3BDE8F08100BF503D0020AC7D020054
:1076C000E47D020046A10200568D0200F8B5437A1F
:1076D00004468372164610F002FD124B1D6875B900
:1076E000114D124FBD421AD91149124840F62802D5
:1076F0000EF0ABFC40F628010D480EF09FFC6B69C4
:107700001BB132462046617A9847AD69E7E76B695D
:107710001BB132462046617A98471C35E2E7F6D322
:10772000F8BD00BF503D0020AC7D0200E47D0200AA
:1077300046A10200568D020070B506460D460A4865
:107740000121FFF741FC044660B106720722294679
:1077500090300FF0D5FF01236372A372A370034B27
:10776000C4F8A830204670BD203000201800280042
:1077700070B505460A480E46FFF782FD044620B163
:107780008378012B04D0FFF79FFD0024204670BDB5
:107790003246294610F0E4FB0028F7D12046F2E7F4
:1077A00020300020F8B505460E480E461746FFF774
:1077B00067FD044620B18378012B03D0FFF784FDD9
:1077C00000240DE036B13246294610F0C9FB08B955
:1077D0002046F3E7637BBB42FAD1237AAB42F7D171
:1077E0002046F8BD2030002010B5837802460B708B
:1077F000C3784B70037A8B70437B082B0FD8264CD1
:10780000E35C0B770023CB77437A4B7710F072FB66
:1078100088779378012B0DD06FF0150010BD1F49AC
:107820001F4840F60E120EF010FC40F60E111B48D9
:107830000EF004FC02F190038B60137A1948C3EB3D
:10784000C30303444B60D47802F19E0302F1970016
:1078500014B11C4603462046C1E90303B2F8A63022
:107860008B82B2F8AC30CB82B2F8AE300B83D2F858
:10787000C03023B15B7BD80644BF0123CB77D2F85D
:10788000C03013B15B7B9B0601D40020C6E7CB7FE1
:1078900043F00203CB77F8E761A2020046A10200A1
:1078A000568D02000020002038B5044608460D46DB
:1078B00010F0A1F838B3154B93F8D030990707D4DE
:1078C000E37873B129462046BDE8384000F09CBA01
:1078D00094F8B5309A07F3D5231DD3E8AF3F5B0585
:1078E000EED42946204610F065FB58B92B88A4F841
:1078F000A8306B88A4F8AA30AB88A4F8B030EB8825
:10790000A4F8B23038BD6FF01500FBE7002000206E
:10791000F7B510F8533C0446A0F160065BBB304657
:1079200010F0C5FB304B1D6875B9304D304FBD426E
:107930001AD93049304840F26C520EF086FB40F2C2
:107940006C512C480EF07AFB6B681BB1304614F872
:10795000541C9847AD69E7E76B681BB1304614F8D3
:10796000541C98471C35E2E7F6D3304603B0BDE817
:10797000F040FFF7A9BC10F85E3C012B1ED1A0F12E
:107980005C056FF40071284610F052FA830517D594
:10799000A36C69460093236D30460193FFF784FF83
:1079A00020B96FF48071284610F042FAD5E8EF3F15
:1079B00043F08003C5E8E23F002AF7D103B0F0BDF1
:1079C0006B460E4A1068516803C369463046FFF79C
:1079D0006BFF0028EAD1D5E8EF3F43F48073C5E898
:1079E000E23F002AE2D0F6E7503D0020AC7D0200E5
:1079F000E47D020046A10200568D020024800200B0
:107A000001460148FFF760BDE42800202DE9F04160
:107A100006464FF0FF334FF0FF3200200C46FFF7D1
:107A2000EFFF737B0546072B4FF0000605D005F0EE
:107A300059FE35462846BDE8F081866100F10C0705
:107A40000C4E3846B6F8FC8012F00CFA80450CD289
:107A5000B6F8FC6054F80C1F3246384612F00AFAA9
:107A60003146204605F010FFE4E7384612F0FAF9F7
:107A700086B2EFE70020002070B5437B04465BB977
:107A80006FF04001043010F0D3F9430604D52046CE
:107A9000BDE87040FFF7C6BA0022002304F13800A9
:107AA00012F0CBF9054658B940F21A322249234860
:107AB0000EF0CBFA404080F311884FF0030002DF54
:107AC0001F4E2A8AB6F8FC309A4207D800230222B9
:107AD00029462046FFF7D6F968B905E02946204631
:107AE000FFF794FF014638B90023AE692846AB6121
:107AF00005F0F8FDCEB970BD012300222046FFF746
:107B0000C1F90028F0D02A8AB6F8FC309A4202D88F
:107B100000230322DCE729462046FFF777FF0146D2
:107B20000028E1D001231A46E8E731462046BDE8A7
:107B30007040FFF783B900BF46A10200568D0200D6
:107B4000002000200B4B58B11A6862B902693AB99B
:107B500002685AB942684AB982683AB942692AB990
:107B60001860002070476FF0770070476FF01500C5
:107B7000704700BF5C3D002068B10023C360074B25
:107B800000F10C02596819B9C3E9002200207047BE
:107B90000A605A60FAE76FF015007047543D002004
:107BA00010B90248FFF76CBB00207047203000205E
:107BB00010B50C4813F062FD0B490A4813F06BFD39
:107BC0000A49084813F067FD0949064813F063FDA8
:107BD00000F01AFF03F086FF044608B910F0CAFA55
:107BE000204610BDF8270020203D0020303D002019
:107BF000403D002008B502460748036823B9074AFC
:107C000042600860184608BD054845210EF031FA6B
:107C10006FF00B00F7E700BF603D002064840200B6
:107C200072A20200F8B505460F46164600234FF42F
:107C3000803204210020FFF747FC044630B92A4671
:107C4000452106480EF015FA2046F8BD04210C30F7
:107C500005F04EFE057047704680F5E79EA20200D3
:107C6000F7B504460026254D254FBD4242D925498A
:107C7000254840F281120EF0E8F940F281112148C6
:107C80000EF0DCF920466B6801A9984700282CDB30
:107C9000019B2A889A829A84A86803F11002D2E88C
:107CA000EF1FC2E8EC6FBCF1000FF8D19E60A16D30
:107CB00003F10802D9B9C4E915221C60D860019803
:107CC00043681B6803B19847019B1033D3E8EF1F4B
:107CD00041F00101C3E8E21F002AF7D1019843688F
:107CE000DB6913B100F1100198470C35BDE70A605C
:107CF000A265E2E7C6D303B0F0BD00BF887D0200F5
:107D0000AC7D0200CBA20200568D020073B50B8A37
:107D10000646032B0D4604D8452122480EF0A9F94A
:107D20000DE0042105F10C0005F0C8FD2A8A438806
:107D30000446934206D045211B480EF09AF90020D4
:107D400002B070BD427812B945211848E6E70278C2
:107D5000012AF4D0132A04D1012BF0D8452114486C
:107D6000DCE7572113480EF084F9617802220120E4
:107D70003568FFF757FF04460028E0D002210C3099
:107D800005F0B6FD00232246037043700521284606
:107D9000009310F0C4F90028D1D0204605F0A2FCD1
:107DA000CDE700BFFCA202001FA3020045A3020012
:107DB0006BA302008CA3020038B50B8A0546032B87
:107DC0000C4608D845210E480EF053F92046BDE870
:107DD000384005F087BC042104F10C0005F06EFD6D
:107DE00042882846114610F0BCF920B957210548B1
:107DF0000EF03FF9EAE7436821465B699847E5E7FB
:107E0000B9A30200DBA3020073B5174B0E46197825
:107E100005460131C9B2012938BF012108221220CB
:107E20001970FFF7FFFE0446D0B108210C3005F0B1
:107E30005FFD338822460380738805214380B38821
:107E40008380F388C38000232846009310F067F9ED
:107E5000054610B1204605F045FC284602B070BD2D
:107E60006FF00B05F9E700BF9E46002023281FD8BE
:107E70001A2804D8431E182B0ED906207047A0F1EB
:107E80001B03082B1ED8DFE803F0051D1B231D195B
:107E9000251D05000320704701230F4A83401A4027
:107EA000C2B90E4A1A40002A14BF012006207047AA
:107EB00000F07F03522B05D100207047012070474E
:107EC0000520704710F0400F0CBF062000207047BF
:107ED0000420704702207047AAAA8A02545545011F
:107EE00007B50438019001A902480AF0D3FB03B09A
:107EF0005DF804FBF026002008B5437B072B08D172
:107F0000042110F02EF9034628B945210B480EF044
:107F1000B0F8002008BD0221943010F050F950B99B
:107F20000749084840F62A320EF08FF840F62A3109
:107F300003480EF083F853F8040CEBE737A4020073
:107F400057A40200568D020010B5044640B90949F5
:107F50000948A6220EF079F8A62106480EF06EF820
:107F6000002114220FF0D7FB2146BDE81040034842
:107F700013F091BB57A40200568D0200DC270020AD
:107F80002DE9F74306460C46D1F81880CB689830A7
:107F9000022110F014F9002847D01B78D22B14D1FD
:107FA00033682146186811F049FB054668B1452140
:107FB0001F480EF05EF8A069FFF7C6FF204605F0E7
:107FC00091FB284603B0BDE8F08304F10C0011F0EA
:107FD00045FFB4F81090C8F80060336807461D6884
:107FE000E3681878FFF742FF052813D8114B2246A3
:107FF00053F8203004212846CDF8008010F08FF887
:1080000005460028DDD06369A4F8109013FA87F7BD
:10801000E760D6E70849094840F257220EF015F804
:1080200040F2572104480EF009F86FF01505C8E733
:1080300086A402008C84020057A40200568D020020
:1080400008B550B917494FF4467217480DF0FDFFB7
:108050004FF4467113480DF0F1FF41B9114940F258
:10806000193211480DF0F1FF40F21931F2E74A6878
:1080700042B90C4940F21A320B480DF0E6FF40F2CB
:108080001A31E7E7D0F89C3043B1064940F21B3281
:1080900005480DF0DAFF40F21B31DBE7BDE8084090
:1080A00010F0F2B957A40200568D020010B5044634
:1080B00000F19403D3E8EF1F41F00401C3E8E21F8D
:1080C000002AF7D11723201FE384E38210F099F9E7
:1080D00004F1BC0003490BF0EDFA2068BDE8104044
:1080E00002F048B9ED4B01002DE9FF414FF00008C7
:1080F0004FF4205305460E46006802A9144617683F
:108100008DF80880ADF80A300FF068FBA0B142F698
:108110000103286803A98DF80C80ADF80E300FF02C
:108120005DFB48B123691BB15A88B24200D25E8020
:10813000012004B0BDE8F081616828680FF04EFBB3
:1081400010B100232361F3E7E368A0681A7832B125
:108150007B8D018A5B1A934201DA0020E9E7042152
:108160000C3005F0C5FB20610680236929465E803E
:10817000074B0194009338460023A26810F0C5F91C
:108180000028EADB2069003818BF0120D1E700BFD2
:10819000694402002DE9F7431768054688460068E0
:1081A000516814467E680FF019FB814600283CD1C7
:1081B00030469522294610F052FF0646207540B100
:1081C000E3681B780BB184F81490002003B0BDE87D
:1081D000F083A06805F0DEFA02210C3005F088FB80
:1081E000134B2061A0F80080009301943346294688
:1081F0003846A26810F089F9002807DA10F1FF0F5D
:1082000032BF0E204042C0B22075DEE72369002B4A
:10821000DBD0A0680FF0B9FF7B8D181AE3681B78DC
:10822000984294BF00200120D0E70120CEE700BF94
:108230009B410200F7B5002304460E460022694622
:1082400029480AF0CFF9054648B12246452127487A
:108250000DF00FFF6FF00B05284603B0F0BD0CF0DA
:10826000A5FA234B29461860302200980FF053FAE4
:10827000009B00221C60009C0023C4E90155C4E956
:108280000A551C4801A901950AF0ACF905460028D9
:10829000E0D10146F82201980FF03DFA0198164B03
:1082A0008360A03013F0EAF9019B9833D3E8EF2FF5
:1082B000C3E8E15F0029F9D1019B1C60A36A019F1B
:1082C0001BB904F10C0013F0D9F9A26A07F1F0030D
:1082D000C7F8F020E26AA36202B9E362019B002BB7
:1082E000B8D004333360B7E7D02600209EA4020044
:1082F000303E0020F02600209C220020F8B5438D5F
:1083000001329A420D4617D80846FFF7AFFD022802
:1083100015D0042813D04FF0FF364FF0FF3700215F
:1083200032463B4608460FF0F7FE044658B92A4647
:1083300045210E480DF09DFE00242046F8BD4FF467
:1083400070260027EBE70A4832463B460AF0F0FC6D
:1083500018B9204605F0C6F9EEE7A061012104F145
:108360000C0005F0C5FA0570E7E700BF9EA2020009
:10837000DC2700202DE9F0470B8A06460C4633B96E
:1083800045212E480DF075FE0020BDE8F087012143
:1083900004F10C0005F092FA56F8043C0746002B55
:1083A000F2D000230178264DA6F1040815F8330019
:1083B0004FEAC30A884205EBC3021AD192F8029031
:1083C000B9F1010F27D1002106F1940010F043F913
:1083D0000028D9D15544228A6B78934220D945216F
:1083E0003B7818480DF045FEB9F1010FCCD10423BC
:1083F00020E001330E2BD9D10846FFF737FD0028C6
:10840000C2D00528C0D00029BED006230022404695
:1084100010F085FAB8E7B9F1050FDBD10121D3E7F8
:108420006B68214640469847B9F1010F0346ABD12E
:108430000028A9D039780029A6D0E7E7C8A402000F
:10844000A4840200E8A40200F0B51E4603680D46AD
:108450000039044618BF012187B01868174610F08C
:1084600072FE48B9052104F1980010F0F4F80028D4
:1084700048D0002007B0F0BD002E45D018220021C2
:1084800068460FF048F967BB236831461B683046E1
:1084900000930023ADF812300C9B1C4A0393BDF8E7
:1084A00034308DF80850ADF8103001238DF81430B9
:1084B0006B460FF0BBFE9DF81430E3B1002FD8D00F
:1084C000019B9869FFF740FD019805F00BF99DF8B5
:1084D0001430002DCDD032462946204610F01FFA28
:1084E000C7E7002239462046FFF708FF0190002821
:1084F000CAD10E20BEE701990029BAD020460FF05C
:10850000DDFFB6E71220B5E70120B3E7CB4102005B
:108510002DE9F0410E8A0446043EF6B2022E0846CA
:108520008CB001D0102E6AD104210C3005F0C6F9B0
:108530000DF1080805884788011D324640460FF0B6
:108540007BF900285DD0002D3AD00026002F36D0D0
:10855000BD4235D84FF42053404601A98DF8046040
:10856000ADF806300FF03AF970BB666814220021AE
:1085700007A80FF0D0F801221121304610F012FAAE
:10858000099000283DD001210C30CDE9074805F0C5
:10859000AFF900230A90394603701B4A0B93284613
:1085A00007AB0FF043FE0A9B1B781BBB099B986926
:1085B000FFF7CAFC099805F095F80A2301E03D464B
:1085C00001232A4610210EE042F60103404607A986
:1085D0008DF81C60ADF81E300FF000F90028C4D0F3
:1085E00010232A461946204610F099F900200CB0B5
:1085F000BDE8F081204609990FF060FFF6E70420FE
:10860000F5E70E20F3E700BFE94001002DE9F04354
:10861000466804460D4685B00121304610F093FDB2
:1086200050B9052104F1980010F015F800283BD14D
:10863000122005B0BDE8F0831022002168460FF03B
:108640006AF800222121304610F0ACF9029068B39C
:108650004FF00108DFF85890009405F10C072B8AC1
:10866000012B04D8204602990FF028FF1CE0384661
:1086700011F0ECFB6B464A46014606468DF80C802D
:108680000FF0D4FD9DF80C30002BE8D0029B9869C8
:10869000FFF75AFC029805F025F8324620212046C3
:1086A0009DF80C3010F03BF90020C2E70E20C0E727
:1086B000BF4602002DE9F043466804460D4685B0EA
:1086C0000121304610F03FFD50B9052104F198001A
:1086D0000FF0C1FF00283BD1122005B0BDE8F083A8
:1086E0001022002168460FF016F800220F213046B4
:1086F00010F058F9029068B34FF00108DFF8589075
:10870000009405F10C072B8A012B04D8204602990E
:108710000FF0D4FE1CE0384611F098FB6B464A4639
:10872000014606468DF80C800FF080FD9DF80C3058
:10873000002BE8D0029B9869FFF706FC029804F032
:10874000D1FF32460E2120469DF80C3010F0E7F89C
:108750000020C2E70E20C0E7794602002DE9FF4164
:10876000D0F8048004460E464046012117461D46B7
:1087700010F0E9FC48B9052104F198000FF06BFFF7
:1087800078BB122004B0BDE8F0818DB31022002127
:1087900068460EF0C0FF00223946404610F002F94C
:1087A000029038B3BDF828302946ADF804300123D3
:1087B00028468DF80C30104A6B4600940FF036FDB9
:1087C0009DF80C307BB1029B9869FFF7BDFB0298C6
:1087D00004F088FF2A46314620469DF80C3010F000
:1087E0009EF80020CEE7204602990FF067FEF8E7DA
:1087F0000120C7E70E20C5E7794602002DE9F041C8
:108800000D8A0446043DEDB2022D08468CB001D01D
:10881000102D50D104210C3005F050F80DF1040852
:1088200006884788011D2A4640460FF005F888B1A2
:108830009EB18FB1B74210D31822656800210DEBAD
:1088400002000EF068FF01220921284610F0AAF864
:10885000089060B90E2007E03E4601233246082109
:10886000204610F05CF800200CB0BDE8F08101213A
:108870000C30CDE9064805F03BF800230990037061
:108880000A2339468DF82C30304606AB0B4A0FF0E0
:10889000CDFC9DF82C304BB1089B9869FFF754FB39
:1088A000089804F01FFF9DF82C30D7E72046089960
:1088B0000FF004FED7E70420D6E700BF9541010082
:1088C0002DE9F0470F460446062186B007F10C005B
:1088D00004F0F4FF0588B0F802808288D7F80C9085
:1088E000C5B10023B8F1000F13D0454512D88DF85B
:1088F00000308DF804304FF42053684601A9ADF8DC
:108900000220ADF806300EF069FF064660B10A237A
:1089100001E0454601232A46062120460FF0FFFFCD
:10892000002006B0BDE8F087D4F804A00146142268
:1089300001A83F7C0EF0EFFE32460721504610F0B2
:1089400031F80290F8B10A2341468DF815302846D7
:1089500001AB0E4ACDE9036901948DF814700FF054
:1089600065FC9DF815304BB1029B9869FFF7ECFA56
:10897000029804F0B7FE9DF81530CCE72046029926
:108980000FF09CFDCCE70E20CBE700BF4342020076
:10899000F0B5CB6804461D885E8885B095B186B178
:1089A000B5420FD847681022002168460EF0B3FE8A
:1089B0000022052138460FF0F5FF019058B90E202E
:1089C00007E0354601232A46042120460FF0A7FF81
:1089D000002005B0F0BD6B4631462846094A009498
:1089E0000FF024FC029B43B9019B9869FFF7ACFA96
:1089F000019804F077FE0A23E5E7204601990FF07D
:108A00005DFDE5E76B43020038B50B4C0B4D20468E
:108A100012F034FE2946204612F03DFE204605F1B4
:108A2000140112F038FE204605F1280112F033FE41
:108A3000BDE8384000F008BEDC270020F43D0020EF
:108A4000002337B505460C4601930BF0AFFE0B4BE8
:108A500001A91B68834204BF00252C462A462346F1
:108A6000074809F0BFFD014630B91C2201980EF0FD
:108A700052FE019803B030BD0020FBE7303E0020DD
:108A80001027002007B5836801904BB19869FFF764
:108A90005BFA019B986804F025FE0022019B9A6016
:108AA000034801A909F0F6FD03B05DF804FB00BF1F
:108AB000102700202DE9F3470446C0300E46174624
:108AC0001D460AF0E7FED4F89C0030B920680FF08C
:108AD0005EFE002002B0BDE8F087114B4FF00008A9
:108AE000984202D1C4F89C80F0E7D0F80490C0F816
:108AF0000480D4F89C00D0F818A0FFF7C3FF2068CA
:108B0000C4F89C800FF043FEB9F1000FE1D020685B
:108B1000CDF800A03B46324629460068C847D8E752
:108B2000343E00202DE9FF4150F8046C0446002E2D
:108B300056D000F1EC0106F128000FF071FD271F5F
:108B400004F19C0800220023404611F076F9054606
:108B500028BBD4F898302BB1024601460E23384684
:108B6000FFF7A8FF002344F8043CB36A002B37D179
:108B700003960398002200230C3011F05EF905469D
:108B8000A0B903984568C5B9056003A9164809F05E
:108B900081FD206804B0BDE8F04101F085BCA86902
:108BA000FFF7D2F9284604F09DFDCBE7A869FFF74F
:108BB000CBF9284604F096FDDBE782682B689542E6
:108BC000436008BF83606E6836B1AB690E210093C5
:108BD000002300681A46B0472846FFF753FFD0E746
:108BE00004B0BDE8F08100BFD026002010B50446D7
:108BF000452104480DF03DFAA4F1BC00BDE8104049
:108C0000FFF790BF0CA50200F8B50C4650B92849F3
:108C100040F6A46227480DF018FA40F6A4612448F3
:108C20000DF00CFA41B9224940F6A56221480DF039
:108C30000CFA40F6A561F2E7FFF75EF9054640B988
:108C4000A069FFF781F9204604F04CFD6FF07F002A
:108C5000F8BD00F10C062146304604F023FDAD6A54
:108C60004DB155F8F04904B1F03C314628460FF0BB
:108C700033FC034680B90020EAE7032104F19800A1
:108C80000FF09DFA074605F198000FF098FA874219
:108C90006FF0010307D11446002CECD0D4F8F0207B
:108CA00022B90233E9D025461446DEE7F03AF8E768
:108CB00057A40200568D020010B50C4650B9144955
:108CC00040F6BA6213480DF0C0F940F6BA61104898
:108CD0000DF0B4F941B90E4940F6BB620D480DF0F4
:108CE000B4F940F6BB61F2E7FFF706F960B1002383
:108CF000236083682BB9C0E901440FF048FD0020D0
:108D000010BD1C608460F8E76FF07F00F8E700BFDB
:108D100057A40200568D020010B5184614460749A4
:108D20001022A047041E06DA2246452104480DF011
:108D3000A0F9204610BD0024FBE700BF3031002021
:108D400024A50200102208B506490748FAF780F862
:108D5000024628B1BDE80840452104480DF089B914
:108D600008BD00BF203100204AA5020052A5020024
:108D700070B50646134D40B12A4615F8011C6C1E0D
:108D80000FF0EEF898B120460CE028460E490FF09F
:108D90007BFF40B90C4905F110000FF075FF20B1C1
:108DA00005F10F0070BD681EFCE70020FAE73046B1
:108DB000217C04F111020FF0D3F80028F5D004F162
:108DC0001000EFE7693E00203599020070B50E4CA7
:108DD000054623780E4683420CD0237BAB4210D14C
:108DE00031460A480FF050FF58B101230C2202FB14
:108DF000034007E0601C0FF047FF0028EDD0002380
:108E0000F4E7002070BD00BF1E4600202B46002066
:108E100010B54A1C0C4638B109780FF0A1F808B11A
:108E2000204610BD0020FCE7104602490FF02CFF41
:108E3000F5E700BF3599020070B50E4C0646237861
:108E40000D4683420BD0237CB34210D128460A49F9
:108E50000FF01AFF58B1012304EB031008E0284675
:108E6000611C0FF011FF0028EDD00023F4E7002073
:108E700070BD00BF683E0020793E002070B5204BD9
:108E8000144682689A420FD1A568C66875B92279DE
:108E9000216830460FF000FF044628B1194901301F
:108EA0000FF015FF25702581012070BDE0680028B6
:108EB000FBD02B888B420AD0F6D2E068A368013839
:108EC0000433E060003818BF0120A360EDE73046AE
:108ED000227921680FF0E0FE054668B9024609498B
:108EE00030460FF0D9FE05460028E6D02168013053
:108EF0000FF0EDFE23792B70A3685B882B81DCE7F4
:108F0000A55401003599020070B5054615F8012BEE
:108F100004468CB0CAB102AE042130460CF045FDC7
:108F200000962B4624210A4A03A8FBF71DFD0422C4
:108F300004F1080103A8F9F78BFF024618B1452197
:108F400004480DF096F80CB070BD0092E9E700BF40
:108F5000EDA702007DA502002DE9F04180460F46F5
:108F600016461D46FFF732FF044678B91549FFF74C
:108F70002DFF044628B9BDE8F041452112480DF007
:108F800078B8394600F8018B0FF0A1FE2289638979
:108F90006AB973B926816581214611F8010B0EF07B
:108FA0004DFD40B12046BDE8F041FFF7ADBF964210
:108FB00003D3AB42EFD3BDE8F081AB422681EBD2C5
:108FC000E9E700BF359902009EA5020010B508210F
:108FD00009480FF071FE002200230848FBF760FDEE
:108FE000041E06DA2246452105480DF042F82046C7
:108FF00010BD0024FBE700BFE83100204031002015
:10900000C2A502002DE9FF410E46174698460446C8
:1090100048B9452128480DF02CF86FF01505284671
:1090200004B0BDE8F08102A90EF0B4FB054628B1FA
:109030002246452121480DF01CF8EEE7204601A903
:109040000DF039FD019840B10A2229460EF06DFA63
:10905000024610B145211A48EDE7002002A9FFF7AA
:10906000B5FE044608BB002ED9D01649FFF7AEFE68
:10907000044630B9452114480CF0FBFF6FF00B0596
:10908000CDE7002302A900F8013B0FF020FE04F118
:10909000080104224046B847041EC0DA2246452192
:1090A0000A480CF0E6FF2546B9E7002EEFD10C2266
:1090B00031460EF030FBB2E775990200FBA50200C5
:1090C0001CA60200359902003CA6020024A502005D
:1090D000012210B5134BD3E8EF1F002903D1C3E8D9
:1090E000E02F0028F7D11CD100200F490F4A0B8830
:1090F0000F4CA24212D900B10B800E490E484FF41A
:10910000A1620CF0A2FF4FF4A1610A480CF096FF97
:109110005068083203449BB20120EAE7F8D300B15B
:109120000B8010BD883E002036460020E47D020002
:10913000FC7D020063A60200568D020070B5044655
:10914000FEF7A4F90E4D55F820309C4217D0207A36
:1091500004F190010EF072FC88B12046FEF796F9FA
:1091600006462046FEF78CF845F826004FF40042EC
:1091700005F108000023BDE870400AF085BB70BD12
:10918000E830002010B50446094901300FF09FFD7A
:1091900004F10800012200210EF0BDFA00230C3476
:1091A000D4E8EF2FC4E8E13F0029F9D110BD00BF9A
:1091B000359902002DE9FF41884616461F460446B0
:1091C00048B9452127480CF054FF6FF01505284693
:1091D00004B0BDE8F08102A90EF0DCFA054628B122
:1091E0002246452120480CF044FFEEE7204601A925
:1091F0000DF061FC019840B10A2229460EF095F964
:10920000024610B145211948EDE7002002A9FFF7F9
:1092100013FE044680B9FFF7ABFD044630B9452183
:1092200013480CF026FF6FF00B05D0E7002302A9CE
:1092300000F8013B0FF04BFDB8F1000F0DD004F129
:10924000080101223846B047041EC0DA22464521F3
:1092500008480CF00EFF2546B9E72046FFF792FFBD
:10926000B5E700BF75990200FBA502001CA602002D
:1092700093A6020024A5020008B513468168074A98
:10928000914209D11A791968C0680FF005FD18B12B
:109290000A2200210EF03FFA012008BDA55401006A
:1092A00038B514460B4B82680D469A420FD122798D
:1092B0002168C0680FF0F0FC48B1D4F8C83004EB66
:1092C00083021581018901335181C4F8C83001201E
:1092D00038BD00BFA55401004FF4A472002301481B
:1092E0000AF0D2BAB831002008B56FF00201064882
:1092F0000FF034FD04480FF0DCFCC30701D5FFF785
:10930000EBFF002008BD00BFE8310020F8B56FF08A
:10931000040117480FF022FD4FF4A47200231548F2
:10932000FBF7BEFB0026144C144F394620460FF0C5
:10933000ABFCC0B9E379DB0715D52146FEF718FA77
:10934000054620B10FF0FFFB2846FDF7BDFF04F1F5
:109350000B056FF0020128460FF000FD6FF00101D0
:1093600028460FF0FBFC103406B1F8BD0126DCE7FF
:10937000E831002040310020693E0020359902008C
:1093800070B58CB0FFF722FD0446E8B1054615F82C
:10939000012BE2B102AE042130460CF006FB009630
:1093A0000C4A2B46242103A8FBF7DEFA03A80DF094
:1093B0005AFB024618B1452107480CF05AFE0C2210
:1093C000002120460EF0A7F900200CB070BD0092DD
:1093D000E6E700BFEDA70200BAA6020070B500F1F3
:1093E000900604463146007A0EF028FB05463146C9
:1093F000207A4DB1FFF7C4FF024670B1BDE870405E
:10940000452106480CF035BEFFF7E0FC28B129469F
:10941000BDE870400C220EF07EB970BDDCA60200E3
:1094200038B505460C460F4801210FF045FC10F0F9
:10943000010F0D4B0AD11D835C830A480FF039FCE4
:10944000830709D4BDE83840FFF746BF198B5A8B14
:10945000A94202D89442EFD838BD94421D83ECD97A
:10946000EAE700BFE83100209831002013B510462C
:109470004FF42812BDF81010094C0829CDE900421C
:109480000BD8C1F108049C42A8BF1C46694422467F
:109490000EF036F9204602B010BD6FF00604F9E771
:1094A000180028002DE9F0471F46BDF82030064679
:1094B0008846D1F80C90002B43D17B1E012B43D85A
:1094C000012F4946157818BF1588FFF7A1FC0446FF
:1094D00078B915B93846BDE8F0874946FFF798FCDA
:1094E0000446A0B306F1900101300FF0F0FB337A8F
:1094F0002370D9F81030C3B9B4F808A02581B9F8A1
:109500000A30AB4203D0494640460FF047FBAA451C
:1095100002D03046FFF712FE002DDBD10D49601C52
:109520000FF0D5FB25702581D4E72A464146304609
:1095300098470028CFDB01380128DDD96FF00D00F6
:10954000C9E76FF00600C6E76FF00C00C3E76FF0E5
:109550001000C0E7359902002DE9F041234B154674
:10956000826807469A4202D1C468638933BB0120EE
:10957000BDE8F081FDF7A8FE0021E3686181002BC2
:10958000F5D038469847F2E705F190084146287A29
:109590000EF054FA68B9164B9C4202D12846FFF7E8
:1095A0001DFF304613490FF092FB002323702381E7
:1095B000E2E7414630460FF08AFBDDE72389002BC6
:1095C000DAD0264616F8011B284632460EF0C8FCB3
:1095D0000028D9D131462078FEF7CAF80028CBD030
:1095E000437B072BC6D1FDF76FFEC0E7A5540100F2
:1095F000DC2200203599020010B56FF0020104460C
:109600000F480FF0ABFB0E480FF053FBC20704D519
:10961000002200230B480AF037F920460FF091FA98
:1096200060B12046FFF7A4FB40B1037ADB0705D504
:10963000BDE8104001210C300FF03EBB10BD00BF53
:10964000E8310020B8310020012208B5144BD3E8DE
:10965000EF1F002903D1C3E8E02F0028F7D11DD167
:10966000FFF736FD00220F4B0F491048C3E90022D7
:109670000AF020F800234FF4A4720C48FBF70AFA12
:109680000B490C480AF016F802210B480FF014FBA6
:10969000BDE8084009490A480AF00CB808BD00BFF7
:1096A0008C3E0020983E0020595901004031002096
:1096B000D55F0100B8310020E8310020AF51020031
:1096C000F030002003462DE9F04178B3008A68BBF2
:1096D00001244FF0140C1749DFF85CE0714524D9E0
:1096E0001649174840F25D620CF0AFFC40F25D6134
:1096F00012480CF0A3FCD1E90076BB4204D30CFB6A
:109700000672143A93420ED93444A2B21446083178
:10971000E4E70CFB057843450AD001356219B542F0
:1097200092B2F6D1F2E70025F8E7E4D3BDE8F08184
:109730001046FBE7E47D0200FC7D020063A6020008
:10974000568D02002DE9F04F89B09946BDF848309A
:1097500004460F4690461BB94FF6FF73ADF84830EC
:10976000374B1B88A34226D2BDF84830ADF81E30D7
:10977000344B1D68002D3AD109B0BDE8F08F149B21
:1097800028680493139B2246039312ABCDE90193FF
:109790000BFB06003B46CDF800800FF0EAFA0028EC
:1097A000EAD001366B680AEB0601B34289B2E6D80B
:1097B0000DE00026F6E74FF0010A4FF0140B224DA2
:1097C00007E0D1D269685144A142F2D289B28A46F7
:1097D00008351E4B9D42F4D91D491E4840F22172A6
:1097E0000CF033FC40F2217119480CF027FC4FF0CB
:1097F000140A083D0DF11E0BAE68BEB96B689E429F
:1098000019D22868149B0AFB0600018A0493139B53
:109810002246CDE902B3CDE900893B460FF0A9FA13
:109820000028A9D00136E9E70026E7E756F8083C0A
:109830001B8AA342F8D8AD68002D9DD0083DDBE718
:1098400036460020903E0020E47D0200FC7D0200B0
:1098500063A60200568D0200002330B5C9B004464D
:1098600069461CAA04A8CDE90033CDE902330DF006
:1098700051FB28B9452114480CF0FBFB49B030BD21
:109880004FF6FF710120114A04AB0FF0DBFB1048CB
:1098900004A90DF0D4FB10B945210E48ECE70822CD
:1098A0000B4B03F11001187811F8015D013A03F830
:1098B000015B0870F7D10CB1FFF744FA04210648A8
:1098C0000FF0FAF9DAE700BFF7A60200E34B020057
:1098D0002031002015A70200E8310020F8B51B490F
:1098E0000446A1F1300015461F46BDF818600AF085
:1098F00017F817480FF0DDF9410702D40120FFF7F0
:10990000ABFF2046FFF734FA68B1037ADA070AD5CD
:1099100000F10C0420460FF0CCF9C30703D4022158
:1099200020460FF0C9F9102E0CD8C6F11004BC4225
:10993000A8BF3C4607492246284631440DF0E0FEC8
:109940002046F8BD6FF00604FAE700BF7031002032
:10995000E8310020203100206FF0080108B51648DA
:109960000FF0FCF9020722D513480FF0A2F90346C5
:109970005B07C0F3800001D4FFF76EFF10220F4990
:1099800088180DF096FE48B90D4809F083FFBDE830
:1099900008406FF0010108480FF0E0B94FF6FF7181
:1099A0000120FFF73DFDBDE80840FFF7CBB90120DE
:1099B000BDE80840FFF750BFE8310020203100200B
:1099C000B83100202DE9F74F044650B9694940F2FB
:1099D000C15269480CF039FB40F2C15165480CF0A6
:1099E0002DFB036843B9634940F2C25262480CF050
:1099F0002CFB40F2C251F1E7436843B95D4940F2A4
:109A0000C3525D480CF021FB40F2C351E6E7FFF77B
:109A10005FFB2368002518684FF4C05369468DF832
:109A20000050ADF802300DF0D9FE20B96FF077008C
:109A300003B0BDE8F08F236801A9186841F601035F
:109A40008DF80450ADF806300DF0C8FE0028EDD0BA
:109A50004A4D0AF08FF92B682768B4F80490ABB927
:109A6000474A1688002F5ED1002204F10803A26045
:109A70006A68002A5FD1C5E9003342480FF019F93E
:109A8000002868D10AF0C2F90020D1E76B68002BEA
:109A90006ED053E90232142101FB023333F8046C17
:109AA000002F46D1002EDFD023681F8AB742DBD8B3
:109AB00029680029E1D00022A1F108031868008A72
:109AC000B84241D904F10803002A37D09168A16057
:109AD0000029CDD09360D0E7398A69B9711C89B269
:109AE00039820E4609F1FF3914371FFA89F9B9F1A5
:109AF000000FF1D14646D5E7B142F2D801AB5A4644
:109B00000846CDF804A00FF09DFA019B4BB11E480A
:109B100045213A8A0CF0ADFA0AF078F96FF0150099
:109B200086E73146DDE798464FF0000ADFF85CB083
:109B3000DDE7B046F8E713606B609EE76A68A160F6
:109B40002B60002A99D1F7E79868002895D01A462B
:109B5000A0F10803B2E71421D4E9002301FB032399
:109B6000108A33F8041CFFF75BFCFFF7CFFB89E793
:109B70001B68FFDE63A60200568D0200903E0020A7
:109B8000364600208C3E002033A70200974B02008F
:109B90002DE9F043B9B00C4617462C496A46409867
:109BA00098460CF064FF48B9452129480CF061FA49
:109BB0006FF01505284639B0BDE8F083009E01A975
:109BC00030460CF078FF36B9452122480CF051FAA6
:109BD0006FF015042AE0019870B900230DF108090F
:109BE000494630468DF814300DF0D4FD054678B165
:109BF00032464521184808E00A2200210DF095FC64
:109C000002460028E9D0452114480CF032FADFE77B
:109C1000CDF81090C4B1C022404608A9B847041E30
:109C200006DA224645210E480CF023FA2546C1E704
:109C3000A40808ABCDE906344FF6FF710120094AAC
:109C400004AB0FF0FFF9B5E72346F3E759A702008D
:109C500060A7020075990200FBA502001CA6020085
:109C600024A502007D4E0100002307B50193FFF7F4
:109C700029FD411C89B20846034A01AB0FF0E2F905
:109C8000019803B05DF804FBBF4D02002DE9FF41D0
:109C90000C461746054650B9534940F64D425348C5
:109CA0000CF0D3F940F64D414F480CF0C7F941B9DB
:109CB0004D4940F64E424D480CF0C7F940F64E4132
:109CC000F2E7437B072B10D100238DF80C3042F6CE
:109CD0000303206803A9ADF80E300DF07FFDB0B985
:109CE000E3689B7913F0300F03D1002004B0BDE886
:109CF000F0812046FFF7B8FF044640B93A4940F6E4
:109D00005F423A480CF0A1F940F65F41CCE70023EE
:109D100020688DF80C3042F6021303A9ADF80E301E
:109D20000DF05CFD68B12046FFF79EFF044640B988
:109D30002D4940F665422D480CF087F940F6654103
:109D4000B2E7002642F60218206869468DF80060E6
:109D5000ADF802800DF042FDD8B9002320688DF8DF
:109D60000C3042F6021303A9ADF80E300DF036FDAB
:109D70000028BAD1E4682846224612F8011B0EF0EA
:109D8000EFF80028B1D023891F4214BF0120002022
:109D9000ACE742F60303206801A98DF80460ADF832
:109DA00006300DF01BFD0028D7D04FF4205320685B
:109DB00002A98DF80860ADF80A300DF00FFD0028FB
:109DC000CBD042F60103206803A98DF80C60ADF8F2
:109DD0000E300DF003FD0028BFD02046FFF744FFF2
:109DE00004460028B0D180E763A60200568D020029
:109DF0002DE9F047154689469422696806460FF01A
:109E00002EF98046002848D1022230466968FFF7C3
:109E10003DFF002844D04FF470200021AF8AFEF7A8
:109E20000FFE0237044680B11D211F4B47613A46A1
:109E30004174C0F80C804360856130460EF0B2FD7D
:109E4000074638B92046FEF71DFE6FF00B05284681
:109E5000BDE8F08701234246414607F10C0A0EF0A7
:109E600093FE0221504603F043FD804628F8029BF2
:109E7000A98A504603F03CFDAA8A296940460DF0A4
:109E80003FFC21463046A760FEF716FF0546002836
:109E9000DDD02046FEF7F6FDD9E74FF0FF35D6E7D7
:109EA0006FF01505D3E700BFB14B020030B5054692
:109EB0000C468BB051B9424940F60D3241480CF086
:109EC000C4F840F60D313E480CF0B8F84B6853B971
:109ED0000B6843B93A4940F60E323A480CF0B5F8EF
:109EE00040F60E31EFE738480EF0E3FE420761D549
:109EF00015B16B7B072B60D160680590FFF7E2FB23
:109F00002268ADF818003AB305A902912F49002341
:109F10000191012100914FF6FF710593FFF712FCAB
:109F2000059B1BB96FF001000BB030BD6360059B52
:109F300004A9186800238DF8103042F60303ADF829
:109F400012300DF04BFC70B90598C3689B799B06E5
:109F500005D46FF01500E7E70028E8D1E2E70FF03D
:109F600023F8ADF81800BDF818003DB101230146F3
:109F700022462846A375FFF73BFFD5E76FF07F0326
:109F800007930223ADF8203042F60213ADF81230E9
:109F900005ABA57502930E4B4FF6FF71019301239C
:109FA00004AA00932B4609948DF81050FFF7CAFBC2
:109FB0000798B9E76FF00A00B6E76FF07F00B3E7E4
:109FC00063A60200568D0200CC200020D74B020071
:109FD00069620100F7B500F130050446A0F12007E1
:109FE00028460EF066FE8307C0F340060AD51749DF
:109FF000174840F29A420CF028F840F29A41134870
:10A000000CF01CF854F8083C6FF00101284601934D
:10A010000EF0A4FE0F4B394644F81C3C0E4B304664
:10A0200044F8183C01AB44F8103C042324F8086CB5
:10A0300024F8066C24F80C3CFFF738FF18B902210D
:10A0400028460EF039FE03B0F0BD00BF63A6020043
:10A05000568D02003C850200F95501002DE9F743B9
:10A06000334B17461468826805469A425CD1002338
:10A07000C66806F10109002B56D13389002B53D055
:10A080004A46204631780DF06BFF00284CD04FF443
:10A090009572294620460EF0E2FF98B1032843D07E
:10A0A000052820460CBF4FF003084FF002080DF0C2
:10A0B00055FF804506D93A7901234245DBD287F81E
:10A0C0000480D8E7314628460EF068FD194B9E42C1
:10A0D0002AD1207A04F19001FEF778FE20B302899C
:10A0E000438952EA03011FD02046ADF80420ADF8A1
:10A0F0000630FDF7CBF918230F49104A03FB001374
:10A100005A600F4A00B29A6001AA1A61042200EB59
:10A11000400001EBC0019A822046FFF7C7FE18B14C
:10A12000452108480BF0A5FF012003B0BDE8F083EE
:10A13000A5540100DC220020503E00203C85020096
:10A14000334F020071A7020030B505460C468BB0B4
:10A1500051B9404940F62D223F480BF076FF40F6BA
:10A160002D213C480BF06AFF4B6853B90B6843B98B
:10A17000384940F62E2238480BF067FF40F62E2172
:10A18000EFE736480EF095FD42075DD515B16B7BC4
:10A19000072B5CD160680590FFF794FA2268ADF850
:10A1A00018003AB305A902912D490023019101211C
:10A1B00000914FF6FF710593FFF7C4FA059B1BB999
:10A1C0006FF001000BB030BD6360059B04A91868F7
:10A1D00000238DF8103042F60303ADF812300DF075
:10A1E000FDFA70B90598C3689B79DB0605D46FF05A
:10A1F0001500E7E70028E8D1E2E70EF0D5FEADF85C
:10A200001800BDF818002DB10146224628460EF070
:10A210005AFFD7E76FF07F0342F60212079301233C
:10A22000ADF8122005AA02920E4AADF82030CDE911
:10A2300000324FF6FF712B4604AA09948DF8105096
:10A24000FFF780FA0798BDE76FF00A00BAE76FF0F2
:10A250007F00B7E763A60200568D0200CC200020E5
:10A26000D74B0200696201002DE9F84315463D4BCA
:10A27000826807469A4203D001273846BDE8F88332
:10A28000C668394B9E4210D03289AB89711C9A4204
:10A29000F2D13078FDF76CFA04460028ECD0437B0D
:10A2A000072B26D0FDF710F8E6E74FF000082F4CFB
:10A2B000DFF8BC90494620460EF0E6FC78B907224C
:10A2C000214614F8010CFDF76DFA78B92B69214687
:10A2D0001A6914F8010C53881288FEF73DFE0C34FD
:10A2E000B8F1000FD0D14FF00108E3E7FCF7ECFF25
:10A2F000F5E7736923B13946984708B92046D1E795
:10A300003946942220460EF0AAFE07460028F5D1D1
:10A31000AB89022B14D133899A0705D42046FCF768
:10A32000D3FF0023AB60A7E720462A69A988FFF77F
:10A330005FFD064678B92A69937D01339375EDE791
:10A34000012BEBD13389DB07E8D520462A69A988A0
:10A350000EF0B9FE06462046FCF7B6FF002E8CDB59
:10A36000DFE700BFA5540100DC2200201F460020CB
:10A3700035990200012370B500F190058EB00446B6
:10A3800003902946007A8DF810300DF057FB90B1FC
:10A39000227A1AB302AE042130460BF006FB009677
:10A3A00024210F4A05A82B46FAF7DEFA05AA104623
:10A3B0000C49F8F7ADFD4FF6FF7101200A4A03ABD7
:10A3C0000EF040FE20460DF0C9FD9DF810108842A9
:10A3D00002D220460DF096FD0EB070BD0092DFE770
:10A3E0005CA70200915B01005D600100F8B50546C5
:10A3F0000E461746064B1C684CB154F8043C043C0E
:10A400001BB13A463146284698476468F4E7F8BDE0
:10A41000983E002007B5009001206B464FF6FF7173
:10A42000034A8DF804000EF00DFE03B05DF804FB46
:10A430005D600100002370B50446C0B00D460D916B
:10A440008DF838003F934FF6FF710120134A0DAB92
:10A450000EF0F8FDECB103AE2246042130460BF0BD
:10A46000A4FA00960E4A2B46242104A8FAF77CFA97
:10A470003F9A82B192000FA904A8F8F7E9FC0446BC
:10A4800020B10246452107480BF0F3FD204640B0BD
:10A4900070BD0094E6E71146EEE700BFA15201004F
:10A4A0005CA7020093A70200F0B5044603464FF6EE
:10A4B000FF7101203B4A8DB00EF0C4FD2046FCF731
:10A4C000E5FF394E054656F8200020B1FCF7FCFEAA
:10A4D000002346F82530354804F1900509F0DAF9F3
:10A4E0002946207A0DF0AAFA78B32946207AFFF798
:10A4F000A1FF2046FEF73CFC0646002845D0227A04
:10A50000083672B102AF042138460BF04EFA2B46E2
:10A510002421274A009703A8FAF726FA237A002B6A
:10A5200035D10127002324210093214A2B4603A87B
:10A53000FAF71AFA3A46314603A8F8F789FC0246B8
:10A5400018B145211B480BF094FD2946207A0DF0E7
:10A5500075FA50B1237A4FF6FF718DF81030012053
:10A56000154A03AB03950EF06DFD2046FEF700FC87
:10A570000646A8B12946207A0DF060FA48B930465F
:10A580000DB0BDE8F040FEF7FDBD0746CAE7012764
:10A59000D0E72946701C0DB0BDE8F0400EF097BB27
:10A5A0000DB0F0BD59550100E8300020F03000201A
:10A5B000E7A70200B6A702007952010008B5054BD3
:10A5C000014618460EF00CFE043B002814BF184646
:10A5D000002008BDF4310020084B00F5D8701A683F
:10A5E000074BD0E8EF1F994204D1C0E8EC2FBCF133
:10A5F000000FF6D1D0E8AF0F704700BF5C3D0020E0
:10A60000F031002008B5FFF7E7FF0346C8B1D0E9F5
:10A61000001221B9002A0CBF0320022010E032B141
:10A62000836813B9094B1B7833B9042008E0074944
:10A63000087828B19B6833B9003A18BF012250004E
:10A6400008BD0320FCE70120FAE700BF9F46002079
:10A6500010B50C4B1B787BB101F00F04FFF7D2FF54
:10A66000094B03281B780CBF04F00B0444F00404CE
:10A670002BB144F0010010BD01F00704EEE704F037
:10A68000FE00F8E79F4600206226002010B5062154
:10A690000DF067FD044628B9452104480BF0E9FC9C
:10A6A000204610BDA0F1EC04FAE700BFF8A70200B5
:10A6B00010B5084C0246D4F8EC0020B9064AEC3438
:10A6C00062600C6010BD054845210BF0D2FC6FF0B4
:10A6D0000B00F7E7F03100204086020018A80200C6
:10A6E00038B50546EC2200210DF015F8102105F1D2
:10A6F0002700FCF727FA044648B9052128460EF042
:10A70000C0FDFCF7ADFA034B1860204638BD0824A5
:10A71000FBE700BFA03E002038B50446051D082118
:10A7200028460EF0AEFD084904F15700FCF7A6FAE2
:10A7300040B1082128460EF07AFD044845210BF06F
:10A7400098FC082038BD00BFD556020042A8020080
:10A7500070B50B4604460D2104300EF041FDC8B122
:10A76000DE68D4F8EC30022003F190052A46197A0D
:10A7700001F0F8FA48B92846FAF75EF84521024692
:10A7800007480BF076FC082070BD102231462A30B5
:10A790000CF0B6FF204609210EF073FD0020F3E710
:10A7A00060A8020070B50B4604460D2104300EF07F
:10A7B00017FDC8B1DE68D4F8EC30042003F1900531
:10A7C0002A46197A01F0CEFA48B92846FAF734F841
:10A7D0004521024607480BF04CFC082070BD1022B2
:10A7E00031461A300CF08CFF204607210EF049FD4F
:10A7F0000020F3E760A8020073B5047A0546022C36
:10A8000023D844B190F8DC30D0F8D840DC4004F0D4
:10A81000010444F08004032128460EF042FD064660
:10A82000D0B110210C3003F063F800901248234699
:10A83000006805F1270205F157010EF0EAFF044612
:10A8400078B1304602F04EFF06E0032C07D02246D6
:10A8500045210A480BF00DFC082002B070BD002411
:10A86000D9E70246314628460EF0EEFC281D214667
:10A870000EF0DDFC2046F0E7A03E00207FA802009D
:10A880002DE9F8430446FFF7A7FE261D07460E21D3
:10A8900030460EF0A5FC38B10C2120460EF001FD2B
:10A8A000054658B9082032E0434B2022196804F1CC
:10A8B00057000CF0FEFE0028EED1F3E740210C30EB
:10A8C00003F016F8DFF8F0902022D9F80010804647
:10A8D0000CF016FF2022D9F8001008EB02001144FA
:10A8E0000CF00EFF0022294620460EF0ADFC227A25
:10A8F000052A59D8DFE802F003390D035855042121
:10A9000020460EF0BEFCFFF777FF00283CD0BDE8E4
:10A91000F8832046D4F8EC70FFF75EFE042105466C
:10A9200004F1D800FCF70EF90028BBD1D4F8D830D8
:10A93000224A84F8DC00B3FBF2F102FB1133C4F8C5
:10A94000D83055B12B6843B10B2130460EF099FC3D
:10A9500038462B68D4F8D8109847032120460EF0CB
:10A9600090FC0E210EF08DFC0EE0204603210EF02F
:10A9700088FC0E210EF085FC30460A210EF081FC89
:10A980007B68D4F8EC009847304607210EF079FC3C
:10A990000820FFF713FE60B92046BDE8F843FFF733
:10A9A000BBBE04212046DDE7452105480BF061FBD5
:10A9B00078E70020ABE700BFA03E002040420F0038
:10A9C0007FA8020070B50D460446FFF705FEEE684D
:10A9D00004F157052022314628460CF091FE202232
:10A9E00004F17700B1180CF08BFE2846FCF7C8F88C
:10A9F00040B9164B1D681DBB201D06210EF041FC01
:10AA000028461CE00E21201D0EF03BFCD4F8EC5033
:10AA1000D5F8C03033B9287A05F1900101F0B4F8C7
:10AA2000C5F8C000D5F8C030002BE2D0DA8902F0BA
:10AA30002402002ADDD05B7B9B07DAD4032070BDA3
:10AA40002046BDE87040FFF71BBF00BFA03E0020BE
:10AA50002DE9F3410D460446D0F8EC60FFF7BCFD4C
:10AA6000D5F80C80074698F80330073B092B03D92B
:10AA7000062002B0BDE8F081D6F8C0305BB1251DDC
:10AA80000F2128460EF0ACFB80B92046FFF728FEC8
:10AA900060B1C0B2EDE7307A06F1900101F074F8D0
:10AAA000C6F8C0000028EAD10820E2E70123062208
:10AAB0004146637204F10A000CF022FE0223237463
:10AAC00098F802102046FFF7C3FDE0742046FFF718
:10AAD00099FDA34B60741B78A3741023237598F819
:10AAE000043003F00303637598F8053003F00103A5
:10AAF000A375E37C1B070DD598F80230180709D51C
:10AB0000052128460EF0BDFB637D03F0020363754B
:10AB10000023A375E37C990607D598F802309A06BE
:10AB200003D5142128460EF0ACFBA37D84F8E83051
:10AB3000637D84F8E930E37CDB0707D598F80230C1
:10AB4000D80703D50D2128460EF09BFB032128468C
:10AB50000EF097FB052198F800800EF041FB40BBFA
:10AB6000B8F1040F45D8E37AA27C1340D9073ED44C
:10AB7000217BE37C194311F0040111D02046FFF73B
:10AB800041FD784B08EB8808984418F80010042918
:10AB900006D1D4F8EC30DB78002B14BF0121022160
:10ABA00021722046D6F8C0100EF020FB18BB0320FF
:10ABB0005FE7237BE07C03EA0002120706D5E27A16
:10ABC00094F812C042EA0C02D207E9D4B8F1040F9B
:10ABD0000FD843EA000111F00401E1D02046FFF74D
:10ABE00011FD614B08EB88084344195CD8E7062146
:10ABF000D6E70021D4E7D4F8EC309B7A032B37D08A
:10AC000025D8013B012B3FF64FAF052128460EF01A
:10AC1000E7FA002840F0B0802046FFF7DDFC074649
:10AC20002046D4F8EC80FFF7D7FC08F190010646E7
:10AC300098F8080001F060F8227AE8B1437BDB075E
:10AC40001AD5CAB9452149480BF013FA2CE7042B51
:10AC50007FF42AAF237D627B934228BF1346102BDB
:10AC60007FF406AF052128460EF0BAFA00289ED0E0
:10AC7000237A002BC9D19AE7062A5ED8DFE802F0D2
:10AC800018552D5D5D5D0400002E5BD0F368002B30
:10AC900058D000230A212846ADF804300EF0F1FA0E
:10ACA000F368D4F8EC0001A99847237A002B4BD124
:10ACB0000F2128460EF094FA002845D1002F43D0EA
:10ACC0007B69002B40D028460A210EF0DAFA7B6916
:10ACD000D4F8EC0098470020CBE604210DEB0100EE
:10ACE000FBF730FF00287FF4DFAE019B204AB3FB67
:10ACF000F2F102FB113301934EB133683BB10B21EA
:10AD000028460EF0BEFA4046336801999847019BE9
:10AD1000C3F3072284F847301B0C84F849301B0A20
:10AD200084F8482084F84A30BFE728460A210EF00C
:10AD3000A8FA404673689847B7E745210D480BF0DD
:10AD400098F9B1E6022094E6032120460EF099FA24
:10AD50000E210EF096FA02B0BDE8F0410EF0C0BA36
:10AD6000A0460020EEAA0200D5AA0200A0A8020078
:10AD700040420F007FA80200237A73B90F212846B2
:10AD80000EF02EFA48B947B17B6933B128460A2143
:10AD90000EF077FA30467B699CE70C212046D8E715
:10ADA0002DE9F043044691B0102200210CA80CF0CC
:10ADB000B2FC227A052A2CD8DFE802F00903030945
:10ADC0002B25042204F1D8010CA80CF099FCD4F82E
:10ADD000EC3004F1470204F1C705CDE9015204F15A
:10ADE000370603F19E0204F12708009231464246DD
:10ADF000973304F1970001F0DDF890B14521384810
:10AE00000BF037F909E0D4F8E4100029DFD0102264
:10AE1000DAE7452133480BF02CF9082011B0BDE8E2
:10AE2000F083D4F8EC3008AF03F197029E3301931E
:10AE300004F11103029200933246414628460397DB
:10AE40000CAB0EF00BFD10B145212748D8E7237A53
:10AE5000052B06D1D4F8E01010220CA8C9B10CF0D3
:10AE60004FFCD4F8EC300DF1100903F19E0297333A
:10AE7000019304F10A0302920093424631462846A8
:10AE8000CDF80C900CAB0EF0E9FC28B14521174829
:10AE9000B6E70CF040FCE4E71022494604F1B700A5
:10AEA0000CF007FC0546C8B90D2120460EF0F9F953
:10AEB00006460028B1D010210C3002F019FD1022F6
:10AEC00039460CF01DFC2A46314620460EF0BCF9EE
:10AED000201D01210EF0D5F928469FE70B209DE7A4
:10AEE000D2A802007FA80200ECA8020014A9020068
:10AEF00038B504460849A0F1EC05943008F0DAFBB7
:10AF000028460EF05CFA054BC434D4E8EF2FC4E8B1
:10AF1000E13F0029F9D138BD4D790100F031002021
:10AF200070B50446CE68051D0B2128460EF07FF94A
:10AF30003146102204F117000CF0E2FB05212846EF
:10AF40000EF04EF920B92046BDE870400EF0ACBAC4
:10AF5000227A012A09D0022A13D1204604210EF0B8
:10AF600090F9BDE87040FFF747BC0A2128460EF073
:10AF700037F90028F1D0284600210EF082F9002090
:10AF800070BD034845210BF074F80820F8E700BFB6
:10AF90007FA802002DE9F041044688B00D46FFF776
:10AFA0001BFB04F13707E968064610223846251DC9
:10AFB0000CF0A6FB052128460EF012F9002841D11D
:10AFC000D4F8EC3004F1470803F19E0204AE973345
:10AFD0000192009339464046029604F1100304F1B1
:10AFE00009020EF007FAE0B91022314604F1170009
:10AFF0000CF05FFB002867D10822394630460CF080
:10B000007FFB082204F1270106A80CF079FB3246E9
:10B01000314640460CF0C5FE38B1452156480BF08C
:10B0200028F8082008B0BDE8F081314610224046DB
:10B030000CF066FB012128460EF023F920460EF0A5
:10B0400068F9EFE7227A052A00F28E80DFE802F045
:10B05000191F1F038C6204AB484900933A460968E4
:10B0600004F1270304F1570001F00CF80028D8D1AF
:10B070000A2128460EF005F9B3680499D4F8EC00CB
:10B0800098470D2120460EF0FCF81021D3E794F8E4
:10B09000DC20D4F8D8303949D34004AE03F00103A2
:10B0A00000963A46096843F0800304F157000EF019
:10B0B000B0FB10B145213248B1E71022314604F10E
:10B0C00017000CF0F6FA08B10420ABE70321204684
:10B0D0000EF0D7F80EF01DF90028A3D194F8DC305B
:10B0E0000133DBB2142B84F8DC3009D10D2120466A
:10B0F0000EF0C7F8102128460EF0C3F8002091E7A3
:10B10000102104F12700FBF71DFD003818BF0120B6
:10B11000C00087E7102104F12700FBF713FD00288A
:10B120007FF47FAF2EB3F3681BB3164BE27A1B8814
:10B13000D207ADF81030A37C03F0010312D4002B2A
:10B1400014BF012303238DF8113000232846C4E9DE
:10B1500038330C210EF095F8F368D4F8EC0004A90C
:10B160009847CBE75B00EEE7452107480AF081FFEF
:10B1700057E7022056E700BF3DA90200A03E00208D
:10B1800057A902003C8002007FA802002DE9F74386
:10B19000C6780446012E05D06FF01504204603B092
:10B1A000BDE8F083FFF772FA0546002800F0AC8096
:10B1B000071D042138460EF013F8002840F0A78040
:10B1C000032138460EF00CF810B16FF00F04E5E7DC
:10B1D000314638460EF004F80028F6D12846FFF72D
:10B1E000FBF9D5F8EC3006469B7A032B42D032D8D7
:10B1F000013B012B48D90B21201D0DF0F1FF002848
:10B20000CAD1D4F8C03083B904F190063246202068
:10B21000217A00F0F3FCC4F8C00030B932460420B3
:10B22000217A00F0EBFCC4F8C000D4F8C030002B49
:10B23000B2D0DA8912F0240FAED0A17A022923D934
:10B24000587BC007A8D503291ED09206A4D51B7B26
:10B25000102BA1D118E0042BCDD12846FFF7D2F94D
:10B26000032804D1002EC6D0F368002BC3D0294B8D
:10B270001B7807E02846FFF7C5F9032804D1002E04
:10B28000B9D0F368002BB6D0D4F8C0303BB1284613
:10B29000FFF726FA804670B16FF068047EE7207AE7
:10B2A00004F1900100F070FCC4F8C0000028EED159
:10B2B0006FF00B0472E70B2128460DF0F2FF0646F3
:10B2C0000028E9D001210C3002F012FB092181464F
:10B2D0002846FFF7BDF9434689F80000324620466C
:10B2E0000621CDF800800CF01AFF044618B1304654
:10B2F00002F0F8F952E738460F210DF0C2FF0121A4
:10B3000028460DF0BEFF49E76FF07F0446E76FF077
:10B31000040443E79F460020F8B50646D0F8EC50F9
:10B32000041D61BB0D2120460DF05AFF074618B1E0
:10B33000D5F8C00000F0E0FD364B1B689BB11C68DF
:10B3400004B10C3C53F80C3C13B1394628469847DD
:10B350004CB12346E4681B681CB10C3C002BF4D1B3
:10B36000F7E7002BF1D130460EF029F86A7AAB7A74
:10B370009A424DD02846BDE8F840FFF707BF013993
:10B38000C9B20E2996BF244B09275F5CD5F8C0309F
:10B3900043B11B7B33BBD5F8C00000F005FD002393
:10B3A000C5F8C030022120460DF01AFF48B9072F1A
:10B3B00094BF1A4B1F213A46284698BFD95DFCF727
:10B3C00085F9032120460DF00BFF0028CBD0114B4F
:10B3D0001B68002BC7D01C6804B10C3C53F8083C18
:10B3E0004BB90BE0022120460DF0FAFE0028D2D125
:10B3F000D8E70C3C23B1394628469847002CB2D0F8
:10B400002346E4685B68002CF3D1002BF3D1AAE754
:10B41000F8BD00BF543D0020C6AA0200B5AA020034
:10B42000F8B50B8A07460D462BB945211E480AF090
:10B4300020FE0020F8BD012105F10C0002F03EFACB
:10B4400004210646A7F1E800A7F1EC040DF0C8FEC0
:10B450000028EED131780E29EBD8144F57F831304F
:10B4600023B9072120460EF0ECF8E2E720460DF064
:10B4700094FF337818B9052BDBD00821F2E707EBEE
:10B48000C3012A8A0979914205D0452108480AF06A
:10B49000F0FD0A21E6E72946204657F83330984761
:10B4A00001460028C5D0DDE775A9020068860200C4
:10B4B000E8A402000A4B10B5186080B1094807F0F3
:10B4C0008FFC094B1C1FD3E8AF3F5B0607D5204616
:10B4D000FFF7D6F9014610B120460EF0B2F810BDC4
:10B4E000A03E0020C4270020F43100202DE9F041C7
:10B4F00090F8E930CF6823F0020380F8E930D0F803
:10B50000EC503B78044605F19008BBB1BB7903F0E1
:10B51000C003C02B12D03846F9F78EF945210246F8
:10B520004C480AF0A6FD4046F9F786F94521024647
:10B5300049480AF09EFD0A20BDE8F08107223946FD
:10B5400040460CF0B6F868B13946287A00F0D4FBD2
:10B55000064638B1014620460DF048FEB8B13046E7
:10B5600000F022FC0D21201D0DF03AFE00285ED0D7
:10B5700042460220297A00F0F5FB064648B94046CB
:10B58000F9F75AF94521024634480AF072FD0820BD
:10B59000D2E7EB78A3BB05F19E010B78012B20D1FC
:10B5A0008B7903F0C003402B1BD10622013106F139
:10B5B0003A000CF0A5F895F8903093B195F89630D4
:10B5C00003F0C003C02B0CD007223946701C0CF0CE
:10B5D00097F80722394640460CF092F82846FCF7C7
:10B5E00037F894F8E9309A070DD51D4940F66362A3
:10B5F0001C480AF02AFD40F6636119480AF01EFD56
:10B6000005F19701C9E73046FAF7CCFC00BB30469C
:10B61000FAF7C8FC40B1124940F67F6211480AF0BF
:10B6200014FD40F67F61E8E73046FAF7CBFC94F86A
:10B63000E9305B0703D50A2120460DF022FEB4F85D
:10B64000E81009B1002077E72046FFF765FEF9E72B
:10B65000032071E795A90200AEA9020060A80200CC
:10B66000BBA90200568D0200F8B504460B46D0F87F
:10B67000EC500D2104300DF0B3FDF0B105F1900751
:10B68000297A3A460420DE6800F06CFB054648B98A
:10B690003846F9F7D1F84521024614480AF0E9FC8A
:10B6A0000820F8BD0222314618300CF029F8082293
:10B6B000B11C05F110000CF023F894F8E93023F0E8
:10B6C000010284F8E9209A0708D5082120460DF0E8
:10B6D000D8FDB4F8E81029B10020E2E75B07F8D5FF
:10B6E0000A21F3E72046FFF717FEF5E760A80200FE
:10B6F0002DE9F0410E460446D0F8EC80FEF76CFFD1
:10B70000F6684521054632780E48271D0AF0B1FC3F
:10B710000A2138460DF041FE38B16DB92046317826
:10B72000FFF7FAFD0020BDE8F0810B2138460DF04F
:10B7300034FE0028F1D1F1E72B69002BEED0404612
:10B740009847EBE7EAA902002DE9F0470546A0F18A
:10B75000E80604460F4688B00121304655F8EC89CA
:10B760000DF01BFE002800F08780E7B10321304672
:10B770000DF036FD00287FD03846F9F799FF0138E3
:10B78000C0B208288CBF00246A4B4FF0020198BF5A
:10B790001C5C30460DF075FD2146284608B0BDE81A
:10B7A000F047FFF7B9BD98F80B30002B64D00321A8
:10B7B00030460DF015FD28B9284608B0BDE8F04721
:10B7C0000DF0FDBD052130460DF00AFDB8B114F8AD
:10B7D000043C1B0707D514F8033C1F0703D51121B0
:10B7E00030460DF04EFD14F8043C23F0080304F835
:10B7F000043C14F8033C23F0080304F8033C14F859
:10B80000033CD80717D5062128460DF03AFD022142
:10B8100030460DF036FD2368D3F8C0209AB903F105
:10B820009000F9F709F845210246434808B0BDE801
:10B83000F0470AF01EBC990701D50821E4E75A0732
:10B84000E5D50A21E0E705210DF0CAFC80B914F81E
:10B85000043CDB070CD523681A2101A8D3F8C0707B
:10B86000FBF770F9814650B1452134480AF001FCDC
:10B8700034F8041C002990D008B0BDE8F0870621F8
:10B8800028460DF00EFD804610B945212C48EDE705
:10B8900010210C3002F02CF83A7B01A982460BF003
:10B8A0002FFF387B0F2805D8C0F1100249465044BD
:10B8B0000BF031FF4146002228460DF0C5FC072160
:10B8C00028460DF0EEFC804610B945211D48CDE715
:10B8D0000A210C3002F00CF88146082205A902303A
:10B8E0000BF00EFF022207A948460BF009FF414664
:10B8F0002846154A0DF0A8FC0D2130460DF070FCCD
:10B900000028B5D03846012100F016FA01A910220E
:10B9100007F14A000BF0F4FE05A9082207F14000E8
:10B920000BF0EEFE022207A907F148000BF0E8FE3B
:10B930009EE700BFBDAA020011AA02002BAA0200C6
:10B940004BAA020077AA02007579010010B50446DF
:10B95000452107480AF08DFBA4F5C0700821FFF7C8
:10B96000DBFCA4F5BE700421BDE810400DF089BCDD
:10B97000A4AA020008B5FAB98378012B1CD10621CC
:10B980000CF0E6FB50B90D490D4840F265220AF073
:10B990005CFB40F2652109480AF050FB10F8043CBA
:10B9A00023F0010300F8043C30F8041C21B9BDE881
:10B9B0000840EC38FFF7B0BC08BD00BFBBA90200CF
:10B9C000568D0200F8B50446FEF760FE05460028D5
:10B9D00000F08480061D032130460DF001FC002894
:10B9E0007CD0D4F8C00008B100F0DEF904F1900773
:10B9F0003946207A00F0C8F8C4F8C00068B9384663
:10BA0000F8F71AFF4521024635480AF032FB28466E
:10BA1000BDE8F84008210DF014BE0E2130460DF0AF
:10BA2000DFFB28B1D4F8C020537B43F002035373EB
:10BA30002A7AD4F8C010032A4B7B3CD8002A41D084
:10BA4000D4F8C020537B43F0010353732B7D697BF3
:10BA5000D4F8C0208B4228BF0B4630461373052113
:10BA60000DF0BEFBD4F8C0305A7BA0B342F01002F8
:10BA70000D2130465A730DF0B3FB78B3D4F8C000F3
:10BA8000202100F059F9D4F8C00005F14701102237
:10BA90001A300BF035FED4F8C00008220021103017
:10BAA0000BF039FED4F8C0000222BDE8F8400021B6
:10BAB00018300BF030BE053A012A03D843F02003BA
:10BAC0004B73BDE723F020034B73D4F8C020537BA6
:10BAD00023F00103B9E722F010025A73F8BD00BF4A
:10BAE00060A8020008B5074B074893F89A3003F0A6
:10BAF00006039A1F53425341044A1370FBF74CF854
:10BB0000002008BD002000200C2300209F460020BC
:10BB100008B550B9074908484FF4E4720AF095FA9D
:10BB20004FF4E47103480AF089FABDE80840FAF7D7
:10BB300049BA00BF0EAB0200568D020070B50F4C23
:10BB4000054614F8013B0E46834207D007220C49F4
:10BB50000C480BF0AEFD48B1002070BD0722204616
:10BB60000BF0A7FD0028F1D10448F6E70722314683
:10BB700004F8015C03480BF0C3FDF5E7A43E002088
:10BB800035990200A53E002008B541B9064907488D
:10BB900059220AF05AFA592103480AF04FFABDE82F
:10BBA0000840FFF7CBBF00BF0EAB0200568D02006E
:10BBB0000B4610B5114604465BB908490848B32244
:10BBC0000AF043FAB32105480AF038FABDE81040FC
:10BBD00018470448C2892242F8D110BD0EAB0200BA
:10BBE000568D0200A43E002008B500220220024922
:10BBF000FFF7DEFF002008BD117B0100F8B5054608
:10BC00000E461446A2B90F490F48C0220AF01DFA89
:10BC1000C0210C480AF012FA8AB18E420FD10722D5
:10BC200021460A480BF045FD012318B9084807E0F2
:10BC30000023074FFA8939782A40002BECD00020E6
:10BC4000F8BD00BF0EAB0200568D0200A53E0020DD
:10BC5000A43E0020F8B506460C4641B921492248C9
:10BC6000E9220AF0F2F9E9211E480AF0E7F90B7817
:10BC7000012B01D00020F8BD8B7903F0C003402BCD
:10BC8000F8D10023194D05F13A07EA89287802F026
:10BC90000202C3B10023EA89297802F00202002BD4
:10BCA000E8D1002AE6D0B142E4D1671C39461048F9
:10BCB0000BF04AFD01230028EDD0062239460D483D
:10BCC0000BF01EFD0BE0002AE5D0B042E3D10622C6
:10BCD0003946601C0BF0EDFC01230028D5D1034848
:10BCE000C9E700BF0EAB0200568D0200A43E002043
:10BCF000CE3E0020DE3E002010B551B90B490C4865
:10BD00004FF48D720AF0A1F94FF48D7107480AF0D3
:10BD100095F9084C2378834204D10722601C0BF06C
:10BD2000C8FC08B1002010BD2046FCE70EAB0200A5
:10BD3000568D0200A43E002008B550B907490848B6
:10BD40004FF495720AF081F94FF4957103480AF0A7
:10BD500075F9C3891943C18108BD00BF0EAB02004C
:10BD6000568D0200F8B506460F46154642B90C49F5
:10BD70000C48D2220AF069F9D22109480AF05EF98A
:10BD8000FFF73CFF044640B929463846FFF7FCFE62
:10BD9000044610B13146FFF7CFFF2046F8BD00BF83
:10BDA0000EAB0200568D020070B504468CB050B93F
:10BDB0001649174840F231120AF047F940F23111A2
:10BDC00012480AF03BF9037A5B0701D5FAF79CF9B0
:10BDD000254615F8012BB2B102AE0421304609F018
:10BDE000E4FD00962B4624210A4A03A8F8F7BCFD7F
:10BDF00003A80AF038FE5C22002120460CB0BDE802
:10BE000070400BF088BC0092ECE700BF0EAB020064
:10BE1000568D0200CEAB020070B506461446184699
:10BE200098B046B945212E480AF023F96FF0150560
:10BE3000284618B070BD502204A9A047041E05DA98
:10BE40002246452127480AF014F9EFE7304602A9B7
:10BE50000BF0A0FC054618B1324645212248F2E716
:10BE6000304601A90AF027FE019840B10A2229466E
:10BE70000BF05BFB024610B145211C48E3E75CB9BF
:10BE800021463F2002AAFFF7B9FE0028D0D05C224D
:10BE900021460BF040FCCBE7002002A9FFF74EFE45
:10BEA000064650B902A8F8F7C7FC452102461048DB
:10BEB0000AF0DFF86FF00B05BAE7502C09D05023D9
:10BEC000224645210B480AF0D4F83046FFF76CFFB4
:10BED000ACE7224604A90C300BF012FCA8E700BF27
:10BEE000759902003EAB0200FBA502001CA60200F1
:10BEF00062AB020086AB020070B504468CB050B94C
:10BF00001649174840F255120AF09FF840F25511B1
:10BF100012480AF093F8054615F8012BDAB102AE83
:10BF20000421304609F041FD00962B4624210D4A9C
:10BF300003A8F8F719FD04F10C01502203A8F6F745
:10BF400087FF044620B10246452107480AF091F8D0
:10BF500020460CB070BD0092E7E700BF0EAB0200B8
:10BF6000568D0200CEAB0200A9AB0200884210B58C
:10BF700000EB02030DD98C18A0420DD20B490C48DE
:10BF800040F215220AF061F840F2152107480AF044
:10BF900055F8F3D09942F0E7013A114411F801291C
:10BFA00000F8012B8342F9D110BD00BF70A0020040
:10BFB000568D02002DE9F0479AB01646DDE9239729
:10BFC0000CAA84468A4690461D462C4B03F1300E3F
:10BFD000144618685968083303C473452246F7D1DC
:10BFE00018681B79614620602371202204A8FFF79E
:10BFF000BDFF6B462022224804A90DF0ECFB04464D
:10C00000C0BB102251460DF13500FFF7AFFF1022E3
:10C0100031460DF14500FFF7A9FF294611F8013B14
:10C0200006220DF156008DF85530FFF79FFF22993B
:10C03000062211F8013B0DF15D008DF85C30FFF731
:10C0400095FF4B463522414668460DF0C4FB044639
:10C0500080B948460DF0B1FB012335228DF8303010
:10C0600041463B4668460DF0B6FB044610B93846DB
:10C070000DF0A3FB20461AB0BDE8F0873E80020019
:10C08000DBAB0200F0B50F461E46144699B00146E0
:10C09000202204A81E9DFFF769FF202239460CA824
:10C0A000FFF764FF1022314614A8FFF75FFF214617
:10C0B00010226846FFF75AFF6B465022184604A923
:10C0C0000DF089FB044660B9042203A928460BF051
:10C0D00017FB2B68044A1BBAB3FBF2F102FB1133C6
:10C0E0002B60204619B0F0BD40420F0038B50B4C14
:10C0F0000B4DAC420ED90B490B48892209F0A5FF24
:10C100008921084809F09AFF54F8043B002BF0D02D
:10C110009847EEE7F8D3002038BD00BFBC7F02008F
:10C12000CC7F0200F5AB0200568D020070B5104BBB
:10C130000546186818B10268CC0010B970BD0246F7
:10C14000FAE74389AB4208D103898B420CD9436893
:10C150001E59181956B9406840B91AB113681046EB
:10C160001A46EAE71346FAE70020E7E71819E5E779
:10C17000003F002000230360044B5A6812B9C3E952
:10C180000000704710605860704700BF003F0020FB
:10C190002DE9F04705460E4686B001F10C08348AB9
:10C1A00034B9304629680DF067FD002029686FE03A
:10C1B000072C40F2D2800822F1680DEB02000BF050
:10C1C0009FFABDF80A305BBA9AB2ADF80A30BDF8F2
:10C1D0000C305BBAADF80C30D31D328A934280F23A
:10C1E000BE80304629680DF033FD0746002800F078
:10C1F000B880082140466C6801F046FB02462046A4
:10C20000012140F8046B338A009104210FF007F9F3
:10C210003946A8680DF084FB9DF80F10BDF80C009E
:10C22000D5F80890FFF782FF00286DD09DF8083000
:10C2300013F0070332D0022B45D003243946A868F7
:10C240000DF06EFBD5F80890022109F10408404674
:10C250000FF090F900285FD04FF0020A424B4046A1
:10C2600004A90493CDF814A00FF07DF9002853D051
:10C27000214640460FF05CF9514600284ED1404619
:10C280000FF080F9304629680DF0F6FC3846296831
:10C290000DF0F2FC204606B0BDE8F0870468A868FF
:10C2A000002C31D00F2104300FF064F92846A0474C
:10C2B0000446A8680F2104300FF064F928B9002C57
:10C2C00008BF0724BAE74468E9E7002CB6D1D9E9EA
:10C2D0000032DB6804A9D21A083A02A80DF00AFB62
:10C2E000D9E90023D0681B1A1382AB6808221B68A7
:10C2F000D8680BF005FA2B683846DB6A9847044685
:10C3000020B13746002699E7082497E74046BDF854
:10C310000A1001F0B9FA42E70221B0E740460FF0F7
:10C3200031F90028AED0D9E90032DB6804A9D21A6D
:10C33000083A02A80DF0DEFAD9E90023D0681B1AEA
:10C340001382AB6808221B68D8680BF0D9F92B68F8
:10C350003846DB6A9847002794E7092421E7092437
:10C36000CFE70224CDE700BF2BAC02002DE9F0415E
:10C370008468064614F0030490B008D019491A489E
:10C38000492209F062FE4921164809F057FE0AF0D9
:10C39000F4FA4FF0013303FB00F7D6F80880444568
:10C3A00003DB012010B0BDE8F081A8EB0405402DAF
:10C3B000A8BF40256A462B46214630460AF096FA29
:10C3C0000028EFDB6A460023AD109D4201D14034C6
:10C3D000E5E752F8041BB94201D10133F5E700202B
:10C3E000E0E700BF2EAC0200568D020070B50C468F
:10C3F00015461E4648B133462A46214607480AF0EC
:10C4000041FA003818BF012070BD054B0348197868
:10C410000AF04AFA0028EED00120F5E7083F002094
:10C420002C4100207FB50D4600285DD12F4B694679
:10C430001878F6F7F3FB024638B145212C4809F08D
:10C4400018FE0124204604B070BD00980AF093FA4B
:10C45000064670B1009B5C68013C2C44214601AA51
:10C460000DF02EFE014630B122464521214809F04B
:10C4700000FE012434E0029BDDE900051D44436811
:10C48000ED1A2A460AF05CFA044630B12A464521E4
:10C490000346194809F0EDFDEBE749212A46174804
:10C4A00009F0E7FD009B99682039A94218D35B6821
:10C4B000194401AA30460DF003FE00980199436823
:10C4C0008568C91A6D1A2A460AF03AFA2A460346BE
:10C4D00010B145210A48DDE749210A4809F0C9FDA4
:10C4E00000980AF002FAADE70324ABE72C410020E4
:10C4F00077AC0200A2AC0200BAAC0200EFAC0200C2
:10C5000015AD020052AD0200012808B508D908494E
:10C510000848322209F099FD3221054809F08EFDC4
:10C5200000200DF072FC0138042828BFFF2008BD50
:10C530002EAC0200568D02007FB50C46054618222F
:10C54000002120460BF0E7F86B68581C02D103204D
:10C5500004B070BD002B5FD12A691F2AF7D9AA68E1
:10C56000511CF4D0C4E90023EE68314B32689A4282
:10C57000EDD1AA69202AEAD88AB900200DF0FCFA88
:10C58000E0B101200DF0F8FA20B901200DF034FAE5
:10C59000002817DA4FF0FF330520E360D8E725487D
:10C5A00003680133E9D0037B9A42E6D169690D3013
:10C5B0000BF07FF80028E0D10020C9E70DF01CFA4D
:10C5C0000028DEDBE0602B7FBBB9207B01A9F6F7FA
:10C5D00025FB064630B90198FFF7C8FE06460198CC
:10C5E0000AF083F9002E0CDB0CBF012300236374D7
:10C5F0002B69A36001232374DEE702A80DF005FB7D
:10C6000008B10120A4E706F1140102A80DF0FCF91D
:10C610000028DADB06209BE7064B1A68E2609A687E
:10C620002260002262606A685B689A42C4D1DFE7D8
:10C630003DB8F3962C41002020232DE9F041846879
:10C6400094B004340CAD062220466149039504934E
:10C650000DF05AFA18B1022120460EF087FF00268D
:10C6600000F0010060B9072014B0BDE8F0816B460E
:10C670002A46304601A900F067F98046B8B1013674
:10C68000022EF4D1314620460EF078FF0028EAD081
:10C690000B2220464F490DF037FA0028E3D0002145
:10C6A00020460EF045FF0028DDD00020DCE73046B4
:10C6B0000DF033FA0F21074620460EF05BFFD8B18C
:10C6C0000422204644490DF01FFAA8B13146204605
:10C6D0000EF02EFF80B10722204640490DF014FADB
:10C6E00050B105A901A800F0DBF8002868DA05229E
:10C6F0003B4920460DF008FA3A480AF0ABFF3949A9
:10C70000024620460DF000FA0028ACD0204603A9CE
:10C710000EF026FF0028A6D00822204632490DF050
:10C72000F3F900289FD00099204681F01001C1F351
:10C7300000110EF029FF002895D0072220462B4932
:10C740000DF0E2F900288ED0204607F001010EF02E
:10C750001BFF002887D00922204625490DF0D4F977
:10C76000002880D02046C7F340010EF00DFF0028BE
:10C770003FF479AF062220461E490DF0C5F9002886
:10C780003FF471AF2046C7F380010EF0FDFE002894
:10C790003FF469AF0922204617490DF0B5F900288A
:10C7A0003FF461AF2046C7F3C0010EF0EDFE002854
:10C7B0003FF459AF0F2120460EF0E4FE013651E759
:10C7C00005A88DF82C800AF045FF05A9024690E7E0
:10C7D00090AD0200D6AD020097AD02009CAD020004
:10C7E000A4AD02004DA50200AAAD0200B3AD020047
:10C7F000BBAD0200C5AD0200CCAD0200002130B5DA
:10C8000097B00446182210A8CDE902118DF8031044
:10C8100001910AF080FF1E4B02AD0C9304230D938F
:10C820001C4B6068CDE90E351B4B02221193072388
:10C8300012931A4B0CA913930DF1030314930430B4
:10C8400001AB0DF087F80546B8B9039A4AB99DF8CF
:10C85000033093B10DF0B5F980B92046FFF7ECFE37
:10C860000CE0202A09D1029904A80AF049FF2946C0
:10C8700004A80DF0AEF9002802DA032017B030BD8D
:10C880009DF8031001D10029E4D10DF07DF9E3E713
:10C890004DA502005F730200E2AD0200A373020027
:10C8A00073B50E46438805460193437819210093DA
:10C8B00003780B4A3046F7F799FF041E03DA4FF06E
:10C8C000FF3002B070BD6B683BB1064AC4F119017C
:10C8D0003019F7F78BFF031EF1DBE018F1E700BF1B
:10C8E000EAAD0200F6AD02000148FFF743BC00BF0D
:10C8F0001423002013B5114B041D00930223694635
:10C90000204601930EF02FFE98B1002120460EF034
:10C910000FFE70B10A4B6946009303232046019332
:10C920000EF021FE28B1074B204659680EF016FE86
:10C9300010B9072002B010BD0020FBE72BAC0200AD
:10C94000FAAD02002C4100202DE9F0438BB00C46DB
:10C950000DF10301064617461D460DF0BCF80146D1
:10C96000002868D12023304602AA0DF095F800284F
:10C9700061D19DF80310DFF8F880A4BB029B43450A
:10C9800040D10DB1069B2B60059BBDF81040304691
:10C990001C44042321460DEB03020DF07DF840B941
:10C9A00046F60813BDF804209A4204BFBDF80630CD
:10C9B000E4180423214630460DEB03020DF06CF819
:10C9C0000546C0BB46F60713BDF804209A4232D193
:10C9D000BDF806800434A04404F10409C14518D907
:10C9E00085F0010028E0082220460AF094FE029B10
:10C9F0009DF80310434505D10822204607A90AF0F7
:10CA00007FFEBEE74FF001325143994213D105201A
:10CA100012E00423214630460DEB03020DF03CF8F2
:10CA200048B99DF80420BDF80630FF2A07D14FF61B
:10CA3000FF72934207D101200BB0BDE8F083102AAA
:10CA400001D1202B04D0043303EB04094C46C3E787
:10CA5000002DF0D10FB90125F8E724344445EAD878
:10CA60003A46494630460DF017F80028F3D0E2E781
:10CA70003DB8F39610B5054C3022002120460AF04F
:10CA80004AFE4FF0FF33236010BD00BF2C41002051
:10CA90000023012230B58DB0CDE90123D0E9014555
:10CAA0000B931C4B07A90793042308931A4B201DD3
:10CAB000099301AB0A9302AB0CF04CFF034630BB69
:10CAC000024603A90198FFF73FFFC8B101980CF097
:10CAD000B2FF0446FFF7CEFF7CB9104B0435059337
:10CAE0000223284605A906930EF03DFD20B12146FC
:10CAF00028460EF01DFD00B9072420460DB030BDBC
:10CB000001980DF039F80028E0D00624F5E7032459
:10CB1000F3E700BF97AD02003B7302002BAC0200AD
:10CB2000F0B50024B7B008AD21464768202206467C
:10CB3000284601940AF0EFFD4FF0FF3321466822AA
:10CB40001CA8CDE909330AF0E6FD4D4B03241893E8
:10CB5000052319934B4B0BAACDE91A354A4B20926A
:10CB60001D9304231E93494B494A1F932E930DABEB
:10CB70002F93484B229231930723474A0AA92492C4
:10CB80002992329309AA454B25912A924449454A54
:10CB9000043733930FABCDE92714CDE92C2434931C
:10CBA0000622384601AB18A923940CF0D3FE0028C6
:10CBB00063D1284602A9FFF7BFFC044600285CD1D8
:10CBC0009DF8183023B9B068FFF794FE044654E08E
:10CBD000354D059B099F2B60029BAB605FB1D5E98A
:10CBE00001120C9B53BB8A42EDD1194610AA0120B9
:10CBF000FFF7AAFEE7E70E9A0D99686005F10D00B0
:10CC00002A730AF07DFD0E9A214602F10D00284498
:10CC1000C2F120020AF07FFD9DF81930002BDED012
:10CC200020460A99FFF7FEFB04460028D7D00023D0
:10CC300010AA19460120FFF787FE1EE00B449A1A3E
:10CC4000534253410B99049A0998FFF7CFFB0446CE
:10CC50000028ECD16B68049A1344AA686B60934275
:10CC6000B1D10346014610AA0120FFF76DFEB0685E
:10CC7000FFF740FE0446FFF7FDFE204637B0F0BD4B
:10CC8000FEAD02003B73020004AE02005F730200BF
:10CC900009AE020011AE020059730200A373020034
:10CCA000FAAD02000DAE02002C410020014806F052
:10CCB000C1BB00BF2C2300200148FFF75BBA00BFB7
:10CCC0002023002007B5002200230648CDE90023D9
:10CCD0004FF40052002308F095F9002003B05DF8EE
:10CCE00004FB00BF98260020002370B544688568C7
:10CCF000043486B02046CDE900330EF036FB10B97F
:10CD0000012006B070BD204602A90EF02BFB0028C2
:10CD1000F6D0039E012E1ED1029B1B78642B1AD1E4
:10CD2000694620460EF01EFB0028E9D020460EF092
:10CD300036FB0028E4D00B4B0435284604A9CDE986
:10CD400004360EF010FC20B1694628460EF00BFCAC
:10CD500030B90720D5E70021204605F009F9CEE7D4
:10CD60000020CEE7CEB0020013B5134B84680093C9
:10CD7000082304346946204601930EF0F4FB28B1E1
:10CD800040F6AB1120460EF0DDFB10B9072002B0D3
:10CD900010BD0A4B694600930923204601930EF00B
:10CDA000E2FB0028F2D0042120460EF0CBFB002845
:10CDB000ECD00020EBE700BF19AE020022AE02006B
:10CDC0000148FFF7D7B900BF3C23002013B5062068
:10CDD00001A9F5F723FF041E06DA45210C4809F0E6
:10CDE00048F9204602B010BD019809F0C4FD38B9D9
:10CDF0004521084809F03DF9019809F076FDF0E772
:10CE000001980021826809F09BFD0028F4DAEFE721
:10CE10002CAE02004BAE020013B5084C204606F0C3
:10CE20005DFB074B204600934FF4905203230549C6
:10CE300006F06AFB002002B010BD00BFA83300203E
:10CE400060870200505D00200022002301480CF0A2
:10CE5000EFBF00BF802900202DE9F8430446DDE93B
:10CE600008981D460F461646002148220AF053FC3A
:10CE70002046C4E90B76C4E90D59C4F83C800CF097
:10CE800008FF2046044906F03BFA04F11000BDE813
:10CE9000F8430EF0F3BB00BF1F5C020010B5044660
:10CEA000103000F0FFFB2146BDE8104001480EF0B5
:10CEB0006ABC00BFA8330020F0B5C36B04460E4621
:10CEC00089B003B306F03CFA10F0050F02D02046FB
:10CED00006F0B6FA01A80EF0D1FB04F1100700220B
:10CEE000002338460CF0A9FF054670B90022002344
:10CEF00001A80CF0A2FF0146A8B923691BB1214685
:10CF00000B480EF040FC09B0F0BD3146E36B98478A
:10CF100020B9214628460CF0AFFEE0E7294601A8DB
:10CF200000F0C0FBDBE7384600F0BCFBDEE700BFEB
:10CF3000A8330020034B1A6882420CBF1846002019
:10CF4000704700BF483400202DE9F74307461646D6
:10CF50001D46FFF7EFFF814648B93A4645212B4869
:10CF600009F087F86FF0100003B0BDE8F08328489F
:10CF70000CF094FE314604462A4625480CF096FEF5
:10CF800010F10C0F0646EDD000280CDA20480CF00A
:10CF9000EBFE10B10023036003711D480CF0D6FEB8
:10CFA0006FF01200E0E7002C28DA19480CF0DCFEE4
:10CFB00080463846FFF7BEFF0446C8B190F8683097
:10CFC000D9070ED44FF42813124A69463846CDE9E2
:10CFD00000230CF0EDFE94F8683043F0010384F870
:10CFE00068304FF42032002304F1080006F04CFCB6
:10CFF000C8F8007099F8693088F804301EB93146D5
:10D0000003480CF08BFE2846AEE700BF93AE02004B
:10D010005C410020060009001FB590F8302003464F
:10D0200012F0010F09490BD06A460868496803C22B
:10D03000694653F8380C0CF0BBFE05B05DF804FBF4
:10D040008868C96802AA03C202A9F2E72C8002001C
:10D0500013B504466B46084A9068D16803C3694615
:10D0600054F8080C0CF0A4FE94F8603023F001038F
:10D0700084F8603002B010BD2C80020038B505463F
:10D08000FFF758FF044629460F48FFF715FF9CB1EC
:10D090000025204684F8695040F8085B06F0FAFB4A
:10D0A00004F1380006F0F6FB84F8685004F16C00D7
:10D0B000BDE8384005F094BE2A46BDE83840452119
:10D0C000024808F0D6BF00BF5C41002093AE0200CA
:10D0D00010B509480C460CF0E1FD00280ADB4CB9FC
:10D0E00005480CF041FE04600471BDE810400248A0
:10D0F0000CF02CBE10BD00BF5C4100202DE9F04FAC
:10D1000004468FB01822002168460AF004FB3B4B0E
:10D11000D4F818900193E3680293394B0493B9F162
:10D12000000F0BD1052604F118000CF021FE20465B
:10D130000CF08CFD30460FB0BDE8F08F484606A9D4
:10D14000FAF752FB06460028ECD19DF83430022B4A
:10D15000E8D120460CF047FE054608B90126E2E773
:10D160004846FFF7E7FE07460028DBD090F8693015
:10D17000002BD7D0227F9A42D4D100F16C0A5046BE
:10D1800005F0C8FEB346B046238A4345CBD997F88D
:10D190006920002AC6D0217F9142C3D108EB050245
:10D1A0009A42C4BFA3EB08039DB269464846ADF856
:10D1B0000C50FCF7C9FF10F10C0F09D1BBF1000FA7
:10D1C00003D1132D18D9C5F34F0507F0C5F9DBE7D7
:10D1D0000028C3D1E26808EB05031FFA83F812FAAE
:10D1E00083F302934FF0FF324FF0FF33504605F0C8
:10D1F00031FE4FF0010BC7E7022694E77C230020A5
:10D20000F75D020008B5E1B90E4A136843B10E4953
:10D210000E48932208F019FF93210B4808F00EFFE7
:10D220000B4910600B7882F869300133DBB2012BB7
:10D2300038BF01230B7002F16C00BDE8084005F017
:10D2400069BE08BD48340020BAAE0200568D020007
:10D25000A14600200148FCF7B5BB00BF48230020D1
:10D2600013B50124124B134913481C7006F022FA1F
:10D270001249134806F01EFA0021224611480EF00A
:10D280001FFA114B114A0193114B12491248009396
:10D29000124BFFF7E1FDFFF7DDFF024630B14521FC
:10D2A0000F4802B0BDE8104008F0E3BE02B010BD68
:10D2B000A146002051900100503400201990010037
:10D2C00080340020B43400208B5D0200E75D020052
:10D2D000715D0200FD9001005C4100207D5D020057
:10D2E000F7AE02003422024B02FB0030704700BF51
:10D2F000142800203421827A064B01FB02331A6B7A
:10D3000093F82430801A1B3323F00303B0FBF3F0AF
:10D31000704700BF1428002038B53424827A094BA6
:10D3200004FB0233DB6A0C685B681A68944294BFA2
:10D330000C600A60D3E90054FFF7DCFF05FB0040F6
:10D3400038BD00BF1428002008B5437A43B10B490B
:10D3500056220B4808F079FE5621084808F06EFE68
:10D36000436833B105495722054808F06EFE57213E
:10D37000F3E703824369C36008BD00BF2DAF02001D
:10D38000568D02002DE9F04F85B0039105461946F0
:10D3900010469146984617461E460EF040FACDE9D3
:10D3A00001013DB95E49F4225E4808F04EFEF421C9
:10D3B0005B4814E005F11C0A4FF02003EFF3118BDA
:10D3C00083F31288BFF36F8F504605F0B1FA40B96E
:10D3D00055499422534808F038FE9421524808F0E9
:10D3E0002DFE504605F0C0FA6B8C002B6AD02A8CBB
:10D3F0009A4247D900220023284605F099FC0446AA
:10D4000000283FD0504605F0A1FA30B94649C22263
:10D41000444808F01AFEC221E0E78BF31188BFF3FD
:10D420006F8F039D002D6FD058EA090310D0B8F11B
:10D43000FF3F08BFB9F1FF3F0AD007F00BFD019B8A
:10D440001F1A029B63EB0106002EBCBF00273E465D
:10D450004FF03409A37ADFF8D4803A4609FB0383FE
:10D46000DB6A20461B6803A9D3F800A03346D047E7
:10D47000606100283CD1A07A214600FB09800EF0B3
:10D4800015F930E06C8C5046631E6B8405F05EFA33
:10D490000028BBD08BF31188BFF36F8F95F8243031
:10D4A0002A8C1B33121B2C6B23F0030302FB034457
:10D4B0001E4B1F4AEB1A9B105343A37295F824305E
:10D4C000E372AEE7504605F041FA00289ED08BF398
:10D4D0001188BFF36F8F4A464346284605F028FC63
:10D4E000044600289DD10024204605B0BDE8F08FF9
:10D4F000039B9D4209D90A4940F25512094808F098
:10D50000A4FD40F2551153E76561002301226360D9
:10D5100022812382039A63696282E360E4E700BFA9
:10D520002DAF0200568D0200908D020014280020BD
:10D53000C54EECC408B550B90C494FF4DC720C4828
:10D5400008F083FD4FF4DC71084808F077FD83880C
:10D5500043B1064940F2B912054808F076FD40F2A1
:10D56000B911F1E783680B44036008BD2DAF0200D9
:10D57000568D020070B50C46054650B9224940F25E
:10D58000C512224808F061FD40F2C5111E4808F09E
:10D5900055FD41B91C494FF4E3721C4808F055FD94
:10D5A0004FF4E371F2E74FF02003EFF3118683F3BA
:10D5B0001288BFF36F8F164805F0BAF938B91549CC
:10D5C0009422124808F041FD94211248DFE71048E8
:10D5D00005F0CAF9002323606B6863B9C5E900440C
:10D5E0000B4805F0B3F948B90A49C222074808F0C8
:10D5F0002CFDC221E9E71C606C60F1E786F311881D
:10D60000BFF36F8F70BD00BF2DAF0200568D0200BB
:10D61000A4410020908D020070B5044650B91D4908
:10D620001D484FF4E97208F010FD4FF4E9711948F4
:10D6300008F004FD4FF02003EFF3118683F3128806
:10D64000BFF36F8F154805F073F938B91449942268
:10D65000114808F0FAFC94211148E9E70F4805F059
:10D6600083F925682DB162682B689542236008BF55
:10D6700063600A4805F06AF930B90949C2220648D0
:10D6800008F0E3FCC221E7E786F31188BFF36F8F50
:10D69000284670BD2DAF0200568D0200A441002027
:10D6A000908D020008B550B90C4940F2DF120C48C9
:10D6B00008F0CBFC40F2DF11084808F0BFFC41B98C
:10D6C00006494FF4F072064808F0BFFC4FF4F071C1
:10D6D000F2E7BDE808400DF0DEBF00BF2DAF02004D
:10D6E000568D02002DE9F041054628B300274FF082
:10D6F00034081A4E2C46237A6D68013BDBB2237244
:10D70000C3B9616959B1637ADB0707D4A37A2046AC
:10D7100008FB0363DB6A1B689B6898476761A07A14
:10D72000E76008FB006367609B6A83B12046984707
:10D73000002DDFD1BDE8F08109490A4840F2EB1223
:10D7400008F083FC40F2EB11054808F077FC214615
:10D7500000FB08600DF0AAFFEAE700BF14280020D4
:10D760002DAF0200568D020008B550B90749084890
:10D7700040F21A2208F069FC40F21A21034808F02E
:10D780005DFC027A0132027208BD00BF2DAF0200BB
:10D79000568D020008B5034650B90849084840F2C2
:10D7A000572208F052FC40F25721044808F046FC8A
:10D7B00018465B68002BFBD108BD00BF2DAF0200EF
:10D7C000568D020070B50D46044650B90E4940F220
:10D7D00062220E4808F039FC40F262210A4808F043
:10D7E0002DFC41B9084940F26322084808F02DFC9D
:10D7F00040F26321F2E746681EB10846FFF7CAFF10
:10D800004660656070BD00BF2DAF0200568D0200FE
:10D8100038B505460C4651B90B490C4840F26E220A
:10D8200008F013FC40F26E21074808F007FC20B90D
:10D83000BDE838400846FFF797BFFFF7ABFF21462A
:10D84000FFF7C0FF284638BD2DAF0200568D0200FD
:10D8500008B5034600689A68821A91420AD90849B5
:10D86000084840F2F23208F0F0FB40F2F23104488E
:10D8700008F0E4FB9A88401A11441860998008BDAA
:10D880002DAF0200568D020008B5828803468A42F9
:10D890000AD20849084840F2524208F0D6FB40F24A
:10D8A0005241044808F0CAFB521A828000680844BA
:10D8B000186008BD2DAF0200568D020008B5034662
:10D8C0009A8800688A420AD20749084840F25E42B4
:10D8D00008F0BBFB40F25E41034808F0AFFB521A70
:10D8E00001449A80196008BD2DAF0200568D0200D8
:10D8F000F8B5858803680E4604465F190CF0B2FA45
:10D90000B0420AD20749084840F2033208F09DFBB2
:10D9100040F20331034808F091FB3544A5803846B6
:10D92000F8BD00BF2DAF0200568D020037B5402371
:10D930000C460A490093411A491105462346084AF4
:10D9400008480CF0BDFA011E05DA2846234603B04C
:10D95000BDE83040184703B030BD00BFBC410020D7
:10D960002F5F02006C7A0200C9B2032908B508D9FA
:10D97000084909487A2208F068FB7A21054808F02E
:10D980005DFB0C22036901FB0233D3F8880000F031
:10D99000070008BD59AF0200568D020070B5C9B22C
:10D9A000032903690AD91949194840F25D1208F0A0
:10D9B0004CFB40F25D11154808F040FB4FF020048D
:10D9C000EFF3118584F31288BFF36F8F0C2606FBEB
:10D9D0000134D4F8884014F0C00408D0A24206D024
:10D9E00085F31188BFF36F8F4FF0FF3070BD0122B8
:10D9F00071430B44C3F8882085F31188BFF36F8F00
:10DA000043680B445B6898470020EFE759AF02007A
:10DA1000568D020070B50D4606490446411A49115B
:10DA200040220548FFF7BAFF2B4601462046BDE8D5
:10DA300070401847BC4100206C7A02002DE9F84381
:10DA40000022012106460520F6F71CF9114802F0D4
:10DA5000C1FB114B984219D102F0DEFB00244FF0BC
:10DA60000C080127DFF834903569494605EB44106E
:10DA700008F060FA002807DB08FB04550134042C89
:10DA8000C5F88870F0D10020BDE8F8836FF004007D
:10DA9000FAE700BFD99A01000000AD0B74870200BD
:10DAA00001460C23002270B54B430948C418883343
:10DAB000D4E920561844C4F880200CF0EEF92DB1BA
:10DAC00032462B46BDE870400248184770BD00BF83
:10DAD000BC4100206C7A020008B505281FD8DFE899
:10DAE00000F003111E130F0D124BD3F8880010F035
:10DAF00007001DD1BDE80840FFF7D2BF0220F9E7BB
:10DB00000320F7E70120F5E70B4940F26E220B48AE
:10DB100008F09BFA40F26E21074808F08FFA064998
:10DB200040F27222054808F090FA40F27221F3E7C1
:10DB300008BD00BFBC41002059AF0200568D020055
:10DB400008B54FF02003EFF3118183F31288BFF380
:10DB50006F8F124A136843F002001060DA0708D48E
:10DB600081F31188BFF36F8FBDE80840012002F0F8
:10DB700079BB4FF05023D3F80C24D3F80C34D307DF
:10DB8000EED507480CF089F981F31188BFF36F8F48
:10DB9000BDE808400020FFF783BF00BF6C420020B3
:10DBA000444200207FB500220123CDE9022304ABCB
:10DBB000CDE90433094A6B46CDF800D0CDF804D046
:10DBC0000CF0AEF9002805DB4FF4804200236846D4
:10DBD00005F040F907B05DF804FB00BF5F5F02008D
:10DBE00010B54FF02003EFF3118483F31288BFF3D5
:10DBF0006F8F074A136823F00201DB07116002D41C
:10DC0000012002F0A7FB84F31188BFF36F8F10BDD2
:10DC10006C4200202DE9F041012206464249D1E83C
:10DC2000EF3FC1E8E02F0028F9D19BB93F494048B8
:10DC30004B60CB608A60F3F7D1FB00280ADA3D49DC
:10DC40004FF40C723C4808F000FA4FF40C7139485C
:10DC500008F0F4F976B3731E012B5CD8012E07D1BE
:10DC60004FF05023D3F81C3403F00303022B21D0D0
:10DC70000DF0D5FC0546F8B9304B1B78E3B14FF0F9
:10DC8000502302220746C3F808234FF05024DFF840
:10DC9000B080D4F81834D4F81824D20316D503F081
:10DCA0000303022B01D0012E10D175B387F3118825
:10DCB000BFF36F8FBDE8F0814FF02003EFF31187C2
:10DCC00083F31288BFF36F8F0125DEE7C5B13846B5
:10DCD000F5F768FFD4F81835DBB2012BD9D1D4F8A9
:10DCE0000421002AD5D00022C4F80421D4F804214C
:10DCF0000222C4F818252022C8F88021A360C8E7B2
:10DD00000021212006F026FDE4E74FF050230222F7
:10DD1000C3F80423CEE7074940F24222064808F040
:10DD200094F940F2422192E7B8410020A841002036
:10DD3000DC41002059AF0200568D0200A6460020AB
:10DD400000E100E008B507480DF02DFC38B10648A9
:10DD5000F6F746FD0448F3F713F8002008BD6FF00E
:10DD60001200FBE7B47A02006D9D01000A2838B565
:10DD70000446074D04D1AB680D2128465B689847DF
:10DD8000AB6803485B68E1B29847204638BD00BFE6
:10DD9000B47A020010B5036941B91C492A221C4813
:10DDA00008F053F92A21194808F048F9486830B9B1
:10DDB00016492B22164808F048F92B21F3E758683A
:10DDC000F8B1884219D19C680868A142586000D116
:10DDD0009860002008602AB15A680A609A68596001
:10DDE00002B99960002010E0814206D108682060E5
:10DDF00098688142EDD19C60EBE7044600680028FA
:10DE0000F2D1002AE8D16FF0150010BDD0AF0200AA
:10DE1000568D020030B5406801F01F04057BB2F555
:10DE2000001F85B044EA451405D1204602F0C0FD2C
:10DE3000002005B030BD0025B2F5800FCDE90255B8
:10DE400014D1B3F1007F0CBF042305238DF80830F3
:10DE500000232046194602AA02F0BAFB2A4B984238
:10DE60004ED10121204602F03DFDE1E7B3F1C06F44
:10DE700023D0B3F1007F14BF012302238DF80830B3
:10DE80008368CB40D807E3D4B2F1A07FE0D1620928
:10DE900004F01F0313D0012A04D14FF6FF72DA40B9
:10DEA000D10713D419491A4840F2472208F0CDF897
:10DEB00040F24721154808F0C1F80323DEE74FF090
:10DEC000FF32DA40D207EDD5124A00E0124A803321
:10DED00052F82330DB07BBD40DF107052946204655
:10DEE00002F09CFC0D4B984201D00395B0E7284608
:10DEF00002F0F2FC044B9842F7D06FF00B0098E769
:10DF00006FF0150095E700BF0000AD0B1F8E0200FB
:10DF1000568D020000258450002884500400AD0B6B
:10DF200010B502F0C9FC044668B902F09DFC084B2C
:10DF300098420AD12146074802F06AFC2246052190
:10DF40000D20F5F79FFE002010BD6FF00400FBE7E9
:10DF50000000AD0B599F01004209034670B502D085
:10DF6000012A1AD070BD124E326951680029F9D0C9
:10DF7000012503F01F030C689D400029F2D08A6838
:10DF80002A400ED04B6853B90A490B484D2208F07D
:10DF90005CF84D21074808F051F8084EE4E7304698
:10DFA00098471CB1236821461C46E6E72346FAE75A
:10DFB0009C7A0200D0AF0200568D0200847A0200E3
:10DFC0002DE9FF41D0F8048001F01F0598F80C30CE
:10DFD000144645EA43150F4628460DF1030102F0A9
:10DFE0001DFC14F4403F064614D1284602F00AFDF9
:10DFF000474B9E426ED19DF8030002F067FCB04291
:10E0000068D044496A22444808F01FF86A21414810
:10E0100008F014F800232846194602AACDE9023375
:10E0200002F0D6FA3A4B984204D06FF0150004B0D3
:10E03000BDE8F08186420CD19DF8030002F046FC59
:10E04000B04206D033497C22334807F0FEFF7C21E2
:10E05000DDE7A6034CD540F206332340B3F5837FBA
:10E0600019D00CD8062B17D004D8ABB1022BDCD1B9
:10E07000042311E0B3F5807FD7D101230CE040F2F7
:10E080000222934228D0B3F5407F27D0B3F5007F1A
:10E09000CBD1022300E007238DF8043084F48033D1
:10E0A000C3F30043E0068DF805304CBF0323C4F3EF
:10E0B000401321038DF8063012D50123D8F804202F
:10E0C000BB4093600022284601A902F029FB104BB7
:10E0D0009842AAD10020AAE70523DDE70323DBE766
:10E0E000620341BF0123D8F80420BB40D360E9E7B5
:10E0F000E3064FF000034CBF0324C4F340141A4658
:10E10000284601A98DF8044002F062FADFE700BF5B
:10E110000000AD0B0CB00200568D020000F17440FF
:10E1200000F5A6000A289ABF024B33F910006FF0E1
:10E130000F007047308A0200024B0B60012313600E
:10E14000704700BF7C8802000048704710880200BA
:10E15000054B994206D14FF0FF324FF0FF3330307C
:10E1600004F078BE704700BF0000AD0B70B50569C4
:10E1700004460F4E28460BF024FF05F148000BF033
:10E1800018FF33788BB92A460A49606802F0B8FF55
:10E19000FFF7C4FFB0FA80F305465B0933702069CE
:10E1A00018300BF006FF284670BD0025F7E700BFCA
:10E1B000A2460020B75F0200F7B54C680546174637
:10E1C000ACB1D4E90043886898B1D0E9006088B167
:10E1D00083B1984207D10133092B0A780DD9572111
:10E1E000164807F046FF6FF0150003B0F0BD234658
:10E1F000E9E7064601330344EEE78DF8013040F2CB
:10E200000113ADF80230002328698DF804308DF831
:10E2100000208DF805700BF0D4FE2146324668468A
:10E2200003F05CF80446286918300BF0C2FE204663
:10E2300003B0BDE8F040FFF771BF00BF50B002006F
:10E2400038B5044600690BF0BCFE256900220023A6
:10E2500005F1480004F0FEFD2B6D4BB90A4D03F0AB
:10E2600099F8A8420AD103F0B7F80022074B1A70B8
:10E270002069BDE8384018300BF09BBE002140F209
:10E28000676006F067FAEAE70000AD0BA2460020DF
:10E290002DE9F04F81460E461C46904685B07AB176
:10E2A000002B00F09C800029426803DB9269CB18A8
:10E2B00093420BD92346324645214A4807F0D9FEFE
:10E2C0006FF01505284605B0BDE8F08FFFF74EFF4B
:10E2D000054600287FD1754205F00305D9F81000E6
:10E2E0000BF06FFEA54228BF2546D8F1000303F0CE
:10E2F000030308F0030758BF5F427F4207F003079C
:10E30000A74228BF2746631BE41B24F0030423F025
:10E31000030AA245C8BFA24603F0030BC8BFA3EB84
:10E32000040BBAF1000F19D008EB0703721951461C
:10E33000184601930CF09AF904460146D9F81000EA
:10E34000FFF706FF284A94423CD1BD4206D0019B0C
:10E350005246194608EB050009F0BBF9BDB1C5F1FD
:10E3600004070421F21B02A80CF080F904460146C0
:10E37000D9F81000FFF7ECFE1B4B9C4222D107F1AD
:10E3800008032A4640460DEB030109F0B9F9BBF139
:10E39000000F16D00821721952440DEB01000CF049
:10E3A00065F904460146D9F81000FFF7D1FE0E4B7F
:10E3B0009C4207D10AEB05005A4602A9404409F0E5
:10E3C0009FF9094CD9F8100018300BF0F2FD2046E7
:10E3D000FFF7A4FE05464846FFF732FF72E71D46E9
:10E3E00070E700BF78B002000000AD0B4FF0502383
:10E3F00002222DE9F041C3F8B82543688AB01E6AAD
:10E4000005460021304607AA0BF0FBFE041E2FDB59
:10E41000079B3268197918680BF006FF041E27DB8A
:10E42000002201212B20F5F72DFC6E682A69304669
:10E430004A4902F065FEFFF771FE041E18DBF37A0D
:10E44000023B012B18D996F80A80A8F10308B8F10D
:10E45000010F8CBF4FF000084FF0010828460BF069
:10E46000D2FD041E0BDA224645213D4807F001FE8D
:10E4700020460AB0BDE8F0814FF00108EEE7E2B2B5
:10E48000C4F38014A04504AE05AF28D0002382F069
:10E490004002ADF810308DF810200122284607A95F
:10E4A000CDE90623059609938DF81C200897FFF700
:10E4B00083FE041E0CD0DBDA2A492B4A2346B8F12E
:10E4C000000F08BF0A462948452107F0D2FDCFE7D3
:10E4D00028460BF098FD041EEEDBE307F8D428462F
:10E4E000FFF7AEFE4FF003080023CDE90683089343
:10E4F0009F23284605968DF81C300997FFF736FEB6
:10E50000024628B12846FFF79BFE6FF01204AFE7E2
:10E51000284607A9FFF750FE04462846FFF790FE5D
:10E52000002CF2D16D684246314605F11C0009F01D
:10E53000C0F8044600289BD0AB7F452103936B7F36
:10E540009DF8102002932B7F094801939DF812300B
:10E5500000939DF8113007F08CFDD6E7B75F0200FD
:10E56000D0B00200CAB00200C6B00200E5B002009E
:10E57000FBB002002DE9F84F15460A1E0646D0F8FA
:10E58000049005DBD9F8183051199942904609D901
:10E590002B4645213B4807F06CFD6FF015042046E3
:10E5A000BDE8F88FC2F30B02002DF6D0C5F30B03C4
:10E5B0001343F2D1FFF7DAFD044668BB30690BF074
:10E5C00007FD214630460BF009FD044608BB3069C3
:10E5D0000BF0F7FCDFF8B0A0D9F81830AB421FD130
:10E5E0000CF047F8AB46074639463069FFF7B0FDF7
:10E5F00057453BD1B5EB0B05D844EDD13069183008
:10E600000BF0D7FC012130460BF0E8FC002C08BFD2
:10E61000044630690BF0CDFC3046FFF711FEBEE733
:10E62000B5F5803F0AD31FFA88F353B9414601205C
:10E6300002F032FF4FF4803B0746D5E7B5F5805F27
:10E6400009D3C8F30B0030B9414602F025FF4FF45F
:10E65000805B0746C8E72B46424645210B4807F03A
:10E6600008FD0B493069FFF773FD094F2B46094838
:10E670004246452107F0FDFC3846FFF74FFD0446B2
:10E68000BCE700BF32B102000000AD0B81B1020057
:10E690000400AD0BA4B102002DE9F34705460F4677
:10E6A0001E4690469AB193B1042B01D99A070ED118
:10E6B000BB070CD1002F6A6803DB9269BB19934238
:10E6C0000BD933463A4645213D4807F0D2FC6FF05E
:10E6D0001504204602B0BDE8F0872846FFF746FD46
:10E6E0000446002863D128690BF072FC21462846B5
:10E6F0000BF074FC044628690BF063FC002C43D13A
:10E70000032E1ED804213A460DEB01000BF0AEFF9C
:10E71000044601462869FFF71BFD2A4B9C4233D172
:10E720003246414601A808F0EBFF04213A460DEBC2
:10E7300001000BF098FF044601462869FFF708FD29
:10E7400022E008F06043B3F1005F34D0DFF874A03A
:10E75000042EB14628BF4FF0040941464A4601A89D
:10E7600008F0CEFF04213A460DEB01000BF07BFFD1
:10E77000044601462869FFF7EBFC544504D1B6EB8B
:10E780000906C8444F44E3D1286918300BF011FC46
:10E79000012128460BF022FC064628690BF009FCF3
:10E7A000002C14BF20463046FFF7B8FC044628462C
:10E7B000FFF746FD8DE73A4631464046B9E700BFD0
:10E7C000C7B102000000AD0B024B0B6001231360C8
:10E7D000704700BF884200200048704798880200B8
:10E7E00070B50D461946284616461C460BF026FC09
:10E7F00040B9084823462A46452107F03AFC6FF005
:10E80000150070BD24B122462946304608F078FF35
:10E810000020F6E72CB2020010B50122064811468E
:10E820000CF04EFF0BF019FF044C20600BF012FFB0
:10E830006060002010BD00BF904200208842002090
:10E84000F8B50E4614460BF005FF21460546304646
:10E850000BF0F4FB374650B3B6FBF5F305FB13633F
:10E8600023B9B4FBF5F305FB134343B1234632460A
:10E870004521114807F0FDFB6FF0150002E0A542AD
:10E8800001D90020F8BD4FF0FF324FF0FF330B48A5
:10E8900004F0E0FA0BF0DEFE0546384602F088FA96
:10E8A000641B2F44F9D1054804F09AFAE9E723469E
:10E8B000324645210248DDE74EB202009042002078
:10E8C0002CB20200F8B50E461946304617461C46D3
:10E8D0000BF0B4FB40B9234632464521164807F0F9
:10E8E000C8FB6FF01500F8BD46EA040515F00305F6
:10E8F00004D02346324645211048F0E7A4B14FF03A
:10E90000FF324FF0FF330E4804F0A4FA24F0030462
:10E91000AC4206EB050009D10A4AD2F80034DB0705
:10E92000FBD5074804F05CFA0020DCE7795902F0D7
:10E930006FFA0435ECE700BF2CB2020072B202009D
:10E940009042002000900350F0B54B79012B29D064
:10E95000032B24D110278B79032B20D1CE790EB134
:10E96000012E1CD10A79012A1ED0022A20D0B2B968
:10E9700014460B684568B3F5164FD5F800C06ED045
:10E9800033D8B3F5165F6DD01CD8B3F5966F6BD046
:10E9900010D8B3F5967F6AD0B3F5167F6AD06FF0C2
:10E9A00085005BE00027D6E74FF480740E22E0E795
:10E9B0000024FBE7B3F5166F5FD0B3F5965FEED199
:10E9C000384B3CE0B3F5E14F5AD007D8B3F5615F5F
:10E9D00058D0B3F5964FE2D1334B30E047F61225CD
:10E9E000AB42DCD14FF4000329E0B3F5613F4BD0DB
:10E9F00013D8B3F5963F4AD009D84DF6C025AB429F
:10EA000047D0B3F5614FCAD14FF46B0317E0B3F5AC
:10EA1000E13FC4D14FF0EB7311E0B3F5612F3BD070
:10EA200008D8224DAB423AD0B3F5E12FB7D14FF021
:10EA3000E86304E01E4DAB42B1D14FF0805305694D
:10EA4000CCF8243543683A431B6834432243C3F867
:10EA50006C252B1D03C983E803000020F0BD4FF493
:10EA60001D03ECE7134BEAE74FF49E23E7E74FF46F
:10EA7000A033E4E74FF41C33E1E74FF41D23DEE756
:10EA80000D4BDCE70D4BDAE74FF06C73D7E70C4B1F
:10EA9000D5E74FF46503D2E74FF07063CFE74FF04F
:10EAA0008063CCE700B0130000A04E0090D00300BC
:10EAB00040420F000050270000C0750000F03A00EF
:10EAC00000903A012DE9F7438046002201210820F9
:10EAD000F5F7D8F80820F5F7A5F80021D8F8047064
:10EAE000D8F810603C6801AAC4F80015C6F8008088
:10EAF000D7F80C9048460BF084FB051E1EDB019BEB
:10EB0000D9F80020197918680BF08EFB051E15DB6B
:10EB10004046311DFFF718FF054678B97B68990715
:10EB20002BD506F1180001F087FC284B984209D03C
:10EB30004521274807F09DFA6FF00405284603B0E9
:10EB4000BDE8F083337E14F10C0F43F00043C4F8AA
:10EB5000A0310AD11F49204840F24E2207F075FA31
:10EB600040F24E211B4807F069FAC4F88C300123AB
:10EB7000327E9340194AC2F804350823C4F80035A0
:10EB80003B7A53B9C4F81031D4F810317369C4F822
:10EB900034350123C4F8383523607B689A075CBF9D
:10EBA0004FF48073C4F804337B68DB0644BF4FF432
:10EBB0008003C4F804333369C4F844350023C4F82F
:10EBC00048350123A360E360B8E700BF0000AD0B48
:10EBD000B6B20200DAB20200568D02000070015097
:10EBE000F8B504460D4607690CF019FDB0B92E4B77
:10EBF0001B789BB1642660680BF0B5FA00BB01205E
:10EC00000BF0ABFC013EF6D10021212005F0A2FD66
:10EC1000F0E786F31188BFF36F8FF5E74FF020031D
:10EC2000EFF3118683F31288BFF36F8F606831466C
:10EC30000BF099FA90B986F31188BFF36F8FEDE767
:10EC40004FF02003EFF3118683F31288BFF36F8F29
:10EC5000606831460BF087FA0028DAD03B691D70F6
:10EC6000626838691368C3F844050120C3F8480591
:10EC70000020C3F82001D3F82051C3F8580152688E
:10EC8000D3F85801D20608D5082062681268C2F885
:10EC900000054FF48002C3F8042301229A6081F337
:10ECA0001188BFF36F8FF8BDA646002010B5064847
:10ECB000F6F7DCFF041E04DA22464521034807F07C
:10ECC000D8F9204610BD00BFE88802002CB302002E
:10ECD00010B5027E0446022A0CD0042A09D0C2B123
:10ECE00045210D4807F0C5F92046FEF7FBFC002042
:10ECF00010BD0522114604F10C000BF0A0F8228A89
:10ED0000E1680648F3F724FC021EEDDA45210448C9
:10ED1000E8E70122EEE700BF5BB30200A842002053
:10ED200070B30200014804F05BB800BFAC270020BC
:10ED300010B51348F3F7CEFB044648B110F1780F35
:10ED400006D0452102460F4807F093F9204610BD32
:10ED50000D4A0E490A48F3F7DBFB044618B1024698
:10ED600045210B48F0E74FF400420023094804F026
:10ED700071F804460028E9D0024645210648E3E739
:10ED8000CC7A02008DB3020044240020A842002067
:10ED9000C2B30200AC270020EBB302002DE9F74319
:10EDA0008046064618F8010B0C46042801F1FF3393
:10EDB0000AD0052800F08180022840F0AD80032BA6
:10EDC00056D84521584803E0012B06D8452157481D
:10EDD00003B0BDE8F04307F04CB973783E2B14D173
:10EDE000F778BB1E5F425F410222414601A808F04E
:10EDF00087FC9DF80530033C9C4208D045214C48D7
:10EE000007F037F903B0BDE8F0830027ECE77FB1E6
:10EE10004FF000084FF0000942464B4639469DF836
:10EE20000400F5F7BFFE054628B9002FF4D0E9E746
:10EE30004FF4A028EEE700F10C07022201A93846A2
:10EE40000BF018F838460BF00DF8844203462246C2
:10EE500004D94521374807F00CF927E0F11C384662
:10EE60000BF008F8284603B0BDE8F043F6F7D8BE2B
:10EE7000002200230320F5F74FFE0546D0B10422FF
:10EE800041460DEB020008F03BFC042205F10C07A3
:10EE900038460DEB02010AF0EDFFBDF80630053CE7
:10EEA0009C4230D04521244807F0E3F82846FEF77D
:10EEB00019FCA7E7452121488AE7032B02D8452101
:10EEC0001F4885E700220023F5F726FE0546B8B166
:10EED000042241460DEB020008F012FC042205F169
:10EEE0000C0738460DEB02010AF0C4FFBDF80630EE
:10EEF000053CC3F30D039C4205D045211148D3E7DF
:10EF00004521114864E738460AF0ACFF84420346C5
:10EF100022469ED8711DA2E7024645210B4803B048
:10EF2000BDE8F04307F0A5B887B4020010B40200B2
:10EF300036B402005FB40200CAB40200ABB40200EF
:10EF4000F1B4020034B5020015B502005BB5020051
:10EF500070B40E4922F07F46D1E90034D01AC318AC
:10EF600044F10004C1E90034A6F50013B3F5400FE5
:10EF700009D2074B1B681A0A1B069C19054B42F164
:10EF80000005C3E9004570BC05F0D6BEE0340020A2
:10EF9000B8420020E83400200D4B1868010A000632
:10EFA000BFF35F8F0B4BD3F80435181841F1000104
:10EFB000B3F5801F0AD2084BD3E90023904271EBCE
:10EFC000030303D210F1807041F10001704700BFCC
:10EFD000B842002000500150E83400202DE9F743EA
:10EFE0002E4BD3F8042390070BD5D3F8042142B15C
:10EFF0000022C3F804212A4AD3F8043113680133EC
:10F000001360264AD2F80433D90327D5254BD3E819
:10F01000EF1F21F00100C3E8E40F002CF7D1CB076C
:10F0200002D4D2F84031CBB100251C4CC4F8405179
:10F03000D4F84031FFF7B0FF4FF02003EFF3118217
:10F0400083F31288BFF36F8F174BD3E90267B04287
:10F05000B94106D282F31188BFF36F8F03B0BDE8C8
:10F06000F0834FF0FF38D3E900104FF0FF391D60F7
:10F07000C3E902894FF48033C4F84833C4F84051DF
:10F08000D4F8403182F31188BFF36F8F0029E5D0A7
:10F09000009032463B4628468847DFE70050015043
:10F0A000B8420020B0420020D03400202DE9F84FB3
:10F0B00004460D46434FD7E8EF8F28F00103C7E819
:10F0C000E23F002AF7D14FF480393F4EC6F808934B
:10F0D000BFF35F8FBFF36F8FFFF75EFFA04271EB4F
:10F0E000050308F0010840D2384B201A65EB0101F6
:10F0F000984271F1000148D2354BD3E902239D4279
:10F1000008BF94423AD04FF0000C24F07F40834671
:10F1100003216FF0020EC6F84893C6F840C1D6F836
:10F120004031DFF8B0A02BF07F43C6F84035C6F879
:10F130004493D6F80425AEEB02035B4423F07F43EF
:10F1400053451BD9D6F840315BB1D6F80425131AC4
:10F1500023F07F43B3F5000F10D9C6F840C1D6F8AD
:10F16000403101EB020B0131DDE71B4BD3E8EF1F10
:10F1700041F00101C3E8E21F002AF7D1144B174AFE
:10F18000C3E902451A6000225A60B8F1000F16D098
:10F19000D7E8EF3F43F00103C7E8E23F002AF7D189
:10F1A0004FF48032084BC3F804230B4BD3E8AF3F36
:10F1B000DB0742BF4FF40012094BC3F80021BDE842
:10F1C000F88F00BFB44200200050015001008000C1
:10F1D000D0340020FDFF7F00B042002051AF01007D
:10F1E00000E100E070B54FF0FF3000254FF0FF3137
:10F1F000134C144BC4F80855C3E902014FF4803393
:10F2000002264FF40012C4F804330F4B0121C4F856
:10F2100004631520C3F880212A46F4F733FD152036
:10F22000F4F700FD0123094AA36000212360084888
:10F230001360FFF73BFF3046FEF7ECFC284670BD3D
:10F2400000500150D034002000E100E0B442002022
:10F25000FFFF7F00431C10B51DD001281DDD104AA3
:10F26000104B9042D4BF04461C46FFF795FE0E4A51
:10F27000D2E90031C01AB0F5000F28BF0024094AB6
:10F280000444944228BF1446E01841F10001BDE84F
:10F290001040FFF70BBF034CE7E70124E5E700BF91
:10F2A000FEFF7F00FFFF7F00E034002008B5FFF77E
:10F2B00073FE024B1B68C01A08BD00BFE03400207B
:10F2C00008B503685A090CD0012A12D00E490F481C
:10F2D00040F2472206F0B9FE40F247210A4806F004
:10F2E000ADFE4FF0FF3222FA03F3D907EED50848FE
:10F2F00008E04FF6FF7203F01F03DA40D207E5D5AE
:10F300000360044808BD00BF1F8E0200568D020036
:10F31000002584500028845010B504460269A2B02C
:10F32000C2F880001E49002001F06EFC002201217D
:10F330002A20F4F7A7FC64688422002101A808F0C1
:10F34000EAF96368B3F5803F03D35721154806F007
:10F3500090FE2368B3F5803F03D35721124806F08F
:10F3600088FE00230120219301AA61680432D9405C
:10F37000C90744BF00FA03F142F8041C2168D940D0
:10F38000C90748BF00FA03F103F1010348BFD16385
:10F39000102BEAD101A801F04FFC002022B010BDD3
:10F3A00075B4010093B50200C4B5020038B5054636
:10F3B0000C461AB157210B4806F05BFE0F2C0ED8F5
:10F3C0006B685B68E340DB0709D501230020A400DC
:10F3D000E4B204F1A04404F52834236038BD6FF092
:10F3E0001500FBE7F5B5020038B50F290C46056995
:10F3F0003BD843681B68CB40DB0736D5D5F8843053
:10F40000CB4003F001031AB9E3B96FF077002BE0AA
:10F41000002BFAD155F821301BB95721144806F0BA
:10F4200028FED5F8843013B92A20F4F7FBFB01221B
:10F43000D5F88430A2401343C5F88430E0B201F01F
:10F4400037FC0AE0C8B201F04FFC0122D5F8843045
:10F45000A24023EA0203C5F88430D5F8843013B9FA
:10F460002A20F4F7EDFB002038BD6FF01500FBE714
:10F4700015B6020070B5D1F880600F2804460D461D
:10F48000736803D81B68C340DA0703D457210D48BB
:10F4900006F0EFFDD5F88430E340DB0703D45721B5
:10F4A000094806F0E6FD05EB840255F824503DB10D
:10F4B00021463046AC46BDE870400023126C6047E0
:10F4C00070BD00BF4AB602006BB602002DE9F041E4
:10F4D00012F0FC6F1346D0E9014706690AD035499E
:10F4E0004FF42D72344806F0B0FD4FF42D713148C1
:10F4F00006F0A4FD02F03002302A08D12D4940F276
:10F50000B7222D4806F0A1FD40F2B721EFE703F046
:10F510000212022A08D1274940F2BB22264806F0EF
:10F5200094FD40F2BB21E2E703F00602042A08D171
:10F53000204940F2BF22204806F087FD40F2BF215B
:10F54000D5E713F4402212D09D0308D4194940F2A4
:10F55000C222194806F079FD40F2C221C7E7B2F590
:10F56000402F14D0154A9A4301D183F4402301253A
:10F5700024688D40254223F4801211D10D4940F2B8
:10F58000D2220D4806F061FD40F2D221AFE70949D1
:10F5900040F2C622084806F058FD40F2C621A6E710
:10F5A0003468DB074CBF2C43AC4334603B68BDE898
:10F5B000F0411847A6B60200568D02000100100067
:10F5C00070B502F4C003B3F5C00F0569D0E901645A
:10F5D0000AD1204940F261221F4806F036FD40F270
:10F5E00061211C4806F02AFD43B91A4940F2652200
:10F5F000194806F02AFD40F26521F2E702F0C863DF
:10F60000B3F5800F08D1134940F26F22124806F07B
:10F610001CFD40F26F21E4E7012336688B40334242
:10F6200008D10C494FF41D720B4806F00EFD4FF443
:10F630001D71D6E7160204D52D682B4218BF82F043
:10F64000C062A46902F0C063A446BDE8704002F045
:10F65000B0726047A6B60200568D0200012310B5B5
:10F6600003FA01F1436804691B6819420AD10C4985
:10F670000C4840F23D5206F0E8FC40F23D5108488B
:10F6800006F0DCFC2368194203D022B183681B69B1
:10F6900003E0002AFAD08368DB68BDE81040184711
:10F6A000A6B60200568D02002DE9F74300244FF064
:10F6B000010825461A4E30683779436808FA07F77B
:10F6C0001B681F420AD11749174840F2E44206F06E
:10F6D000BCFC40F2E441134806F0B0FCD0F81090B6
:10F6E000836801A95B689847002809D00FDB08FAF6
:10F6F00005F31C430135042D06F10806DBD10BE0B0
:10F70000D9F80020019B53403B42F3D0EFE745215D
:10F71000064806F0AEFC0024204603B0BDE8F083A6
:10F7200034890200A6B60200568D0200D7B6020048
:10F73000002870B50CBF4FF400164FF098660025F6
:10F74000064C2068217932460135FFF739FF042D38
:10F7500002D008340028F4D070BD00BF3489020004
:10F7600010B54FF02003EFF3118483F31288BFF339
:10F770006F8F1D4803F0DCF840B91C4994221C48E7
:10F7800006F063FC9421194806F058FC164803F073
:10F79000EBF80020FFF7CCFF18B14521154806F023
:10F7A00068FC154B1A78B2B9012214481A7021224C
:10F7B000002304F069F80C4803F0C8F830B90B498D
:10F7C000C2220B4806F041FCC221DCE784F3118819
:10F7D000BFF36F8F10BD0A490548BA2206F035FC09
:10F7E000BA210748D0E700BF68430020908D02008F
:10F7F000568D0200F1B60200A5460020F03400202C
:10F800000FB702002DE9F041074688460025104E4B
:10F8100027FA05F212F0010210D128FA05F3DB07EE
:10F820000ED531793068FFF719FF044640B1452104
:10F83000084806F01EFC2046BDE8F0810122F0E7F2
:10F840000135042D06F10806E2D10024F3E700BFDC
:10F85000148902004DB702002DE9F041FFF724FFA3
:10F8600004463A4BD3E8EF2FC3E8E14F0029F9D122
:10F87000374B384F1A7832BB3E68A64219D0364B08
:10F8800066401B680BB1314698474FF0FF334FF08D
:10F89000FF32324803F09EF8314B1D6835B1043D0C
:10F8A0002B683146204698476D68F7E72B4803F0F0
:10F8B00047F93C6054B1BDE8F0414FF4A472002315
:10F8C000284803F0E1BF00221A70F2E74FF020034E
:10F8D000EFF3118583F31288BFF36F8F224803F093
:10F8E00027F840B921499422214806F0AEFB942123
:10F8F0001E4806F0A3FB1C4803F036F81D4B187891
:10F90000012819D11C70FFF713FF0446164803F0B5
:10F910001DF830B91549C222154806F096FBC221E0
:10F92000E6E785F31188BFF36F8F6CB1BDE8F04156
:10F930004521114806F09DBB10490D488A2206F06A
:10F9400084FB8A210D48D4E7BDE8F081784300208C
:10F9500085260020484300207C4300204C430020A3
:10F9600060430020F034002068430020908D0200A6
:10F97000568D0200A546002068B702000FB70200AE
:10F9800070B500260C4CE2882068217942F40032E0
:10F99000FFF79CFD054648B90136042E04F1080422
:10F9A000F1D1BDE870400F21FFF72CBF452103487E
:10F9B00006F05FFB284670BD1489020085B702007F
:10F9C000054BD3E8AF3F00B10360044811B10268B2
:10F9D0005A400A6003607047784300204443002087
:10F9E0002DE9F8433A4B18603A4D3B480BF033FE93
:10F9F0002E464FF000082F46F288306812F0010FB3
:10FA000014BF1023202331791A4342F48032FFF7C8
:10FA10005DFD044630B14521304806F02AFB204602
:10FA2000BDE8F88308F10108B8F1040F06F10806F3
:10FA3000E2D1064680464FF00109286829794FF443
:10FA40000012FFF7BDFD044610B145212448E4E74C
:10FA50002B7908F1010809FA03F3B8F1040F46EA1B
:10FA6000030605F10805E8D10546DFF878801E4B4E
:10FA7000C8E9013657F835008368DB693BB10122DC
:10FA800041469847044628B145211848C5E76FF01C
:10FA90008504F9E70135042DECD11549154803F02B
:10FAA00009FE0122144B13481A700023002203F0B0
:10FAB00087FE21462046FFF783FFFFF7F5FD0F4B3A
:10FAC000D3E8EF2FC3E8E10F0029A8D0F8E700BF83
:10FAD0007C430020348902004C430020A4B702007C
:10FAE000C6B702006C43002061B70100E6B7020010
:10FAF00059B80100F0340020A546002078430020CA
:10FB000003280A4610B507D945210B4806F0B1FA7B
:10FB10006FF01504204610BD084B03EBC0010979B6
:10FB200053F83000FFF79AFD04460028F2D0452133
:10FB3000034806F09EFAEDE7FFB7020014890200C1
:10FB40004DB702000348452108B506F092FA00209F
:10FB5000F4F7F4FB33B8020030B5816885B0103992
:10FB600021F00704054606F008FF1022014668460A
:10FB700007F0D1FD10226846064907F0C1FD1023A9
:10FB80006A462146284606F0C6FE003818BF012006
:10FB900005B030BD468A020030B50D46816887B099
:10FBA000102302AA1039044606F0A0FE002802DA4B
:10FBB000012007B030BD1022204602A90AF01DFC2A
:10FBC00000283AD110221E4902A807F072FD002831
:10FBD0000CBF012302232B7020460AF0FAFB0123FD
:10FBE00001460DF10702204606F080FE0028DFDB0B
:10FBF0009DF80730204603F00F021B096A702B7135
:10FC000001220DF107010AF0F8FB10B96B78042B03
:10FC100003D901236B7000232B71A2682046183A88
:10FC200022F00702083AA91C0AF0FAFB0028BFD10B
:10FC30002046E91C0AF04DFCBBE70323CBE700BFDD
:10FC4000468A02000E2A13B504460AD90D490E4809
:10FC50004FF4CE7206F0F9F94FF4CE71094806F070
:10FC6000EDF90E29F2D841EA02118DF807100AF0D9
:10FC7000B0FB012301460DF1070220460AF0ECFB20
:10FC800002B010BD55B80200568D02007FB569461E
:10FC9000054606F0EBFD0128044604D16946022022
:10FCA0000AF01DFC044614B1FF2004B070BD05200D
:10FCB00002A90AF014FC012836D12A464921284815
:10FCC00006F0D7F9274B8DF80C40029300229DF8DF
:10FCD00000509DF80860244C294620780AF07FFBEC
:10FCE00048B3314660780AF07AFB20B3A378042B3E
:10FCF00003D09DF8031099421DD1E378042B03D063
:10FD00009DF80B10994216D12379042B0FD16379FA
:10FD1000022B1BD1154A1648492106F0AAF9607931
:10FD2000831E022BC1D9BFE70028CFD0BCE79DF8C6
:10FD300002109942EBD00132032A04F10604CBD120
:10FD40000C48492106F095F90120AEE7032B05D0B8
:10FD5000094A0A49042B08BF0A46DCE7084ADAE7E1
:10FD6000BBB80200030103032EB902009DB80200D4
:10FD700006B9020019B90200A2B80200B4B8020024
:10FD800098B802007FB50E46052001A9F2F746FF9C
:10FD900000283BD1019802A9FFF7FEFE044638B9BE
:10FDA0009DF80850022D1FD0032D07D0012D22D120
:10FDB000019806F09AFD204604B070BD0198FFF747
:10FDC000CBFE04460028F3D101985EB10AF07AFB1D
:10FDD00004460028ECD1002229460198FFF732FFA3
:10FDE0000446E5E70225F6E701982146826806F019
:10FDF000A7FD0324DCE70649064840F2312206F05D
:10FE000024F940F23121024806F018F90124D2E722
:10FE100055B80200568D02004FF47F03D3F830210D
:10FE2000D3F83431072A05D1023B032B02D8024A0A
:10FE3000D05C70470020704751B902004FF050234A
:10FE4000D3F85825034B02F00302D340024A136053
:10FE5000704700BF0020A1076424002008B5FFF709
:10FE6000DBFF58B14F4BD3F8202A3AB90D21C3F824
:10FE7000201A0121C3F81C19C3F81C290022D30041
:10FE800003F57F03D3F80013013107D0D3F8001333
:10FE90000132D3F80433202A0B60F0D1FFF7BCFF06
:10FEA000002876D1FFF7B8FF40B13F4B3F4AC3F877
:10FEB00030254FF050230122C3F858254FF47F031B
:10FEC000D3F83021D3F83431072A09D1023B032B70
:10FED00006D8374AD35C1BB10022364BC3F84C25F9
:10FEE000FFF79AFF50B14FF05023D3F80024D10709
:10FEF00042BF0022C3F81421C3F818214FF47F0336
:10FF0000D3F83021D3F83431072A09D14FF05023E8
:10FF1000D3F80024D20744BF6FF00102C3F80024D5
:10FF2000FFF77AFF18B165221E4BC3F80C274FF478
:10FF30007F03D3F83021D3F83431072A16D11D4B73
:10FF4000D3F82034002B11DA4FF050230322C3F8EA
:10FF5000182501229A60D3F80421002AFBD0002240
:10FF6000C3F804210122DA60C3F81825124AD2F836
:10FF70008C3043F44063C2F88C30104A104B116847
:10FF8000C3F84415D269C3F84C25BDE80840FFF713
:10FF900055BF2922034BC3F80C270322C3F83C2783
:10FFA00080E700BF00400050009003504400EFBEC7
:10FFB0004DB902000020035000ED00E00080FF007A
:10FFC0000060005070B501250268B2FA82F3C3F1F7
:10FFD0001F03DBB205FA03F422EA0404D0E8EF6F52
:10FFE000964204D1C0E8EC4FBCF1000FF6D1EBD142
:10FFF00001480B7070BD00BF0000AD0B10B5036869
:0200000290006C
:10000000CB40DB0710D401238B40026843EA020196
:10001000D0E8EF4F944204D1C0E8EC1FBCF1000FD0
:10002000F6D1F2D1014810BD0148FCE70000AD0B4C
:100030000400AD0B4FF05023002273B5032838D8CD
:10004000DFE800F0020D212C0221C3F80813C3F8E9
:100050000421D3F804210122DA60002409E00121FF
:10006000C3F80813C3F80021D3F800210DF10704E9
:10007000596001238DF80730032800F29680DFE8ED
:1000800000F0214364854FF40071C3F80813C3F8EE
:100090002421D3F8242101225A62DEE74FF4807133
:1000A000C3F80813C3F82021D3F820210122DA6114
:1000B000D3E745494548D82205F0C7FFD821424833
:1000C00005F0BCFF42F210754FF0502694B1D6F8FF
:1000D000183403F003032370D6F81834D90307D576
:1000E0009DF80700012803D10AF037FA013DEDD150
:1000F00002B070BDD6F81834DA03F9D501200AF041
:100100002CFA013DF6D1F3E742F210754FF050267C
:100110008CB1D6F80C3403F001032370D6F80C34FC
:10012000DB03E5D59DF807000128E1D10AF015FAB7
:10013000013DEDD1DCE7D6F80C34D803D8D5012049
:100140000AF00BFA013DF6D1D2E742F210754FF0FA
:1001500050268CB1D6F85C3403F001032370D6F836
:100160005C34D903C4D59DF807000128C0D10AF03A
:10017000F4F9013DEDD1BBE7D6F85C34DA03B7D52D
:1001800001200AF0EAF9013DF6D1B1E742F210751B
:100190004FF05026D6F85434DB03A9D57CB90120A2
:1001A0000AF0DBF9013DF5D1A2E70949074840F221
:1001B000473205F04AFF40F24731054880E79DF895
:1001C00007000128ECD093E755B90200568D0200D4
:1001D00092B9020008B550B90A490B4840F215120D
:1001E00005F033FF40F21511064805F027FF074BD5
:1001F0001A7922B90122186005481A7108BD05480C
:10020000FCE700BF55B90200568D02008043002074
:100210000000AD0B0C00AD0B08B50F4B1B7953B9AB
:100220000E490F484FF4977205F00FFF4FF4977186
:100230000A4805F003FF0520F3F716FD10B9052065
:10024000F3F7F0FC4FF050230122C3F81825C3F850
:100250001425C3F8802508BD8043002055B902004D
:10026000568D020008B5384B1B7953B937494FF406
:10027000B472374805F0E9FE4FF4B471334805F025
:10028000DDFE4FF05023032854D8DFE800F00231A0
:100290003B47D3F81824D3F81814C90312D502F039
:1002A0000303022B1DD14FF05022C2F81835002352
:1002B000C2F80431D2F804310223C2F80433012316
:1002C00093600DE0D3F81424D2070FD5D3F81C2483
:1002D00002F00302013A012A05D80222C3F80423DE
:1002E00008BD012B02D00020FFF7A4FE0123DAE7AE
:1002F0000022C3F80021D3F800210122C3F804230F
:100300001A60EDE70022C3F82421D3F824214FF42A
:100310000072C3F8042301221A62E1E70022C3F845
:100320002021D3F820214FF48072C3F80423012246
:100330009A61D5E705494FF4D372054805F085FE6B
:100340004FF4D3719AE700BF8043002055B90200F3
:10035000568D020008B5094B1B7953B90849094865
:1003600040F2AD1205F071FE40F2AD11044805F007
:1003700065FEBDE80840FFF75DBE00BF804300207A
:1003800055B90200568D02004FF0502310B5D3F836
:10039000002152B10020C3F80001D3F8002101224E
:1003A000C3F80823234B1B6898474FF05023D3F81A
:1003B00004218AB10022C3F80421D3F80421D3F820
:1003C0001824D3F8181402F00302012A4FF0020196
:1003D00028D1C3F818159A604FF05023D3F8202184
:1003E00062B10022C3F82021D3F820214FF480729B
:1003F000C3F808230F4B04201B6898474FF0502385
:10040000D3F82421AAB10022C3F82421D3F824214F
:100410004FF40072C3F80823064B0520BDE81040D6
:100420001B681847C3F80813024B01201B68984744
:10043000D2E710BD8043002001460148FFF7C2BD4E
:1004400068240020034B083033F81000C0F340103C
:10045000704700BF6C240020044B083033F81000B4
:1004600010F01C0018BF0120704700BF6C24002052
:10047000034B083033F81000C0F34000704700BF52
:100480006C24002070B50D4C00F1080334F81330D3
:100490000546DA050E4607D5C3F3432304EBC30232
:1004A000526854F833309847A3682BB13146284638
:1004B000E268BDE87040184770BD00BF6C240020A2
:1004C00010B5184A083032F81030D9051DD5C3F3DD
:1004D000432123F4F85322F81030002002F10E04D7
:1004E00034F8023F13F4807F03D0C3F343239942CF
:1004F0000BD001303028F3D100230B4842F83130C3
:10050000FFF77CFD094B984200D110BD084909480E
:100510004FF4997205F099FD4FF49971044805F074
:100520008DFD00BF6C240020E02400200000AD0BF6
:10053000DBB90200568D020038B50246FFF782FF94
:100540000B4C02F1080560B1002134F815305B0B4B
:100550009B0003F1A04303F55043C3F81015C3F803
:1005600010151046FFF7ACFF002324F8153038BDF6
:100570006C24002008B502680146104609F0EFFF20
:1005800050B90F4940F247220E4805F05EFD40F297
:1005900047210B4805F052FD02F01F0352090B6082
:1005A0000AD0012A0AD006494FF41372054805F013
:1005B0004CFD4FF41371ECE7034808BD0348FCE71A
:1005C0001F8E0200568D02000025845000288450A2
:1005D000F0B5044617461D4685B0D9B109F0D0FFE5
:1005E00000BB0B46CDE900008DF80E008DF80F0022
:1005F0000DF10F020DF10E01204609F0CCFF444A27
:1006000004F1080132F8113023F0020343F0010332
:1006100022F811306FB320463E787A68FFF728FF42
:1006200010B1DAB13B4826E0394804F1080C30F843
:100630001C1021F02001C904C90C20F81C106AB15B
:10064000032EEFD87B681F78BA0002F1A04202F5B2
:10065000504296B9C2F81065C2F810652C4A04F1F0
:10066000080132F8113023F01C0343EA860322F814
:10067000113015BB284805B0F0BDD2F8103541EA5D
:10068000473123F00303C2F81035D2F8103541F09A
:10069000200123F44F3323F44073C2F810352302B2
:1006A000D2F810E503F47C5343EA064343EA0E0311
:1006B000C2F8103520F81C10D0E72046D5E90067B5
:1006C000FFF7FEFE002ED5D0114DD5E9002396424E
:1006D00001D19F4219D011480DF10F01FFF772FCB3
:1006E0000D4B9842C7D19DF80F2005EBC20304F1D2
:1006F00008005F6035F8103045F8326043EA422365
:1007000043F4807325F81030B4E70022EDE700BF12
:100710006C2400200400AD0B0000AD0BE024002091
:10072000F0B50446154685B021B3FFF7A1FE20B908
:100730002046FFF787FE002861D12046FFF78CFE98
:1007400010B14B78012B5AD001238DF80F300023C4
:100750004A1CCDE9001320468B1C0DF10F0109F056
:100760001AFF284A04F1080132F8113043F003035C
:1007700022F8113015B9244805B0F0BD2046FFF726
:1007800077FE00283BD095F800C0002361461D4E3F
:1007900004F1080736F81700890020F0200001F165
:1007A000A041C00401F55041C00CC1F8103526F835
:1007B0001700C1F810356A78002ADCD0D1F810355E
:1007C000AD7823F4991323F4F853C1F81035D1F818
:1007D00010E5230203F47C53120402F4403243EA8E
:1007E0000E0313432A0502F4801240EA4C301343EF
:1007F00040F02000C1F8103526F81700BBE7034889
:10080000BAE700BF6C2400200000AD0B0400AD0B64
:10081000014BC3E9020170476C240020024608B571
:1008200051B90C490C4840F2352205F00EFC40F25B
:100830003521084805F002FCFFF704FE38B1074BEC
:10084000083233F8123006485B0B0B7008BD0548C0
:10085000FCE700BFDBB90200568D02006C240020CB
:100860000000AD0B0400AD0B38B50F4C94F8785078
:10087000BDB96022294604F1100006F04CFF0D209E
:10088000F3F7D0F9094B0A48C3F87C51D3F87C211F
:100890004FF00042C3F80423012384F878306367E3
:1008A00038BD0448FCE700BF6C24002000D0005095
:1008B0000000AD0B0500AD0B034B93F8780000383A
:1008C00018BF0120704700BF6C240020014601487A
:1008D000FFF794BBDC24002001460148FFF772BB00
:1008E000DC24002037B50446FFF7B6FD50B92C498B
:1008F00040F2DF322B4805F0A8FB40F2DF312848F8
:1009000005F09CFB2046FFF79DFD274A04F10805F2
:10091000F8B12046FFF7ACFDD8B932F81520520BDC
:10092000930003F1A04404F5514403F1A043206077
:1009300003F550432068D3F8100540F00100C3F8D8
:10094000100521B101239340184AC2F8043303B0C3
:1009500030BD41B9124940F2EE32124805F075FB44
:1009600040F2EE31CBE732F81530C3F38203042BAB
:1009700011D0052B11D001A80194FFF7FBFD019BBD
:100980000169D94001F001010231204603B0BDE800
:10099000304009F04DBE0321F7E70221F5E700BF23
:1009A000DBB90200568D02006C24002000D00050FC
:1009B00008B50246FFF746FDC8B11046FFF758FDDF
:1009C000A8B90E4B083233F8123001225B0B9A4063
:1009D0000B499B0003F1A043C1F8082303F55043E2
:1009E000D3F8102522F00302C3F8102508BD00211A
:1009F000BDE80840104609F01BBE00BF6C24002073
:100A000000D0005013B5104B00F1080233F812303B
:100A10000446DB0716D5FFF7CBFF2046FFF78CFD1A
:100A200001A80194FFF7A6FD019B00EB8300D0F81D
:100A3000003203F0E04343F00203C0F80032034801
:100A400002B010BD0248FBE76C2400200000AD0B93
:100A50000400AD0B2DE9F04F002601223446644B13
:100A60006448654987B01D6835B1D0F80453154214
:100A70001EBF1C601D68164304338B424FEA4202BE
:100A8000F1D1DFF870A1DAF87C31002B00F093800F
:100A9000DFF86881D8F820300493C8F82030584B2C
:100AA0001A6A05921A624FF000090DF1100B4FEA15
:100AB000491300934AE094FAA4F4B4FA84F4009B36
:100AC000504A1C4404F1080332F813700123E00873
:100AD00004F0070103FA01F11BF80030BA0823EA19
:100AE00001030BF8003003A801920394FFF742FDC5
:100AF000039B019A803350F82330C7F382055207D5
:100B00002F46C3F301432BD539462046DDB2FFF70C
:100B1000B9FC03A80394FFF72DFD039B803350F825
:100B20002330C3F301439D4207D10021204609F041
:100B30007FFD2946204609F07BFD03A80394FFF7BB
:100B400019FD0122039B02FA03F303625BF82940BB
:100B5000002CB0D1B9F1000F1DD14FF00109A6E76B
:100B6000022B0CD10321204609F062FD05F005039C
:100B7000012BE2D139462046FFF784FCDDE7022154
:100B80002046019309F054FD032DF3D0019B032B64
:100B9000D3D1022DEDE7CAF87C41DAF87C31D8F8E0
:100BA000203017490493C8F820300A6A134305928D
:100BB0000A627FF478AF012416B907B0BDE8F08F60
:100BC00096FAA6F3B3FA83F304FA03F29B0003F157
:100BD000A04303F55043D3F81005D3F81015C0F324
:100BE0000520C1F3014126EA0206FFF74BFCE3E7CB
:100BF00000D1005000D0005020D10050002584507A
:100C0000002884506C24002070B5084C0E462379CF
:100C1000154643B92A20F3F705F801230448237148
:100C20002660A56070BD0348FCE700BF8843002034
:100C30000000AD0B0C00AD0B38B540B9184945228A
:100C4000184805F002FA4521154805F0F7F9164B4A
:100C50001B79012B06D012494622124805F0F5F9FE
:100C60004621F1E70023114A50F8234003F5A27111
:100C70000133102B42F82140F6D100230B4A00F13A
:100C80003C0103F5B27451F8045F0133102B42F8B4
:100C90002450F6D1D0F88030C2F8043338BD00BFFC
:100CA00025BA0200568D02008843002000A00250A1
:100CB00008B5094B1B79012B08D0084908486B225D
:100CC00005F0C3F96B21054805F0B8F9054A8340E2
:100CD000C2F8043308BD00BF8843002025BA0200D3
:100CE000568D020000A0025008B5094B1B79012B5C
:100CF00008D008490848712205F0A7F97121054874
:100D000005F09CF9054A8340C2F8083308BD00BFCE
:100D10008843002025BA0200568D020000A0025030
:100D2000F8B501260027124B124DD3F80C4304B935
:100D3000F8BD94FAA4F0B0FA80F006FA00F30F2898
:100D400024EA03040ADD0C490C4840F2E71205F0DE
:100D50007CF940F2E711084805F070F9084B820071
:100D60009F502B68002BE2D0A9689847DFE700BFAF
:100D700000A002508843002060BA0200568D020095
:100D800000A102500022034BC3F88425C3F80425B8
:100D9000704700BF00900350044AD2F80034DB07CC
:100DA000FBD50160BFF35F8F704700BF0090035019
:100DB000B0F5801F08B513D2C0F30B03DBB90222D4
:100DC0000E4BC3F88425C3F804254FF0FF320260B0
:100DD000D3F80024D207FBD5FFF7D4FF084808BD9D
:100DE000084909484FF4837205F02FF94FF48371D5
:100DF000044805F023F90548F1E700BF00900350CF
:100E00000000AD0B92BA0200568D02000A00AD0B35
:100E1000B0F5801F08B511D300F17F4303F50043FF
:100E2000B3F5805F0AD311494FF4CA72104805F038
:100E30000CF94FF4CA710D4805F000F9830708D08A
:100E40000A4940F295120A4805F0FFF840F2951160
:100E5000F1E70122074BC3F88425C3F80425FFF707
:100E60009BFFBDE80840FFF78DBF00BF92BA0200AC
:100E7000568D02000090035070B5424D95F83040F9
:100E800044B941496822414805F0DFF868213E48ED
:100E900005F0D4F830B93C4969223C4805F0D5F852
:100EA0006921F4E700F06046B6F1005F65D186077E
:100EB00063D1012C01D09C4261D12C6804BB022B70
:100EC000334B0BBFC3F81025C3F80425C3F8140532
:100ED000C3F808050BBFC3F81815C3F80C15082292
:100EE00004220021C3F8001102F1A043012203F5FE
:100EF0002C331A60264AD2F80031002BFBD00DE0CB
:100F0000AE68234C66B1022BE8606961EA612DD1BD
:100F1000C4F81025C4F81405C4F818151D4870BD90
:100F2000022B85F830302961AA61A8600CBFC4F893
:100F30001025C4F804254FF000020BBFC4F81405B7
:100F4000C4F80805C4F81815C4F80C1508BF082320
:100F50000F4918BF0423C1F80021012203F1A04367
:100F600003F52C33C1F804231A60D7E7C4F804252D
:100F7000C4F80805C4F80C15D0E70748CFE70748C0
:100F8000CDE700BF94430020CEBA0200568D020088
:100F900000B002500000AD0B0A00AD0B0B00AD0B12
:100FA00038B56424064DD5F8003133B90A2009F06C
:100FB000D4FA013CF7D1034838BD0348FCE700BF31
:100FC00000B002500700AD0B0000AD0B084B9A6853
:100FD0005A621A699A629A69DA62DA689A6032B178
:100FE0005A691A61DA699A610022DA6070477047BB
:100FF0009443002008B543090CD0012B1DD01349A0
:10100000134840F2472205F020F840F247210F48EC
:1010100005F014F84FF0FF33C340DA07EFD50D4A5F
:1010200002EB8002D2F8003203F0E04343EA0121F0
:1010300041F00201C2F8001208BD4FF6FF7300F044
:101040001F00C340DB07DAD5034AE9E71F8E020021
:10105000568D0200002584500028845010B50E4B98
:101060000238D3F83C26D3F83836072813D8DFE8FF
:1010700000F0110F0D0B0A080604100EC871100CB9
:101080008871100A48710A711A0ECA701A0C8A7097
:101090001A0A4A700B7010BD00B0025002380728BF
:1010A0001FD8DFE800F02927251123211F04CB7961
:1010B0001B068A7943EA02434A7943EA02230A7902
:1010C00013430E4AC2F83C36CB781B068A7843EAB3
:1010D00002434A7843EA02230A781343074AC2F8D4
:1010E000383670470023E4E70023E5E70023E6E70E
:1010F0000023EBE70023ECE70023EDE700B002500C
:10110000F8B50D461646044650B96D496D484FF482
:10111000887204F09AFF4FF48871694804F08EFFDA
:10112000694F97F83030002B40F0C680C27C12B176
:10113000037D002B70D12079FF2800F0BF806379F8
:10114000FF2B00F0BB80A379FF2B00F0B780E17983
:10115000FF2900F0B3806368DFF870C123F07F439C
:10116000634540F0AB800E2940F0A880237AFF2B26
:1011700002D00F2B40F0A280637AFF2B02D0102BFD
:1011800040F09C80D2B90321FFF734FF032160793E
:10119000FFF730FF0321A079FFF72CFFE07903214F
:1011A000FFF728FF207AFF2802D00321FFF722FF54
:1011B000607AFF2802D00321FFF71CFF237D5BBB71
:1011C0002379FF2B14BF1A464FF0FF32404BC3F870
:1011D00024256279FF2A08BF4FF0FF32C3F8282583
:1011E000A279FF2A08BF4FF0FF32C3F83025E27919
:1011F000FF2A08BF4FF0FF32C3F83425227AFF2AB6
:1012000008BF4FF0FF32C3F83825627AFF2A08BFC3
:101210004FF0FF32C3F83C2523682D4AC2F8403511
:10122000237BE07AA17A9B0143EAC0030B43617BF5
:1012300043EAC113C2F84435617CD2F84435B1BBEE
:1012400043F44033C2F844354FF4C063C2F840362B
:10125000D2F80016A37B21F07F4121F0FF010B4360
:10126000E17B43EA0163217C43EA4163617C43EA19
:101270000173C2F80036E37CC7E9005687F83130C5
:101280000123C2F8083315B12B20F2F7CBFC002163
:101290000122C7E902110E4B87F83020C3F8002560
:1012A000C3F800111A60BDE8F840FFF779BE23F4D7
:1012B000003343F48033C5E70648F8BD0648FCE731
:1012C000CEBA0200568D02009443002011120D0088
:1012D00000B002500500AD0B0400AD0B70B5144614
:1012E000254A054692F8302052B924494FF4A77296
:1012F000234804F0AAFE4FF4A771204804F09EFE94
:10130000012A36D100221F4EC6F8002111B14078C3
:10131000FFF7C4FE0123C6F80833AB786A781B03D5
:1013200043EA02232A781343EA7843EA42332A79CC
:1013300043EA82336A7943EAC233C6F83436FFF7A8
:101340002FFE114B98420AD12B798BB90B4940F2F1
:101350006B120B4804F079FE40F26B11CDE70023CD
:10136000C6F800311CB121466878FFF777FE0748C0
:1013700070BD0748FCE700BF94430020CEBA0200CE
:10138000568D020000B002500700AD0B0000AD0BFF
:101390000B00AD0B1FB500230C4A02A802920DF101
:1013A000070211468DF80730ADF80C30FFF796FFB5
:1013B000074B984206D19DF8073013F0010F054BFB
:1013C00018BF184605B05DF804FB00BF0502000118
:1013D0000000AD0B0B00AD0B2DE9F843294E96F83C
:1013E000303053B9284929484FF4FF7204F02DFEDC
:1013F0004FF4FF71244804F021FE2B20F2F720FC6B
:10140000234BD3F8342602F44032B2F5803F04BFB8
:10141000204AC3F834260122C3F808231A610022A7
:10142000C3F80025C3F8002196F8312022BBD3F879
:101430002405D3F82895C0B2D3F83085D3F8347595
:10144000D3F83855D3F83C4509F00AF95FFA89F02A
:1014500009F006F95FFA88F009F002F9F8B209F02C
:10146000FFF8E8B2FF28E4B201D009F0F9F8FF2C48
:1014700002D0204609F0F4F8002386F83030BDE8A9
:10148000F88300BF94430020CEBA0200568D0200BC
:1014900000B002500001030010B51A4A92F8303033
:1014A00053B9194919484FF40A7204F0CEFD4FF4AC
:1014B0000A71154804F0C2FD8C071ED114680CB1E6
:1014C000012B1CD1042382F83030114BC3F81C15BA
:1014D0000021C3F82005C3F800110121D96010686C
:1014E00040B9D3F800110029FBD0012382F8303035
:1014F000084810BDC3F80413FAE70748F9E707489E
:10150000F7E700BF94430020CEBA0200568D0200D8
:1015100000B002500000AD0B0A00AD0B0B00AD0B8C
:1015200010B5174BD3F80021E2B10022154CC3F8D7
:10153000002194F83020032A15D0042A15D0022A5D
:1015400004D1012384F82030FFF740FDA36813B9CC
:10155000012384F83030D4E900310020984700237B
:1015600084F8203010BD0223ECE7032284F8202009
:10157000D3F81C256262D3F8203584F82830E5E7DB
:1015800000B00250944300202DE9F0410E4617466A
:101590000C4D55F8184FAC4203D16FF01200BDE866
:1015A000F081314654F8440CA4F1440806F062F886
:1015B00030B9C7F800804046BDE8F04109F056B99F
:1015C0002468E8E7C843002010B5D0E909124A6052
:1015D000416A00F124031160C0E9093343680446FD
:1015E00003B19847054B1A78062A05D95B681BB1E9
:1015F0000720226802499847002010BDC8430020F8
:101600000ABB02002DE9F04107460D460B4E56F885
:10161000084FB44202D16FF001000AE0394654F895
:10162000240CA4F1240806F025F820B91DB1C5F852
:101630000080BDE8F0812468EBE700BFC8430020CC
:1016400010B5044610B96FF0150010BD00680028F1
:10165000F9D005F0FFFF0028F5D000212068FFF742
:10166000D1FFC8B104F11C03C4E907330C4B04F1EA
:101670002402D96803F10800DA60A16260620A609E
:101680001A78062A01D95B680BB90020DDE707202C
:10169000226804499847F8E76FF01000D5E700BFCB
:1016A000C84300200CBB0200014610B508B14068D9
:1016B00040B907490748512204F0C7FC51210448AA
:1016C00004F0BCFCC36813B1BDE81040184710BD5E
:1016D0001FBB0200568D020010B50446006810B909
:1016E0006FF0150010BD05F0B5FF0028F8D0A36815
:1016F000012BF5D8064B04F144016360054BDA6910
:1017000003F118006064A264D96100201160E9E768
:10171000E8240020C843002038B505460D4C20229F
:101720002046002105F0F7FF2B682846636023461A
:101730002A7903F8082BC4E9023304F11003C4E941
:10174000043304F11803C4E90633BDE8384000F05F
:101750000FB800BFC843002008B500F011F8BDE87D
:10176000084020220021014805F0D5BFC8430020D1
:1017700008B50248FFF764FF002008BDE8240020F8
:101780000148FFF721BF00BFE82400200EB4431E2C
:10179000062B33B588BF0020094B05AC54F8045B19
:1017A00053F82010074804F08EF92146284601948A
:1017B000EFF7ECFA02B0BDE8304003B0704700BF6D
:1017C00054890200E69902002DE9F04F9A46836A97
:1017D00006469342174687B041D300254FF0180BB9
:1017E000BD4203D1002007B0BDE8F08F0BFB05F828
:1017F000D6F82C90B26909EB0804231D0593CAB9E9
:10180000606961680368B4F80CC0C91AA3680CF178
:10181000030E5C1E04EB0C145B4204EB4E041C40F4
:1018200004EBCC0384680633A14228BF4FF0FF319C
:1018300008F0E8FF59F8083030460293336AA9B23D
:101840001B6A0193109B53F8253000935AF825200A
:10185000059B09F050F80028C5D10135C0E70148C3
:10186000C1E700BF40F4FFFF10B5044690B1828C81
:1018700043899A4209D0084B1A78032A05D95B6834
:101880001BB142680549042098472046BDE8104036
:101890000AF085B810BD00BFC8430020EEBB0200AF
:1018A00030B544898C4212D9036A013C5D882C40D2
:1018B00003EBC40359609A60BFF35B8F026A5388DD
:1018C00001335380C38C0133C384002030BD0148F1
:1018D000FCE700BF41F4FFFF70B4039E144658B10B
:1018E000006A48B143B1013406D0002E04DB846F96
:1018F00014B1A44670BC6047014870BC704700BF7B
:101900002DF8FFFF70B4039E144660B1006A50B119
:101910004BB1013407D0002E05DBD0F8884014B15C
:10192000A44670BC6047014870BC70472DF8FFFFAB
:1019300070B50C46114605461E460C4B2022002968
:1019400008BF1946204605F071FE049B6662A3623B
:10195000059B2562E362069B23636A6804F13403F6
:10196000C4E90D526B60A26B136070BDC1B302007D
:101970002DE9FF47DDF834900D4692461F46064696
:1019800000286CD000296AD0B9F1000F67D001F1AE
:101990005808404609F018F9781C40D1AC6C05F1A4
:1019A000480314F001040BD000240134802C54D0DF
:1019B000620953F8222004F01F01CA40D107F4D471
:1019C0000121600953F8202004F5806704F01F040A
:1019D000A1400A4343F820200E9B5246CDE90193D3
:1019E0000C9B3146009328463B46FFF7A1FF40463B
:1019F00001F0F6F9347874B195F890405CB1B36AAF
:101A000001332ED10021304609F00DF9044610B102
:101A1000304609F0DFF8204604B0BDE8F087B7F59E
:101A2000806FD9D3A7F580637F2B05F148010FD8CC
:101A3000580951F8204003F01F0324FA03F2D2079B
:101A40000BD4012202FA03F3234341F82030C3E709
:101A5000054C404601F0C4F9DDE7044CF9E7024CBF
:101A6000D9E70024D7E700BF2DF8FFFF29F8FFFFD3
:101A70002DE9F041A3F1100853F8087C002388B049
:101A80000693ADF81E301023CDE904120E9D0446D6
:101A9000D0F8AC00ADF81C5001688668A8EB0101D5
:101AA000B14228BF4FF0FF310DEB030208F070FE8A
:101AB0001028BFB20AD023494FF4D672224804F04E
:101AC000C4FA4FF4D6711F4804F0B8FA04F158066E
:101AD000304609F038F9D4F8A0309B69CBB9D4F876
:101AE0009420D4F8A030D4F8A8009B69C3B9CDE9FC
:101AF0000282CDF80080012202A908F029FFA8B1D6
:101B0000104940F2B912104804F09FFA40F2B9119E
:101B1000D9E73946D4F8A80008F0B0FF0246E0E75C
:101B2000012B03D13946FFF7BBFEE8E7D4F8A80044
:101B300008F0FBFF304609F004F9284608B0BDE87C
:101B4000F08100BF10BC0200568D02002DE9FF415C
:101B500003685F6A07F15806304609F0F4F8384622
:101B60000DF10A0203A909F061F90446304609F0B3
:101B7000E8F8002C4ED0BDF80A303046A36009F0DA
:101B8000E2F84FF0FF3300213846626809F07FF831
:101B90000546304609F0D5F8E5B1AB6AE96B01338B
:101BA00008BF2368284608BFAB622368A28900915A
:101BB000D5F82C8004F11001C04700280ADA174933
:101BC000174840F2432204F040FA40F24321134800
:101BD00004F034FA304609F0B6F8A368002B06DBAF
:101BE00021463846BDF80A30039A09F036F93846DE
:101BF0000DF10A0203A909F019F9044618B130469B
